:020000040000FA
:10000000D8100020A5020000B7020000B9020000CD
:1000100000000000000000000000000000000000E0
:10002000000000000000000000000000BB02000013
:100030000000000000000000BD020000BF02000040
:10004000C1020000C1020000C1020000C1020000A4
:10005000C102000000000000C1020000C102000057
:10006000C1020000C1020000C1020000C102000084
:10007000C1020000C1020000C1020000C102000074
:10008000C1020000C1020000C1020000C102000064
:10009000C1020000C1020000C1020000C102000054
:1000A000C1020000C10200000000000000000000CA
:1000B0000000000000000000000000000000000040
:1000C00000F002F800F040F80CA030C808382418FE
:1000D0002D18A246671EAB4654465D46AC4201D180
:1000E00000F032F87E460F3E0FCCB6460126334272
:1000F00000D0FB1AA246AB46334318475C360200D9
:100100007C360200103A02D378C878C1FAD8520778
:1001100001D330C830C101D504680C6070470000BD
:100120000023002400250026103A01D378C1FBD813
:10013000520700D330C100D50B6070471FB5C046D1
:10014000C0461FBD10B510BD00F004FF1146FFF7FB
:10015000F5FF00F0CBF800F01CFF03B4FFF7F2FF4F
:1001600003BC00F021FF0000401E00BF00BF00BF25
:1001700000BF00BF00BF00BF00BF00BF00BF00BF87
:1001800000BFF1D170470000401E00BF00BF00BF9C
:1001900000BF00BF00BF00BF00BF00BF00BF00BF67
:1001A00000BFF1D17047000070B505460C461646F9
:1001B00002E00FCC0FC5103E102EFAD2082E02D34B
:1001C00003CC03C5083E042E07D301CC01C5361F5E
:1001D00003E021782970641C6D1C761EF9D270BD75
:1001E0002749264808607047264A108CC0B201286B
:1001F00017D1918C090714D1118D09060B0F03D16A
:10020000938D1B061B0F0FD0090F012903D1938D6E
:100210001B061B0F08D0032903D1918D0906090F76
:1002200002D0012807D015E0184917484860C813C4
:100230001749886102E0908C00070BD1108D0006F1
:10024000000F042806D1908D0006000F02D111493D
:10025000012088601048808D00070DD40F48104998
:10026000C26A4A62026B8A62426BCA62826B0A632A
:10027000C06BCA0510434863704700000024F400B7
:1002800000000020C00F00F0DFFF07C000050040A5
:10029000006C00400006004080000010C00000100C
:1002A000001700400A48026803210A430260094817
:1002B000804709480047FEE7FEE7FEE7FEE7FEE766
:1002C000FEE7000005480649064A074B7047000054
:1002D00024050040E9010000C1000000D800002012
:1002E000D8100020D8080020D8080020F0B500253C
:1002F00083B001203E4900902E462C4608603D4ABE
:10030000294615603C4A1723D360192353613B4BA0
:1003100053623B4B9D60DD615D6204231360394A8B
:100320005160394988600860384908603849086078
:10033000384F0102F9600103B96037490860374955
:1003400008608020B8603648FFF70EFF8020F86014
:1003500000F0FDFA00F087FB00F092FC8020B8600E
:1003600000F0A1FB01204003B8600199681E00293C
:100370003BD1234F00F0FEF8B9680029FAD00021E4
:10038000B9601D498969002EC9B206D02A461532C6
:10039000904206D90C020546ECE701260C02054600
:1003A000E8E70C43A1042206A3070026A00B890E50
:1003B000920E9B0F032B00D11B1F00F03CF96846E7
:1003C00000F0DEF90028D5D000980B4A0104090E90
:1003D000D161F9690129FCD10021F961C0B2D06174
:1003E000F8690128FCD1F961C4E703B0F0BD000051
:1003F0005C070050640700500025004000A04E003C
:100400000021004000230040002000402007005051
:1004100030070050000500501C0700503407005002
:1004200040420F00F9490A78012A05D8002805D072
:10043000012808D002280AD000207047F4488861BB
:100440000820487007E0F3488861092002E0F2487C
:1004500088610A20487001207047EC4A41B2137845
:10046000012B04D828312D2901D2810701D0002089
:100470007047506101207047F0B4E84800240460E0
:10048000012581050D6001680029FCD0DF498869DC
:100490004560C5600522120282185460C31DF933FD
:1004A0001C645C649C64DC64012303261B04360228
:1004B00086197360DB111D50042313614B6B1364A9
:1004C000FF230533536405600C614A69FC20134621
:1004D000834308D150B2042805DC2823D84202DB2C
:1004E0000B7A032B02D9F0BC04207047CC4E0320BA
:1004F000B060CC480460CC480461CC4E35610769DB
:10050000002FFCD0046174603460C9488C81C260E3
:100510000361426A120A12024262436A8A6A160E32
:10052000334343621202C2610563C4624A79CB79E4
:1005300012021A4342630A79CB7812041B021A434F
:100540008B781A4342618A8C0B8C52061B061A4325
:100550008B8B1B041A438B791B021A432532826151
:100560004C72B4480D700169102211430161F0BC56
:1005700000207047F8B5AF490869102210430861A0
:100580000127A24C0025A848C16800292CD0C560CD
:10059000A949022008602078042825D1A348476093
:1005A000A648006801281BD1A548017842780907B0
:1005B000090F022914D8252A12D800291CD0012994
:1005C00026D055230021002A07D94618B6789E4226
:1005D00006D1491CC9B29142F7D3A089401CA08121
:1005E0002721974800F0AFFCA069FF300130016C73
:1005F00000290FD00564C6E79249801C00F010FC6A
:10060000002803D000200028E7D1E9E70120FAE71D
:100610000F23D7E7406C0028B5D0A069FF30013028
:1006200045646078C006C00E874083480760206933
:10063000401C2061F8BDF8B516460A46734DF1B26C
:10064000A972AB630124EA636C720027EF812F78F3
:10065000002F08D0002808D003280AD0012F13D07B
:10066000EC810220F8BD0520F8BD00F0B2F80020B2
:10067000F8BD2846012FF3D081890122D20311430E
:10068000E98100F0A6F814E0272A02D9EC810120C4
:10069000F8BD0027AF81012802D002280BD008E066
:1006A0002721674800F04FFC012000F071F804207A
:1006B00028700020F8BD252902D9EC810320F8BD5F
:1006C0001F073F0F5E485B1C0770584F417026D0D4
:1006D000012B06D0022B0AD0032B0ED0EC81042074
:1006E000F8BD32465749801C00F0C7FB0AE00F22D4
:1006F0003146801C00F002FC04E055223146801C8B
:1007000000F0FCFB002000F043F8A9694448FF31E9
:10071000413101614761446002202870C9E7002E21
:100720000CD0012E0AD0022E12D0032EC1D1002AE5
:1007300018D0012A1AD0022A1DD00FE0002000F0A4
:1007400027F841490320086036490C603C60E4E723
:1007500050B228302D2801D2900701D00420F8BDD6
:100760006A61A6E72A48A861082002E02948A86132
:10077000092068709DE72848A8610A20687098E7FA
:1007800022490246487A00234B72C989116070479A
:1007900070B42D4900240C601C4B2549DA6A8A6329
:1007A0001A6BCA63DA6B5200921C8A60244A4A6050
:1007B0001D4A14601B4E03253560002805D0D46007
:1007C0001A490120486070BC70475869C86070BC05
:1007D000704710B41C480022026011480124846054
:1007E00002614261032181600E4802600E4802618D
:1007F0000E4B1C6101690029FCD002615A601A602D
:1008000002488281047010BC704700000400002080
:10081000008000400090004000A000400001004027
:1008200000F501400012004000110040001000409F
:100830000015004000ED00E080E200E00014004000
:1008400050000020B60F000040150040F0B596465D
:100850008C4602002BD0F848FA49F84E0123F84F95
:1008600000250C15002A33603B600D6021D0311D3E
:100870000B600B2201198A600F22CA6009220A61EB
:10088000F1491A038A600121090702195162614680
:10089000002906D001291AD002291AD003291AD01A
:1008A00000217446002C18D01943516516E0E74822
:1008B000D2E7E7490B600B2201198A600F22CA6058
:1008C00009220A610121E04A09079160DBE7022160
:1008D000E7E70421E5E70621E3E75165FF21093158
:1008E0000D501360F0BDF0B594460024D74A9E46E3
:1008F0002546904201D11C2300E00C2301229A409E
:10090000D14BDA6000291ED91B15C718FF30013002
:100910006646765DFE610326360300E0641C83684C
:10092000002B01D1B442F9D3B44203D1C64882604E
:100930000020F0BD00268660BE6973465E556D1CC2
:10094000ADB28D42E4D3C04882600120F0BDF0B565
:10095000002283B011461046FFF778FF0027009071
:10096000002824D00124B84D2407EC60AB21009866
:1009700000F0FBF9AC601E20FFF706FCEC609F2145
:10098000009800F0F2F9009800F00DFA019000983C
:1009900000F009FA0602009800F005FA304301461B
:1009A000AC600198EF2802D1AA48814204D0AA483D
:1009B0000770002003B0F0BD012003B0F0BD70B59A
:1009C000002211461046FFF741FF00280CD00124F9
:1009D0009D4D2407EC60B92100F0C7F9AC600320FD
:1009E000FFF7D2FB012070BD9B490020087070BD4D
:1009F000F3B500220C4681B011461046FFF726FFE2
:100A00000090002829D001258F4E2D070022114685
:100A10001046FFF71BFF070021D0F560052100F00D
:100A2000A4F9384600F0BFF9B560C007EED100F078
:100A3000D9F9F5600199009800F097F92002010EAC
:100A4000009800F092F92004010E009800F08DF952
:100A5000E1B2009800F089F9B56003B0F0BD7E49BD
:100A600000200870E3E770B57B4E23242403B068B0
:100A700001252D0470600146D820FFF7B9FF70688A
:100A8000641B40197060AC42F5D2002C0AD00125DD
:100A90002D0301462020FFF7ABFF706840197060FE
:100AA000641BF6D170BDF0B56C4B6E4E9D446C4D21
:100AB000314601A800F049FA6B4C3146206800909D
:100AC0006A48684400F041FA69496068694408600E
:100AD00061485D4F81680024416000221146104644
:100AE000FFF7B4FE634900286944086040D001263E
:100AF0003607FE605F4805216844006800F035F95C
:100B00005C486844006800F04EF9BE60C007E4D15C
:100B100000F068F9002211461046FFF797FE060024
:100B20002AD0012048490007C8600321304600F060
:100B30001CF9494F78680002010E304600F015F9A3
:100B4000B8880004010E304600F00FF939793046BC
:100B500000F00BF90120C002854239D305200002C4
:100B6000321800200021FF23D361F31DF9330AE07E
:100B7000394900200870CBE7374900203E4B087008
:100B80009D44F0BD491C9F68002F03D103273F03FC
:100B9000B942F7D303273F03B94203D12E4B0021BB
:100BA000197003E0002199609169C9B26B4619542C
:100BB000324B6D1E1B5D641C8B4200D0FEE7401C57
:100BC000012180B2C9028842CCD308468542C8D2EE
:100BD0000021002D29D90520000232180020FF2312
:100BE000D361F31DF93300E0401C9F68002F03D14F
:100BF00003273F03B842F7D303273F03B84203D18B
:100C0000154B0020187003E0002098609069C0B276
:100C1000174B6B445854194B1B5D641C834200D026
:100C2000FEE7491C89B2A942D8D301200649000732
:100C30008860114B9D44F0BD004000402C070050DF
:100C40003C070050240700500005005000300040D1
:100C5000700700501450000044000020FCEFFFFF1C
:100C600074270200FC070000DC0F000004080000ED
:100C7000000800000010000004100000E40F000055
:100C8000F0B583B0634801906348614FFF268168E7
:100C9000013641606048019C4568002211461046BB
:100CA000FFF7D4FD0090002854D001205B490007D5
:100CB000C8600521009800F058F8009800F073F81B
:100CC0000121564A09079160C007E6D100F08AF871
:100CD000002211461046FFF7B9FD009000283DD0D4
:100CE00001214E480907C1600221009800F03DF83B
:100CF0002802010E009800F038F82804010E009830
:100D000000F033F8E9B2009800F02FF8711E8DB2B0
:100D1000002E09D02178641C009800F026F828469F
:100D20006D1EADB20028F5D101203C490007886056
:100D30003948BF1B416889194160019880190190A9
:100D4000FF200130874200D8384686B2002FA1D15B
:100D500003B0F0BD304900200870B7E72E480021ED
:100D60000170E5E72C4800787047052310B4002295
:100D70001B02C318D96103210903FF30013000E0D1
:100D8000521C8468002C01D18A42F9D300248A4283
:100D900004D12148047010BC002070478460986919
:100DA00010BC0120704710B405220021FF2412025C
:100DB0008318DC6103221203FF30013000E0491C7C
:100DC0008468002C01D19142F9D30024914204D1CE
:100DD0001148047010BC002070478460986910BCF2
:100DE000C0B2704770B5002211461046FFF72EFDC5
:100DF000002808D00124094D2407EC600621FFF7E4
:100E0000B4FFAC6070BD04490020087070BD0000E4
:100E100074270200E40F0000440000200005005089
:100E2000034610B50B439B070FD1042A0DD308C806
:100E300010C9121FA342F8D018BA21BA884201D9AA
:100E4000012010BD0020C04310BD002A03D0D307ED
:100E500003D0521C07E0002010BD03780C78401C22
:100E6000491C1B1B07D103780C78401C491C1B1B19
:100E700001D1921EF1D1184610BDF8B5042A2CD329
:100E8000830712D00B78491C0370401C521E830745
:100E90000BD00B78491C0370401C521E830704D0F2
:100EA0000B78491C0370401C521E8B079B0F05D00A
:100EB000C91ADF002023DE1B08C90AE0FFF774F916
:100EC000F8BD1D4608C9FD401C46B4402C4310C067
:100ED000121F042AF5D2F308C91A521EF0D40B7857
:100EE000491C0370401C521EEAD40B78491C037045
:100EF000401C012AE4D409780170F8BDD2B210B5C3
:100F000013029A1813049A1800F00EF810BD01E0AD
:100F100004C0091F0429FBD28B0701D50280801C65
:100F2000C90700D00270704700290BD0C30702D058
:100F30000270401C491E022904D3830702D5028097
:100F4000801C891EE3E70022EEE70022DFE77047FE
:100F500070477047754600F023F8AE4605006946B5
:100F60005346C008C000854618B020B5FFF7AAF95F
:100F700060BC00274908B6460026C0C5C0C5C0C52C
:100F8000C0C5C0C5C0C5C0C5C0C5403D49008D462F
:100F900070470446C046C0462046FFF7DEF8000012
:100FA000004870477800002001491820ABBEFEE7DA
:100FB000260002007047FFC1FBE84C90728BE7B33C
:100FC000518963AB232302841872AA612F3B51A875
:100FD000E53749FBC9CA0C18532CFD00FF0000007F
:100FE000FF00000000000600B0F80100B000008023
:100FF000280100801001008018010080200100807D
:10100000FC5F018028010080F4C00080280100807E
:1010100028010080502300802801008028010080E2
:10102000C427008054270080E426008074260080B6
:1010300004230080280100804C700180280100807A
:101040002801008028010080280100804071018073
:1010500090C00080280100802801008028010080C5
:1010600028010080280100802801008028010080DC
:1010700028010080280100802801008028010080CC
:1010800028010080280100802801008028010080BC
:101090002801008028010080280100800C107CCFEE
:1010A000EB0602000860A5A504702C60A5A50C50F5
:1010B0002000B1672474C675A2FD0C701C2F0C6053
:1010C000CC30F203B1072474C676A2FD0C70CC308C
:1010D0000C607CCFF203B1072474C676A2FD0CE04D
:1010E000202D0CD0202DF204307EF17024E4C6EDCA
:1010F000A2FC4B390F00ABA40F000000B920280060
:101100000422F20DB92028000423F209B920280096
:101110000420F205B92028000421F201B92024009E
:10112000B9302C00D94030000140EB0D02003820CE
:10113000240038302C0058403000B9102400B93059
:101140002C0008300050B9030010D9403000D9807D
:101150004000D9C0500001400151C9406000B92091
:10116000200008200100B1233043D64292FE09003E
:1011700001000423B9230010F2014840600011155A
:10118000110458C05000588040005840300048209A
:101190002800381024006100341404700466B1F192
:1011A0002F47030010F4B4612F57020091F524710A
:1011B00092F830F12414E1F0341404700464B1F1B5
:1011C0002F47030010F4B4612F57020091F52471EA
:1011D00092F830F12414E1F0087000402C70000304
:1011E000305706657768DC60FF00920508600100F3
:1011F0006665B1673870E42F2471B970E42F087008
:101200000F001117E1F000003870E42F3471C47042
:10121000B970E42F120C087000402C700003306786
:10122000085000FF2C50FFFF5665B167E1F0000049
:101230000672B022820F28670A0026623066C460F8
:10124000B1679203B9070400286708003461A967F1
:101250000800E1F03418C1E106E26B0F00002F7EB8
:101260000E00267E0C40683657712F6704003856F2
:10127000080024742647C6549205EB10000004E0D1
:10128000F224307538450400B174B9470400207663
:101290003471A176067E4B980F00000007002800ED
:1012A000140018001C001C001C002000200014EC7E
:1012B000F20714E4F20514E8F2031CE0100026E53E
:1012C000F20204E0EB100000062E40E12418E1F0E9
:1012D00018220100F7205421E1F0000018621700E5
:1012E000187216005762777206266627E1F0000032
:1012F00017A11C702100D73256766637993201004B
:10130000E1F00000E1F000001820F545E1F00000F8
:10131000C421D2039920F545E1F000001820F645DC
:10132000E1F00000862282039920F645E1F00000FA
:1013300028205E43E1F0000018206043E1F0000047
:1013400018201D44E1F00000C423D20399201D445D
:10135000E1F0000018701D442F670700267606672D
:10136000D761267624710C208E432627E1F00000F9
:1013700018201C44E1F0000038202844E1F000006F
:101380000C601C43387610012471B9761001E1F02D
:1013900028204E44E1F0000018205044E1F0000005
:1013A00018205144E1F0000028205244E1F00000F0
:1013B00038207C44E1F0000038208044E1F0000057
:1013C00038208444E1F0000038208844E1F0000037
:1013D00038208C44E1F0000038209044E1F0000017
:1013E00038209444E1F0000038209844E1F00000F7
:1013F00038209C44E1F000003820A044E1F00000D7
:101400000C601C43387684012471B9768401E1F0C4
:101410003820A444E1F000003820A844E1F00000A6
:101420003820AC44E1F0000086228203A9205E430C
:10143000E1F000000420E1F00420E1F00420E1F0FC
:10144000C42D9920293ED20424211322F202042D16
:10145000B920703EE1F00000C423D2039920C900F6
:10146000E1F000001820C900E1F00000C421D2031F
:101470009920C530E1F000001820C530E1F00000EF
:10148000C423D20399209930E1F00000182099304C
:10149000E1F00000C423D2039920BF30E1F0000046
:1014A0001820BF30E1F00000C421D2039920A230FF
:1014B000E1F000001820A230E1F000003414B1F196
:1014C0001830F02E0C40F52E04500460F20B10740E
:1014D000B3F73205C62582092451135524611366DA
:1014E0002443C663A2F5047030F106272414E1F00A
:1014F0003414B1F11830F02E0C40F52E0450046075
:10150000F20B1074B3F72205C62582092451135536
:10151000246113662443C663A2F5047030F10627E4
:101520002414E1F01870F02E1860A430C667A204ED
:1015300034719970A4301870A4302F670700267694
:101540000C60F02E267618270700E1F01860F02EC8
:10155000C46004710C40F72E04502676920B04717F
:10156000F20910342443C63292049950A430F20890
:101570002451B47192F7067634719970A430E1F079
:10158000B37222071840F02E0C50F62E0470F21998
:101590005C207F00C42FD21A0C70EC2B262710225F
:1015A000F21610350667C63224712453920A2F763C
:1015B000060026670C70F02E266718260700F20733
:1015C0001367C664A2EF0420F2020420E1F00000D9
:1015D0001820B430E1F000001830F02E0C40F52E49
:1015E0000460F2131074065676725C707F00C4704B
:1015F00024612443920A2F75050026570C70F02EA3
:10160000265718250700F2051376C673A2EC0420AE
:10161000E1F00000B372221A1840F02E0C50F72EA1
:101620000470F21010350667C63224712453920AF2
:101630002F76060026670C70F02E26671826060007
:10164000F2051367C664A2EF0420E1F0B8221C0083
:101650008205087000602627F2020420E1F00000F5
:10166000B82220008205087000602627F2020420BC
:10167000E1F0000086338205087000A02637F202F0
:101680000430B9322000E1F0B8222400820508704D
:1016900000602627F2020420E1F000008633820574
:1016A000087000A02637F2020430B9322400E1F0BD
:1016B0003C101000D1C10450F21810E2046004780C
:1016C00006FE63F6D4F113D6920A04715376667E51
:1016D000D75191722F250D001322F20AB4712461A3
:1016E00092F0245113552421C653A2E8132450C16B
:1016F0002C101000E1F000000673F77126725437C9
:10170000046110575363156656659167E1F0000058
:10171000087000302C700498306714525665B16719
:10172000E1F00000087000302C70049830676461AC
:10173000B167E1F0087000302C7004983027542114
:10174000E1F000003414B1F14B3A0000C4208217DC
:10175000087000302C7004983067085000306C60BE
:101760000010B167087001002C70A186F203B471FB
:10177000820638650898DC60400082FA30F1241453
:10178000E1F00000087000302C70049830671C50A5
:1017900001105665B167E1F0C431920EC420820594
:1017A000087000A02627F2020420087000302C7078
:1017B000B498B127F20FC430920DC420820508708E
:1017C00000A02627F2020420087000302C708898B0
:1017D000B127E1F0C421920A087000302C70B4984F
:1017E000B077820204201322F20FC420920C0870FA
:1017F00000302C70889830770421C4708202042055
:101800001322F2020420E1F0087000302C70009ADC
:1018100030676464B167E1F0087000302C70009AA2
:10182000306714555665B167E1F000001870CC00C0
:10183000C471820C1870C500C472920A9870C530C9
:101840008209C471820A0470F20A0473F2080472F5
:10185000F2060C703200F2030C70120008600030C7
:101860002C60809AB176E1F0087000302C709C9A60
:10187000306757285C60FFFFB16730676626B12785
:10188000E1F00000087000302C709C9A3414B1F123
:1018900030670850FFFF5665B16730676662B16711
:1018A000EB43000030F12414E1F000000870003038
:1018B0002C70A49A306714545665B167306754236E
:1018C0006626B127E1F00000087000302C70A49A61
:1018D00030671C5021005665B167E1F00870003098
:1018E0002C70A49A30676C602000B167E1F00000B2
:1018F000087000302C70A49A30676C604000B167AB
:10190000E1F00000087000302C70A49A30671C5081
:1019100041005665B167E1F0087000302C70A49A60
:1019200030676C608000B167E1F000000870003043
:101930002C70009B306714525665B167E1F00000CF
:10194000087000302C70009B30676461B167E1F073
:10195000087000302C70849D306714555665B1674F
:10196000E1F00000087000302C70849D30676C60DE
:101970000008B167E1F00000087000302C70849D11
:1019800030676C600010B167E1F000000860003063
:101990002C60A49D3056047153726675B176E1F0E7
:1019A000C4210870003092042C709C9DF2032C70AE
:1019B0008C9DB0778205082000602627F202042063
:1019C000E1F000002F72020026720667D7622676C9
:1019D00026272421F2020471B42192FEE1F00000D6
:1019E000087000302C7098983027E1F008700030B3
:1019F0002C704C9830676462B167E1F00662D76181
:101A00000C70383F2676386704000850003038756F
:101A100008980646D64792FCC4300C70383FD72150
:101A2000262730728205086000A02636F2020430B4
:101A3000B137E1F00662D7610C70383F267638671F
:101A4000040008500030387508980646D64792FCC6
:101A50000C70383FD7212627307204213077C470AC
:101A6000820204205421E1F03022F72E5423E1F0C9
:101A700086338205087000A02637F2020430B9329E
:101A80001000E1F0B82210008205087000602627DF
:101A9000F2020420E1F0000028726C0057386673EF
:101AA000B9726C00E1F0000086338205087000A076
:101AB0002637F2020430B9327800E1F0B8227C0017
:101AC0008205087000602627F2020420E1F0000081
:101AD000387280000860FF002C60FFFF5676573C8C
:101AE0006673B9728000E1F038728000086000FF10
:101AF0002C60FFFF567657386673B9728000E1F0AC
:101B0000387280001C6001FF567657346673B972D4
:101B10008000E1F0386280001C7000015676667328
:101B2000B9728000E1F00000B862780082050870A8
:101B300000602676F2020470182283002627E1F066
:101B400037E30860FF0F2C60FFFF5676573E0860B2
:101B5000FFF02C60FFFF66735676574C0860000F4D
:101B60005646086000FF66742C60FFFF5676575893
:101B70006675B7E3E1F000003C101000D1C106E348
:101B80002FD404008B560000B05E066D57612662AC
:101B90008205087000A02675F202047024D157D186
:101BA000B17626D2286E0400207D576866760860DC
:101BB000FFFF5676286E06006676B17D50C12C1068
:101BC0001000E1F03418C1E106E38B56000026EE68
:101BD00057E126E2B02E8205087000602627F20247
:101BE000042040E12418E1F0087000302C70089ABD
:101BF000306737E30850FFFF7765567523666676D2
:101C0000B7E3E1F03C101000D1C106E32FD404008B
:101C10008B560000067D57712672B06782050870EA
:101C200000602676F202047024D157D126D2B17E0C
:101C3000307D06677768A96E0400A97E060050C152
:101C40002C101000E1F000003418C1E106E2EB5363
:101C50000000C422920A386E14001471C667042171
:101C6000820204201322F202042040E12418E1F051
:101C70000C60D03F3876C8002471B976C800E1F016
:101C80001072CC70DD0092180C70D03F176218678C
:101C90000700C6569213176318670800C6569210BD
:101CA00017A418770900C667920D18220500742141
:101CB0003421F72FF2080420F2060420F204042055
:101CC000F2020420E1F0000034211322C422C202F7
:101CD0000420E1F03414B1F106724B980F000000BB
:101CE000080034001C00160016001C00240024000C
:101CF0002C002C0091030421F20E04719173042135
:101D0000F20A047291730421F206047391730421A0
:101D1000F202042030F12414E1F000001072CC70C3
:101D2000DD00921898720200921717E3CC705000F1
:101D3000921517E4CC70F200921317E5C472921258
:101D400017E6C471D2111822070074213421F72F2D
:101D5000F20C0420F20A0420F2080420F206042007
:101D6000F2040420F2020420E1F000001072CC70B2
:101D7000DD00921798720200921417E3CC705000A5
:101D8000921017E4CC70F200920C17E5C47292091D
:101D900017E6C472920617E7C47192032428E1F093
:101DA0002422F2FE3414B1F1992066420B46000061
:101DB00030F12414E1F0000034140C704C42B1F105
:101DC00018671B00C461920C046299671B00CB4822
:101DD00000001870C500C47482038B47000030F106
:101DE0009900AD302414E1F0C623D20A3F2203004B
:101DF000CC20FF070471020204701327F208362377
:101E0000CC2000080471120204701327E1F00000D6
:101E1000C623B2063F720300CC70FF07020BC62335
:101E2000C20B3623CC200008047112020470132761
:101E3000F2040421F2020420E1F00000CC303F0063
:101E4000D20E0673F77126271072543763735471DC
:101E5000C4700421820204201322F2020421E1F062
:101E60001860BC301870983004212676C4731202B2
:101E700004205421E1F000002F7202002672066750
:101E8000D76126760C601C43267618777200CC70DA
:101E9000680082030420F2020424E1F0CC2039001F
:101EA00012053C2030001322F20D0C7066003672D1
:101EB000C47612053C2057001322F2043C20370060
:101EC0001322E1F03C101800D9C10800C1A106E2BC
:101ED00006B306C204D0F210102C8B75000006A2C7
:101EE000182C010057A28B7500002F7D0E0026A232
:101EF00024D124C291A7137DC67BA2EF58C108004C
:101F000040A12C101800E1F010621073C667920D0A
:101F100017A117F1C667920B1822020017F2762755
:101F200013223421F72FF2040420F2020420E1F0FE
:101F3000C421D20CC4210C70043E9205046199673F
:101F40007900F204046299677900E1F018207D3E7F
:101F500074213421F72FE1F0C421D20CC4210C707C
:101F6000C0469205046199670100F2040462996712
:101F70000100E1F01820C14674213421F72FE1F06F
:101F80001820B73074213421F72FE1F0C4219208D2
:101F900004619960B73004629960C046F206046239
:101FA0009900B7309960C046E1F0000018204C421B
:101FB00074213421F72FE1F0C421D20AC420920504
:101FC000046299604C42F204046199604C42E1F071
:101FD00010720662B3570C2018003209547CC47882
:101FE0000C2018009207F20424241322E1F00C20A4
:101FF0001A0018760100F773C47192F9F2F6000026
:102000001870B730C47192030425F2020423E1F082
:102010001870B730C47192060C70B82B26271022A6
:10202000F2057C2010001622F72FE1F00860003046
:102030002C603C9906750C70383FB960383F0C60D5
:102040008000B9670400086000302C603499B967DB
:1020500008000C600008B9670C00086000302C60B4
:10206000949CB967100008602000B96714001860DC
:10207000B730C461921F086000302C602C99B9679A
:102080001000086000302C602499B96718000860BF
:1020900000302C601C99B96720000C600004B967FF
:1020A00014000C600002B9671C000C600001B967E5
:1020B0002400E1F0063206270C201C3C18701C3C62
:1020C00034142F670700266757613F770600577162
:1020D0002672B1F138771C00F17030F12414E1F070
:1020E0001870D23FC472920718201C447421342106
:1020F000F72FF2020420E1F03C101400D9C10400D3
:1021000006E2062306C506D4B1012B7F0000067E39
:1021100006524B980F0000000500440010002200FA
:1021200022004400100018701C44C4719217207DD6
:10213000046491613478F2111870D23FC471920E28
:10214000C4E2207D9206046891613C701000F205A3
:1021500004683C7014009161A17D207D3474367256
:10216000A17C0672D473820304522652307158C186
:102170000400265723252C101400E1F018501C44AD
:10218000C45192060672547334719970F4450C7000
:10219000D03F18670200C461920B0642D444820308
:1021A0000441F20204429947EC009900F445C452FC
:1021B0009207C4629205542334219920F445E1F03A
:1021C0000C201D40E1F00000E1F000001820E83F85
:1021D000E1F00000C424D203B920E83FE1F00000A0
:1021E0003820EC3FE1F00000B920EC3FE1F00000C6
:1021F0003820F03FE1F00000B920F03FE1F00000AE
:102200008622820C17A217E1C667820A18220300F1
:102210007C2010003421F72FF2040421F202042163
:10222000E1F0000018708F30C471920418205842F9
:10223000F2020420E1F00000B3553213C4308213DF
:102240000C7037002674C44F577126373073D20D87
:10225000C470820D98670600820C18770A00F20A93
:102260000470F2080470F2060470F2040470F202C2
:10227000047037611C60000156656667B7A1E1F024
:10228000C421C2080C604C42387654002471B976DF
:102290005400E1F08622820618220500F72154211D
:1022A000F2020420E1F000008622820618220600D5
:1022B000F7215421F2020420E1F00000C44004613F
:1022C000067204502664920E0461F20C2F4507003A
:1022D00010242F4503001044C624A208C624D205AA
:1022E0002451B46192F4F20206370623E1F00000B3
:1022F000C440047104602674920E0471F20C2F56CF
:10230000020010452F5603001055C645A209C645C8
:10231000D2062461B47192F40623F2020623E1F09E
:102320001870D23FC4719213C4208213B872300364
:102330008212B877C001821118672600C461920F1B
:1023400018272C0074213421F72FF20A0421F208F7
:102350000420F2060420F2040420F2020420E1F03A
:1023600006730653D75257713F7705000C50C0468D
:10237000265738654800546F916218753C005473B5
:10238000D7726676917218655400C46192046C70BD
:102390001000917206735771D73236370C70C046F1
:1023A000263738634000546F97A138734400577242
:1023B000667697E128734C00F77297E2777497E39B
:1023C0000424E1F03C101000D1C104D126D32F73B6
:1023D00002001C60230023DD91672F7D020024D1C1
:1023E0000C60180023DD91672F7D020024D123DDCE
:1023F00091072F7D020024D10C60500023DD9167EE
:102400002F7D020024D1146E23DD91672F7D020001
:1024100024D1046223DD91672F7D020024D1046161
:1024200023DD91672F7D0200916724D11860592F19
:1024300023DD2F7D0200546F91671850582F06E25C
:10244000C45192051C5080006665916724D123DD3C
:102450002F7D0E0024D123DD2F2D0E000431910796
:10246000AB9B000026D223DD2F2D0E000430AB9B4A
:10247000000026D223DD2F2D0E000432AB9B00007E
:10248000262D2322262E0433AB9B000050C10C20A6
:102490001A002C101000E1F00C70D03F18670200F9
:1024A0003414C461B1F1920918271400C4218208C0
:1024B00074253421F72FF205AB870000F2020421C6
:1024C00030F12414E1F000001870D23F3414C471CC
:1024D000B1F19206AB9900001622F72FF202042107
:1024E00030F12414E1F000005443D74254376643DE
:1024F0009942180099021900E1F0000018708F301D
:10250000C4719227C4208225C43FD2230C70E600F8
:10251000267357712672B077821698670E00821361
:1025200018772C01C472820FC474820D04739174E5
:10253000F20A98670600820D18770B00C4719209A1
:102540009174F2072C302D0157312632B07392F27C
:10255000E1F00000C4200C701435920718670500E4
:10256000646199670500F206186704006461996761
:102570000400E1F0C4200C701435920818670500BF
:102580005C60FE0099670500F207186704005C6054
:10259000FE0099670400E1F018709B30C471920B43
:1025A000C420820927ECC4302471A7EC820427EDF3
:1025B0002471A7EDE1F00000E1F000000420E1F05B
:1025C000E1F000000420E1F00420E1F0E1F000007F
:1025D000E1F000000420E1F0E1F000000420E1F06F
:1025E000E1F000000420E1F00420E1F018708F30E9
:1025F000C47192071822D80374213421F72FF202F4
:102600000420E1F018708F30C4719211C42082113F
:1026100018706442C471920F1872D803C471920D7D
:102620001822E30374213421F72FF2080420F20664
:102630000420F2040420F2020420E1F0E1F00000A2
:1026400018708F30C471920E1872D803C471920C36
:102650000673F77126271822E803543763235421A1
:10266000F2040420F2020420E1F000000420E1F072
:102670003C105C00C9E15400043006E20C405400F8
:102680000621AB9D0F002870BA00062EA9715200DA
:10269000107E06312F670700266757613F770600D7
:1026A0005771267E38770400F17048E154002C10F1
:1026B0005C00E1F0C4213414B1F1D211C42199209D
:1026C000933092046B490000F20A087000302C70BD
:1026D000A49A30671C5081005665B16730F124140C
:1026E000E1F0000018209330E1F000001820C10054
:1026F000E1F000000420E1F0E1F000001820CA0041
:10270000E1F00000C4203414B1F11870CA0082094D
:10271000C471821304719970CA000B500000F20D4D
:10272000C470820B087000302C704C9830671453C2
:102730009900CA005665B16730F12414E1F0000039
:102740000420E1F0E1F000001820B400E1F0000006
:10275000A920B400E1F000001820A130E1F0000051
:102760009920A130E1F000000420E1F0E1F0000048
:10277000C4213414B1F1D214C4209920CB008205B5
:1027800018704F43C4729207046299606A3EAB4A64
:102790000000F206046199606A3E0B4A000030F1C5
:1027A0002414E1F01820CB00E1F0000008700030A4
:1027B0002C70009830670676777EC479C2042C703E
:1027C0003700F2032C7030000C50BC3699750100B4
:1027D0000C702E00997502000870000F5676777CF9
:1027E000C479C2042C703700F2032C7030000C50F6
:1027F000BC361377997503000C702E009975040090
:102800000870FF00567677781377CC709F000657D4
:102810007752C2042C503700F2032C503000547F02
:10282000C4799950C136C2042C703700F2032C7061
:1028300030000C50BC36997506000C702E0099754E
:10284000070006765C7000FF7774CC709F00065717
:102850007752C2042C503700F2032C503000547FC2
:10286000C4799950C436C2042C703700F2032C701E
:10287000300013660C50BC36CC609F00997509007F
:102880000C702E0099750A0006767772C2042C70BF
:102890003700F2032C703000546FC4699970C7364A
:1028A000C2042C603700F2032C60300006270C2095
:1028B000BC3697AC046C9960BC36E1F00C20003556
:1028C000E1F00000E1F000000423E1F01820CB006B
:1028D00034140461B1F199604F432BBC000030F116
:1028E0002414E1F01820293E24211322E1F00000F5
:1028F000C42E3414B1F1D20534211322AB220000CE
:1029000030F12414E1F0000018709B303414C471CD
:10291000B1F18204CB290000F202042030F124142A
:10292000E1F000001820A730E1F00000C4223418C4
:10293000C1E106E2D2079920A730CB29000099E037
:10294000BE0040E12418E1F01820CC00E1F00000C6
:10295000CC20FF00C208A9204E44087000302C7023
:10296000849AB127E1F000001C70000126722377E1
:10297000CC70001E3414B1F1D20A0672D4718203F5
:1029800034212322A9205244CB44000030F12414E6
:10299000E1F00000147126722377CC70FE00D2099A
:1029A000132299205044087000302C70849BB1276A
:1029B000E1F00000147126722377CC70FE00D2097A
:1029C000132299205144087000302C70809BB1274D
:1029D000E1F000001870C700C47182041820C5001F
:1029E000F2020420E1F00000C424D20DC4209207BA
:1029F00004719970C7009970C500F2059900C7006D
:102A00009920C500E1F000000420E1F0E1F00000B1
:102A10001820B230E1F00000C426D2039920B23071
:102A2000E1F00000C422D2039920C600E1F00000CA
:102A300018209030E1F00000C421D203992090309A
:102A4000E1F000000420E1F0E1F000000420E1F0FA
:102A5000E1F000000420E1F0E1F00000C421D20325
:102A600099209E30E1F0000018209E30E1F0000037
:102A70001870C630C47192049920C830F2091860E9
:102A8000293E0C70C02E267610679960C8301870E9
:102A9000C830CC703F00C2039900C830E1F000009C
:102AA0001820C830E1F000001870C630C4719204DC
:102AB0009920C930F2091860293E0C70D02E267674
:102AC00010679960C9301870C930CC703F00C203DC
:102AD0009900C930E1F000001820C930E1F0000091
:102AE000862282039920604318506043995017351D
:102AF000E1F000000672777C997098000870FF0082
:102B000056727778997099000672777499709A0066
:102B100099209B00E1F0000018709A00186099005D
:102B20005774576866761820980018609B00572CD9
:102B300066766627E1F000000672777499700530BA
:102B40000870FF005672992004307778772C9970BE
:102B5000063099200730E1F0187005301860063013
:102B60005774576866761820073018600430572C61
:102B700066766627E1F000009920C200E1F00000CF
:102B80001820C200E1F000001870C630C471920431
:102B90009920CD00F2091860293E0C70E02E2676AF
:102BA00010679960CD001870CD00CC703F00C20650
:102BB0001870C80016779970CD00E1F01820CD008C
:102BC000E1F000006820B600E1F00000B9008444A4
:102BD000E1F00000B9008844E1F00000B9008C4445
:102BE000E1F00000B9009044087000302C70949817
:102BF000B107E1F0B9009C44E1F00000B900A04445
:102C0000E1F00000B900A444E1F00000B900A844DC
:102C1000087000302C708C98B107E1F0B900AC441A
:102C2000E1F000001820C630E1F000009920C63025
:102C3000E1F000001820C430E1F000009920C43019
:102C4000E1F00000E1F00000E1F00000E1F0000040
:102C5000E1F00000E1F00000E1F00000E1F0000030
:102C60000420E1F00420E1F00420E1F0E1F00000B4
:102C70000420E1F0C420920399009130E1F00000BB
:102C800018209130E1F00000C42092039900B9307F
:102C9000E1F000001820B930E1F00000E1F00000A0
:102CA000B9205830E1F0000038205830E1F0000041
:102CB0009870A8309205387058303027F2020420FE
:102CC000E1F000009870A830920538705830102755
:102CD000F2020420E1F000009870A83092043870ED
:102CE00058309127E1F000009870A83092053870B4
:102CF00058302027F2020420E1F000009870A8303C
:102D0000920438705830A127E1F000009870A83084
:102D1000920438705830B127E1F000000420E1F04F
:102D2000E1F000000420E1F0E1F000000420E1F017
:102D3000E1F000000420E1F0E1F000002820BA00FA
:102D4000E1F00000A920BA00E1F0000028202843AB
:102D5000E1F00000B9202843E1F00000282064439E
:102D6000E1F00000B9206443E1F000002820BC003D
:102D7000E1F00000A920BC00E1F000002820B8002C
:102D8000E1F00000A920B800E1F00000C4213414F3
:102D9000B1F1D20EC4219920C40092081870674284
:102DA000C47192062B480000F203CB48000030F1BA
:102DB0002414E1F01820C400E1F000000420E1F048
:102DC000E1F000000420E1F00420E1F0E1F0000077
:102DD0000420E1F0E1F00000182076427421342153
:102DE000F72FE1F0C421D20CC4210C704C429205A3
:102DF000046199672A00F204046299672A00E1F0ED
:102E0000C421D2039920582FE1F000001820582F38
:102E1000E1F000000420E1F0B9209400E1F00000AE
:102E200038209400E1F000009920C730E1F0000064
:102E30001820C730E1F00000E1F00000E1F00000F0
:102E4000E1F00000E1F000003418C1E11C607700FF
:102E500006E70CE0BC360C20BE360430990E0100AB
:102E60009960BC366BA00100062E40E12418E1F009
:102E70003414B1F11072CC7089009205242204310F
:102E80006BA0010030F12414E1F00000142AE1F0FD
:102E90003414B1F12870B2000C30902B0C6000405B
:102EA000F2020672CC70FFFF042126272322920330
:102EB0000C2000C00643045430743077F20D28F71C
:102EC0001A00C6F29207B46192EDA920B200042064
:102ED000F20A38770C00C47092F3B451244492ED96
:102EE000A920B20030F12414E1F0000027EC37A54E
:102EF0000653266777549956F000247137A5237737
:102F000026679936F0002471A7ECE1F027AC37E58D
:102F100006532676775C9957F00024613765087070
:102F2000FF0023665673265677789975F000047172
:102F3000267637A523770653266777549956F000EF
:102F4000247137A5237726679936F0002471A7EC02
:102F5000E1F000008622821227EC37A51451266783
:102F60009956F000F20537A526679906F0002471FE
:102F7000A7EC27ECCC704300C2F7E1F00652D45125
:102F80003414A1018207C4300205107234312421A7
:102F900097D1C4300673F77004602471320704714E
:102FA000F2052042343226642422B47192FBC431EB
:102FB0009203107291712021C450266206767778B0
:102FC0005C60FFFF2F270600067277785C20FFFF0A
:102FD00026278209067257745C2000FF5C70FFFF91
:102FE0007724662723222414E1F000000C7073007C
:102FF00099722E000C70740099722F000870008076
:103000002C7048F7B7E5087000802C70C0CCB7E68C
:10301000047699722600187034309972270018705F
:10302000353099722800187036309972290018705E
:10303000373099722A001870383099722B00187046
:10304000393099722C000C70DC05A97224000C70C8
:10305000320099722D000420E1F000003870FC2F3E
:103060003C101800B7D3046C3870702F26610C2008
:103070004F00043004400458B9F11400B7D4B10132
:10308000B9010400B90108000B2E0B0038F114003F
:103090002C101800E1F0000004600470F20B2F46C1
:1030A00002001054170157542654235524622675E4
:1030B0002366C663A2F5F2045C70FFFF26760667FE
:1030C0007768C46092FA15772327E1F00860004022
:1030D00038761400D47182FD38261000E1F000002B
:1030E00090733414B1F182032BB4000030F1241436
:1030F000E1F00000063206270C201C3C18701C3C36
:1031000034142F670700266757613F770600577111
:103110002672B1F138770800F17030F12414E1F033
:10312000063206270C201C3C18701C3C34142F67F8
:103130000700266757613F77060057712672B1F185
:1031400038771400F17030F12414E1F03414066281
:10315000B1F137E1383608003022F17030F1241433
:10316000E1F00000E1F00000C4203414B1F1821459
:10317000C43082140C7090232637262710631072F7
:103180000C30FF002F2706008B960F000C70902448
:1031900026721027F2040420F202042030F12414D5
:1031A000E1F000003C101400D9C10400B1B104707A
:1031B0000454F2152FD60C0006B610DDB4F1D7B1C9
:1031C00053DB66ED246192F72F6703003066B4513C
:1031D0002FF70400766EB16F247482072FC70200A8
:1031E00004E0046004F4F2E758C1040030B12C108C
:1031F0001400E1F0341804700464C1E12F57020098
:103200002FE70300305530EEB4612FF70400765EEF
:10321000B15F247492F440E12418E1F034140460A6
:103220000454B1F12F7603002FF6020030FF3077FF
:10323000B451767F06F777F499F4010006F791749C
:1032400077F8777C99F4020097C32464244492EBC6
:1032500030F12414E1F000000C40200036420461FB
:10326000536434611556565373545663536206259E
:103270006626E1F01872CC01C471920A0C60C83362
:10328000387604009902CC013471B97604000462E6
:103290003872C0019162B902D801046199672600B1
:1032A000E1F00000E1F0000008700030C4202C7054
:1032B000481E3077820406676461F2031462566721
:1032C00008700030C4202C70481EB1678207087057
:1032D00000802C7080006676F2060870FF7F2C70EC
:1032E0007FFF5676086000302C60481EB176E1F012
:1032F0003C102400D941080001610170C9611C0023
:10330000B9F11800C1216B0F000006650C602C326A
:10331000B8760C00820638202C3238360800F1705E
:10332000EB10000048611C0038F118004021111614
:103330001107584108002C10240061003C101000B7
:10334000C16101610170C96108004861080011167E
:10335000110740612C10100061000000E1F0000036
:10336000276327A41375C656A2033676137706275C
:10337000E1F000000672547AC47A9206B372320603
:10338000F7225421F2040420F2020420E1F00000AC
:103390003870B42F0C301400263718770C00777271
:1033A000C475C2323475577123470470F22B2F57FE
:1033B00003001065C4618206C461A226C462921D26
:1033C000F2032471F21E18650100C464921D0463A7
:1033D0002667C66432191865020018550300576441
:1033E0006665145126562355CC50B305C2030C60B4
:1033F000B405A1622474F205986501008205267661
:103400002377C674A2D5E1F03418C1E1046706E75A
:103410000CE0BC360C20BD36043004479960BC3645
:10342000AB9D0F0004710C603500997E0100996E10
:1034300003000478046A062E997E0600996E070040
:1034400040E12418E1F0000034140C20CC300430AA
:103450000C408000B1F1AB9D0F0030F12414E1F07D
:103460003C102000C9E118003830A00006E20C2012
:10347000C0010BC30F00063E04460C201C432B9ECC
:103480000F00063E04460C2034302B9E0F003830CF
:10349000A0000C20D0010BC30F001870343038206E
:1034A000A000B17118703530B7D1187036300C30BB
:1034B000E001B7D218703730B7D318703830B7D4AE
:1034C00018703930B7D5EBC40F0048E118002C1044
:1034D0002000E1F08633341CB9F10800820CB121E0
:1034E000B93104003820A0000C30F401EBC40F0007
:1034F0000421F202042038F10800241CE1F000004D
:103500001870A8303C101000C471D1C106D28AA531
:103510000000C421D25B3830A0000C2000020BC395
:103520000F000CE01C43383E60010C2028024B27A2
:103530000100383E90010C2038024B270100383E34
:1035400080010C2044024B270100383E68010C200A
:1035500054024B270100383E6C010C2064024B27BB
:103560000100383E70010C2074024B2701000CE072
:103570004C42383E2C000C208C024B270100383E78
:1035800030000C209C024B270100383E34000C20F8
:10359000B0024B270100383E38000C20C8024B27F0
:1035A0000100383E44000C20E0024B270100383E69
:1035B00054000C20F4024B2701003830A0000C20EE
:1035C00004030BC30F00C4D0F202C4229246383069
:1035D000A0000C202C030BC30F003830A0440C209B
:1035E00050034B270100087000302C708C98303746
:1035F0000C205C034B270100087000302C7094985D
:10360000303723330C206C034B2701000870003047
:103610002C70989830370C2080034B2701000870DD
:1036200000302C709C9830370C2090034B27010001
:103630000CE04C42383E48000C20A4034B2701000C
:10364000383E64000C20B4034B2701003830A00042
:103650000C20C4030BC30F0050C12C101000E1F06C
:103660003C103C00D941140001610170C961340073
:10367000D9C124000870023008E002302CE0145454
:103680002C701C54C9210C003820A00030DE30778B
:103690000C30E8030160B1D1B791B7D2EBC40F0091
:1036A000087000402C70000364D2B1DE386704005B
:1036B0006462B96704004861340048210C001116A7
:1036C000110758C12400584114002C103C0061001F
:1036D0003C103C00D941140001610170C961340003
:1036E000D9C124000870023008E002302CE01454E4
:1036F0002C701854C9210C003820A00030DE30771F
:103700000C3000040160B1D1B791B7D2EBC40F0007
:10371000087000402C70000364D1B1DE38670400EB
:103720006461B96704004861340048210C00111637
:10373000110758C12400584114002C103C006100AE
:103740003C103C00D941140001610170C961340092
:10375000D9C124000870023008E002302CE0145473
:103760002C701C54C9210C003820A00030DE3077AA
:103770000C3018040160B1D1B791B7D2EBC40F007F
:10378000087000402C70000364D8B1DE3867040074
:103790006468B96704004861340048210C001116C0
:1037A000110758C12400584114002C103C0061003E
:1037B0003C103C00D941140001610170C961340022
:1037C000D9C124000870023008E002302CE0145403
:1037D0002C701854C9210C003820A00030DE30773E
:1037E0000C3030040160B1D1B791B7D2EBC40F00F7
:1037F000087000402C70000364D4B1DE3867040008
:103800006464B96704004861340048210C00111653
:10381000110758C12400584114002C103C006100CD
:103820003418C1E1046606E70CE0BC360C20BD3656
:103830000C301C4304469960BC362B9E0F00062EAC
:1038400040E12418E1F000002F72020026720667A2
:10385000D761267634140C601C43CC406800B1F16B
:1038600026769947720082030445F202044D2F72B6
:10387000020026270672D77126270C708E4324215A
:1038800026272B9E0F0030F12414E1F03418C1E1FB
:103890004B1B00000C601C431876010106322F57A9
:1038A000070026750657D7512675266718467200F9
:1038B000F74106E70CE0BC362F6404000C20BD364F
:1038C0009960BC362B9E0F00062E40E12418E1F0D3
:1038D0003418C1E1046606E70CE0BC360C20BD36A6
:1038E0000C30E84504469960BC362B9E0F00062E2E
:1038F00040E12418E1F00000341424240446B1F11E
:103900002B9E0F0030F12414E1F000003414242A1F
:103910000446B1F12B9E0F0030F12414E1F00000B9
:1039200034142C2010000446B1F12B9E0F0030F10E
:103930002414E1F004742672341406230446063776
:10394000B1F12B9E0F0030F12414E1F0047A2672BD
:103950003414062304460637B1F12B9E0F0030F1D4
:103960002414E1F00C70100026723414062304466F
:103970000637B1F12B9E0F0030F12414E1F0000066
:103980003414B1F117E15471C4719204CB4B0100AE
:10399000F2034B4A010030F12414E1F0341CC9E178
:1039A000040006E2B1312B170000C421303192052A
:1039B000062ECB4B0100F204062E0B4B010048E112
:1039C0000400241CE1F000003C107400D981540074
:1039D000D9C1640006E2384E140038220800B9410B
:1039E0004000B92144000C404000062138DE0C00A4
:1039F00038CE10002B9E0F003831440030B10870D3
:103A00006AD738514000263B2C7078A42637066CC4
:103A1000157D566D5675667626730667D763F77CF7
:103A2000667637912F3D07000870C7E826562C7040
:103A300056B7265706631573566D567C66762675FF
:103A400006675766777A667638F108002F530700C5
:103A50000870202426FC2C70DB7026F7066515758F
:103A60005663567D6676267F0667D768F777667653
:103A700037932FF507000870BDC1266D2C70EECE70
:103A80002667064F157F56455673667426670646A9
:103A9000574B776537D4666408807CF5266F2C8099
:103AA000AF0F268706461576564F567566742683E1
:103AB0002687064838311400D743F78C089087478B
:103AC00066842C902AC62686269326951578065855
:103AD0005656567F6675269706495746779A6694D6
:103AE000269838211800084030A8157906592C402E
:103AF0001346565826425676264F66752674065744
:103B000038F11C00D758F77708A046FD66752CA041
:103B10000195267926AF26A6065715675659566889
:103B2000666526A6065A575B77A566A526A73718A9
:103B300008208069156A065A2C20D89856572624E2
:103B400056696665262826260682D783F72C37997C
:103B500066280850448B262A2C50AFF7265606427A
:103B60001562564A566726596664266506465746C4
:103B7000776A6664371A26623C404FA42647065689
:103B800015765652567A667526740657D758F777C3
:103B900038812C00667508505C892C50BED726767B
:103BA000265826A50647155756465652665426A54A
:103BB000064A574B77A53891300066A40840906BB1
:103BC0002C4022112F870A00264926421558062824
:103BD00056275656665226540625D723F75C66525A
:103BE000084098FD382134002C4093712658264215
:103BF000266406251545562856476642266406263D
:103C00005726776A66622665154638213800B9411D
:103C10005000084079A62C408E4326422647387132
:103C2000500006A656A55678667A267406A7D7A829
:103C3000F777371F667A08A0B44926762CA02108AA
:103C4000159726A4B99148002F980A0038A148007A
:103C50000687568656A566A826A9068A578B77A595
:103C60003891040066A808801EF62C80622526A7DD
:103C70002689389150002658068A569756866689B6
:103C800026580695D792F75D388118006659089036
:103C900040C02C9040B3265A2698388148002669A7
:103CA0000695568A5697669826690686D784F76BD6
:103CB000666808905E2638812C002C90515A266543
:103CC00026982679158A06965685569A66982679F4
:103CD0000687578777790890B6E966782C90AAC747
:103CE0002676269B26A915850697568656956698AC
:103CF00026A9068A578A77A608902FD666A82C9000
:103D00005D1026A7269326591586069A568756963D
:103D1000669826590695D792F75D66592F8A050051
:103D200038912800085044022C5053142659266517
:103D300015970658569A5657665926560695D7949B
:103D4000F75B0860A1D866592C6081E62658266486
:103D50002676159A06655698566A66692676066727
:103D60005767777966762F95070037940870D3E701
:103D70002C70C8FB267626A71568067956655678F6
:103D8000667626A7066A576A77A666A60870E121B6
:103D900037992C70E6CD26A9267626871565067AF2
:103DA00056695675667626780667D762F77D667619
:103DB000086037C32C60D607267A266226561589F6
:103DC0000667568A5669666826560685D784F75B65
:103DD00066580860D5F438810C002C60870D265792
:103DE00026682696158A06655687566A6668269658
:103DF000068957877799669808605A453881200068
:103E00002C60ED142695266826A61587066956852A
:103E100056676668266A0686578A7766666808A0C7
:103E2000E3A9388134002CA005E9266926A8267A62
:103E3000158506A6568956A566A8267A0687D782CE
:103E4000F77D667808A0EFFC388108002CA0F8A365
:103E5000267626A8265A158906A7568656A966A844
:103E6000265A0685D784F75B08A06F6766582CA092
:103E7000D902265726AF269A158606A5568756A636
:103E800066A8269A068957877799669808A02A8D8A
:103E9000388130002CA08A4C269526A8266A1587E2
:103EA00006A9568556A766A8266A08A0FAFF0686C0
:103EB0002CA0423926A3578A77666668267A06A917
:103EC000266976A576A6267A06875782777E667853
:103ED00008A07187388120002CA081F626A8265AD8
:103EE00006A6267676A976A7265A0685D785F75A96
:103EF000665808A09D6D38812C002CA0226126A850
:103F0000269A06A7265776A676A5269A0689578862
:103F1000779866980880E5FD2C800C382682266804
:103F20000685269576877689266806A6D7ABF76438
:103F300038810400666A08A0BEA42CA044EA26A822
:103F4000068926697685768626A726A8067A577278
:103F500077AE3881100066A70870DE4B2C70A9CFB1
:103F600026782657067626A67679767A2657068507
:103F7000D785F75A0870BBF666582C70604B068AD6
:103F8000265A267F7686768526792678069757984C
:103F900077783881280066790890BFBE2C9070BC75
:103FA0002698266906952675769A76972669068656
:103FB000D78BF764666808909B28388134002C9072
:103FC000C67E269826A9069726677695769626A910
:103FD0000890A1EA068A2C90FA27269B578277AE92
:103FE00066A82659069626A67697769A26590685B5
:103FF000D785F75A66580890EFD438810C002C907A
:10400000853026982679069A265A769676952679C8
:104010000687578877786678089088043881180072
:104020002C90051D269806852675768A7687269615
:1040300026980669D76BF794388124006696086045
:10404000D4D92C6039D0266806872697768576895C
:10405000266A266806A657A2776E38813000666AFF
:1040600008A0DBE62CA0E59926A8265A06A9266911
:1040700076A776A6265A0685D785F75A08A0A21FE6
:1040800066582CA0F87C0686265626A47689768566
:1040900026A726A8067A577877A83881080066A749
:1040A0000870ACC42C7065562678068526A57686E1
:1040B000768A267926780697D79BF77466790890D2
:1040C00029F4267A2C904422158526B96687768AAB
:1040D000266B266806B657B3776D666B08B02A4321
:1040E00026672CB097FF159A26FB66967697265F73
:1040F000265906855785775B665808F094AB265697
:104100002CF0A72315B7262F66B576B626A226ABC8
:10411000069AD797F7A866A9082093FC26A52C2015
:1041200039A015F6263266FA76F52673267F06B78D
:10413000D7BAF77538913000667B08305B65267A10
:1041400015252C30C35926396627762A2663266220
:1041500006F638210C0057F3776D08300C8F666F28
:104160002C3092CC26672632152A662676272653CF
:10417000265206F557F5775B38812800665F0830D0
:10418000EFFF265615272C307DF426386625762637
:1041900026A326A206FAD7F7F7A83891040066AF3F
:1041A0000830848526A515262C30D15D2639662A4F
:1041B00076252673267206F738212000D7FAF77580
:1041C0000830A86F667F2C304F7E267A2632152560
:1041D0006627762A2663266206F657F3776D666FA2
:1041E00008302CFE26672C30E0E6152A264366268A
:1041F00076272654265206F53831180057F5775B96
:10420000084001A3665F2C40144326562643153709
:104210006635763626A426A3062AD727F7A838813E
:10422000340066A20840084E26A515362C40A11180
:104230002648663A267476352637389110000623CC
:10424000087053F7D72AF7352C70827E66322679AC
:104250002F4A0300266715756674767A26760667F8
:104260005763777D38212C00667608603ABD2C6054
:1042700035F2266226742656156A666776642656D7
:1042800006655765775B3831080066560860D72A9F
:104290002C60BBD22663265726A615646665766712
:1042A000266A0636D737F768666338314400082037
:1042B00086EB2637B93E08003881240026652C207D
:1042C00091D31577262866767675264226740637AA
:1042D00038914000D73AF77526D66637263D26C670
:1042E0002659B93E0C00B9CE1000B95E140058C171
:1042F0006400588154002C107400E1F0066366627B
:10430000D4633414B1F1065206F3067482042B9E72
:104310000F00F2180664D463777182032471F202ED
:104320002377C470046104402667920A0461F2088E
:104330002F340F0030232F7405002444B127B461BB
:1043400092F830F12414E1F03C101400D9C10400BB
:10435000B1B138E3040006C206D306B40635062E12
:1043600004462B9E0F000426063B262E04462B9E59
:104370000F000478997E0C000470997E0D00387C43
:104380001800062C063DF17058C1040030B12C1005
:104390001400E1F03418C1E10C60200006E70CE0E5
:1043A000BC360C20BD360C3048040C40200099600F
:1043B000BC362B9E0F00062E40E12418E1F00000D1
:1043C0003C101000D1C106D28B9A0F00CC201F00E8
:1043D0000CE02000D20213E2063D064E0C202E43D4
:1043E0002B9E0F000C701C4326E7990E120050C143
:1043F0002C101000E1F00000C4303C101800D9C1AE
:104400000800C1A10CA040000CC0610006720CD0D5
:1044100074310CE0B43126A20CB04C3126C2921398
:10442000063D0C4040002B9E0F00063E062A0C4025
:1044300021002B9E0F00062C063B0C4028002B9ED3
:104440000F00F21D06370C404000062D2B9E0F007A
:10445000062D8B9A0F00063A0C40210099208C30D3
:10446000062E2B9E0F00062E8B9A0F00063C9920DD
:104470008B300C402800062B2B9E0F0058C10800E3
:1044800040A12C101800E1F0CC3040003414B1F100
:1044900006720643C2030C40400006260C201D4055
:1044A00099401D402421063713444B990F0030F1E9
:1044B0002414E1F03418C1E106E28B9A0F001332A4
:1044C000062EEBA4010040E12418E1F03C10180096
:1044D000D9C10800B12106E33820A0000C306C04DB
:1044E00006C4B711EBC40F0086CC04D0920204C1FD
:1044F0002F7D0E0010773820A0000C30E000B17145
:10450000EBC40F00B4C124D1820A067DD47792F1A6
:104510003830A000042A2BC40F00F2EB3830A00082
:10452000042A2BC40F0058C108002C101800E1F019
:104530003418C1E106E2063E0C207C0404460BA7B9
:104540000100063E0C20E84504462B9E0F0040E18A
:104550002418E1F03C101000D1C10CD06645062DA6
:104560008B9A0F0006E70CE0BC369920BC3604217C
:10457000262E063D0B9B0F00062E50C12C1010005E
:10458000E1F000003C101000D1C1062D0C202E439C
:104590008B9A0F0006E70CE0BC369920BC3604214C
:1045A000262E063D0C302E430B9B0F00062E50C1CD
:1045B0002C101000E1F0000034140446B1F18BA37C
:1045C0000F00C42004718202047030F106275421C8
:1045D0002414E1F017E1647297E1E1F017E16C70E7
:1045E000400097E1E1F0000006570C50E8451860E4
:1045F000E84518750100576466671875020018458C
:104600000300577466741845040057741855050064
:10461000667457746675085000302C501498B16554
:10462000086000302C601898B176E1F037E6086039
:1046300000F02C60FFFF567657380860FF0F5636A3
:104640006673B7E6E1F0000037E60860FFFF5676D4
:104650006673B7E6E1F000003C101800D9C108000D
:1046600028C3060006E224C426C423CC06D3063C95
:104670006B550000062E0431AB580000062E063C98
:10468000EBB20100062E04300BB20100406D062E85
:10469000C16127D3063124740440A7D36B5C0000AA
:1046A00058C108002C101800E1F0000004761062D8
:1046B00024611366C46091629204B471242192F85B
:1046C000E1F000003C1010000C701000D1C1267108
:1046D00020D7067206E64B980F00000004005C002D
:1046E0000E001C00140018000C703600F207047E47
:1046F000F2050470F2030C70220024735C707C00DD
:104700002F630700C66D121AC4E0B105820526E7C3
:10471000B9E50400F203B9050400047299750D00AF
:104720000471A9350800A9350A0099450C00A9753E
:104730000E000625F2040420F202042050C12C10C1
:104740001000E1F086338232C4208232C430320756
:10475000166327E52366C676B203F22C2363176C33
:1047600037E1C4508203C453920C0C5010003F63D5
:1047700007002652C665B7A1B20FB7E10421F221A6
:1047800034512355C451D218C43032182765C65647
:10479000A2173673B7E127E523332673A7E527E48D
:1047A0002637A93208000420F20C0420F20A042063
:1047B000F2080421F2060421F2040421F202042189
:1047C000E1F0000006720420F20424213077132265
:1047D000C47092FCE1F000008622820427E7247175
:1047E000A7E7E1F0C420820FC4309206F20C2764E0
:1047F0002675A7E40626B06227F492FA27A4B13200
:104800002676A7E4E1F000003418C1E106E3CBBF4F
:104810000100062E6BBF010040E12418E1F000000A
:10482000C4203C101800D9C10800C1A106D206E37B
:104830008249C430824927A427F4C667A24704B03E
:1048400004C0287D0A0028AE0A00367C36ABC67A42
:10485000220323AAF20223A7382D0400383E0400C5
:10486000262C263B064A2B9E0F0026BA287E0A00DD
:1048700023BBC67B26CA23CCD20330EE04B0287DEE
:104880000A00C67C9207B0DD9204C4E08219F220CF
:1048900004C0C4E08209286E0A00287E0800C667AA
:1048A0009203B07E9217C4D08209286D0A00287D39
:1048B0000800C6679203B07D920FC4E092C3042043
:1048C000F20C142EF20A142EF208142EF206142EF4
:1048D000F2041426F202142658C1080040A12C103C
:1048E0001800E1F0C4203C102000D9C11000D18193
:1048F00006D306E4822DC430822D06C204B0049093
:10490000F222C4508208287C0A00C657A2043657F7
:104910002355F21828AC0A0036A5237AC67EC202B7
:1049200006AE383C040023AA2F290D002635064A7E
:104930002B9E0F0026BA269A36EA23BB239923EE34
:10494000045030CCC4E08207C4C092DCF20404B04E
:10495000F20204B058C11000062B50812C10200028
:10496000E1F00000C4203C101800C1A1D9C108002A
:1049700006A38222C430822227E4C674A22106E460
:1049800006D204C0F215287D0A0006BE2367C6E6DB
:10499000C20206B723BB382D04002F3C0A00064B89
:1049A0002B9E0F0026CB36EB30DD23EE23CCC4E06C
:1049B00092EB0420F2060420F2040420F202142EEA
:1049C00058C1080040A12C101800E1F03C10140060
:1049D000D9C10400B1B137E106D218B7090038E0F7
:1049E000CC2F04C0F22E187E1000C67B9220B06E31
:1049F00082053870402FC667921AB87E140082175D
:104A0000382E1800063E064D0C501C2FF170C420A5
:104A1000820EC4C0820E387E0C00B97C0C00387047
:104A2000CC2FB9E0CC2FB97E0C00F2030470F20356
:104A3000047104D0C470386E0C00920706CE06E6EE
:104A4000C4E092D20420F202042158C1040030B123
:104A50002C101400E1F00000283236000672CC3031
:104A60001C1137AA28422C00376CC2030C301C11D1
:104A70003F25040026263F330200C4302204A94704
:104A80002E00F20E3F450600C4400205A9072E0085
:104A90000420F2063F6605000420A9672E00E1F01D
:104AA000387070003820382F2627B9207000E1F0C8
:104AB00038602C2F3418C1E1067604F0F213C627B3
:104AC000820E28571200C654920BB0E7823FC430C2
:104AD000823FB053823FC6E59203F23E04F138773D
:104AE0000C00C47092EDC43082033073F202047083
:104AF000C440B17292232870B0000C500040F20202
:104B00000674CC70FFFF04412647234492030C40F7
:104B100000C00676F20D28371200C6349207B45151
:104B200092F0A940B0001428F21C38770C00C47031
:104B300092F3C440A940B0008211C4F0A72992109A
:104B4000B7A3B9202C2F0420F20C1428F20A142841
:104B5000F2081428F2061428F2041428F2020420A1
:104B600040E12418E1F000003C101000D1C1A8720F
:104B7000120006E206D306C49207063204402BD682
:104B8000010086229220C4D08203307DF20204709C
:104B9000B97E0400187E1000A9CE14006474997EBA
:104BA000100038602C2F0676F205C6E7820B3877A6
:104BB0000C00C47092FBB96E0C00B9E02C2F0420DD
:104BC000F202042050C12C101000E1F03C1028002B
:104BD000D9C11800D9810800B13106E406D506868E
:104BE00006B204A004C00471F21E289B0A00382BF0
:104BF00004000639B7D18BFC0000D49126C2066CA4
:104C000077685CC0FFFF26C637D1820C066C5764FC
:104C10005CC000FF3FAA07005C60FFFF77C413AAD7
:104C200066C630BBC4B092E2C4A08209067C577449
:104C30005CC000FF5C70FFFF77C466C7307157D45B
:104C40003067307E065677585C60FFFF2665065752
:104C50005C50FFFF26657778267626D7067857744E
:104C6000778466782377267D26C7066C77685CC0D4
:104C7000FFFF26C6067C77785CC0FFFF2F270C005D
:104C8000152258C118002322588108002C10280032
:104C9000E1F000003414B1F18BFC000030F115227A
:104CA00023222414E1F000003C101800D9C10800B0
:104CB000C1A106D204C004E004A1F21C28BD0A0070
:104CC000382D0400063B8BFC0000D4B126E2067EA2
:104CD00077785CE0FFFF26E7820C067E57745CE085
:104CE00000FF3FCC0A005C70FFFF77E413CC66E75F
:104CF00030DDC4D092E4C4C08209067E57745CE003
:104D000000FF5C70FFFF77E466E7152E58C10800CE
:104D1000232240A12C101800E1F000003870202F51
:104D2000F20E18672D00D4618209305238670400F2
:104D3000766538570800D665820D3077C47092F2D8
:104D4000B8207C2F820818722D00D47192040420A0
:104D5000F2020627E1F000003418C1E106E2062362
:104D60008BE901008622820CA862240082093C6043
:104D700028002356C6E5067EC202067623E7062EE5
:104D800040E12418E1F00000146126621473C66744
:104D9000D21418732D00D472821237B1C626821134
:104DA00037F27662D667920F15775627C6270461C9
:104DB000820204601326F2080421F2060420F204A1
:104DC0000420F2020420E1F006620672577C776C40
:104DD000666706725C7000FF577466670870FF00B4
:104DE0005672777406266627E1F000003C10180022
:104DF000D9C10800C1A1B8D2700006E28244307D5A
:104E00000CB06C00B972700026B238C26C00F203AC
:104E100006BC30CCC4C0822A385C0C001865050082
:104E20001875040057646667187506001825070092
:104E300057786676572C6627EBEE0100385D0C003C
:104E400006A2186505001875040057646667187592
:104E500006001825070057786676572C6627EBEE74
:104E600001003F220A00C42022D4B1CDB1DBB07DC5
:104E70009203A90E6A00187E4600B90E380024710C
:104E8000997E460058C1080040A12C101800E1F09E
:104E9000B87270003418C1E106E2822B18721E004D
:104EA000D47492270BF00100287E4C00286E60001D
:104EB000C676C205F760A96E4E00F204F770A97EAF
:104EC0004E00287E3600285E4E002F670700C6562B
:104ED0003203A96E4E002F6707002676286E4E001B
:104EE0002676A97E4C00187E1E006474997E1E00F2
:104EF00040E12418E1F000000C70D0300460045848
:104F00003047C642920738470800C643920333260B
:104F1000F208B451246113662C70100092F214212F
:104F2000E1F00000C4213C100C01C9E1040106E3DA
:104F3000921804240C30E80026210B9B0F00042B50
:104F40000C400C01063E262126412BA50F000474BF
:104F50003820A00026710C30F000B171EBC40F00B6
:104F600048E104012C100C01E1F000003C10140099
:104F7000D9C1040038C30C0006E328D306000C7026
:104F8000EC1304240C308804B171CBF90100187EB5
:104F90003900CC70800092221860A3300C7024007D
:104FA00034D4F2132F570C001045C44392091875DE
:104FB000020034711377C47DD20A0667F2081855CF
:104FC0000100245226752377C67D22ED0C70BC3774
:104FD0002666266720762471A1760C70EC130424D3
:104FE0000C309404B171CBF9010058C104002C10AD
:104FF0001400E1F03C10080104240C400801264193
:105000002621B9F104012BA50F0004743820A0005B
:1050100026710C30F000B171EBC40F0038F10401BF
:105020002C100801E1F000003C101C00B131D9C186
:105030000C000C306C0406E2B9B1080006D406B5C9
:10504000B7514B00020086BB04C0920204B12F7C12
:105050000D001077062E0C30E000B1714B000200FD
:10506000B4B124C1820A067CD47792F2062E0C30A9
:10507000CC0A4B000200F2EC062E0C30CC0A4B009E
:10508000020058C10C0038B108002C101C00E1F0DF
:10509000085000400C70891338650400D4619203F5
:1050A000B47192FB08700040B127E1F0C43A3418A3
:1050B000C1E106E39204042D2B050200062E2B0508
:1050C000020040E12418E1F038609C000870008084
:1050D0002C70C040B1763860A000B1763870A40062
:1050E000086000802C60E020B167087000402C70E0
:1050F0000008B107087000402C700003B107B90721
:105100001000B9071400B9071800B9071C00B90747
:105110002000B9072400B9072800B9072C00B907F7
:105120003000B9073400B9073800B9073C00B907A7
:105130004000B9074400B9074800B9074C00B90757
:105140005000B9075400B9075800B9075C00B90707
:105150006000B9076400B9076800B9076C00B907B7
:105160007000B9077400B9077800B9077C00B90767
:105170008000B9078400B9078800B9078C00B90717
:105180009000B9079400B9079800B9079C00B907C7
:10519000A0000C600104B96710000461B1670870D9
:1051A0000F001117E1F000003C103800D9C12800B1
:1051B00006620674042826210C30A004B161B7D120
:1051C00004D06BC20F000CE0200004C826C126CD1D
:1051D000102CC42A9208042D2B050200102C2B053C
:1051E0000200F2062B050200B4E124D192EF58C16F
:1051F00028002C103800E1F0CC4013003414B1F139
:105200000672D209F20491372471F2022441B441AA
:1052100092FBF22B0662D463820B0474367606523C
:105220000667B4619135245192FD2672244106F33C
:105230000653575857F426F50663576C26F326F69F
:105240000664776106572461F203B1F52454B46112
:1052500092FD066477415463574126742461F2033A
:1052600091372471B46192FD30F12414E1F0000013
:105270003C101800D9C10800C1A108D000304B3A39
:10528000000008E000302CE0849D2CD0009A06A29B
:1052900030CE30BD6B0F00002B390000307E54C47F
:1052A0006474B17E0473B17DEB400000087000307F
:1052B000C4A12C70089A30E730D79203CB39000094
:1052C000C4C092032B4B0000087000302C70009A71
:1052D000B1B7EB100000C6DEC20A0C2024273F3E07
:1052E0000D006B880F002421B920740058C10800FC
:1052F00040A12C101800E1F0383074003418B9F1D6
:105300000400B1012B970F00C4200471267292068D
:105310000471F20430612662B161B47192FC38F11B
:1053200004002418E1F000003C101000D1C106E296
:1053300006D36B0F00002F7D0D0026D70C5068366A
:1053400057D12F7D050024D438670400265DB95E4F
:105350000400B9E70400B16EB9E6040020672461D7
:10536000A167EB10000050C12C101000E1F000000C
:105370003414B1F1067306524B980F00000005007B
:10538000AE0036005400720090001000CC200740A0
:105390008250CC208040824FCC208440824ECC2052
:1053A0008540824DCC5088400C20FF009249042457
:1053B000F2470C60042704200C7042002046C645CA
:1053C000823FB4712421246C92FA0C20FF00F23841
:1053D0000C60202C04200C7012002046C645823040
:1053E000B4712421246C92FA0C20FF00F2290C6085
:1053F000582A04200C701A002046C6458221B47138
:105400002421246C92FA0C20FF00F21A0C609025E3
:1054100004200C701F002046C6458212B47124215E
:10542000246C92FA0C20FF00F20B0C20FF00F20813
:105430000420F2060421F2040422F202042330F1D3
:105440002414E1F03C101400D9C10400B1B104D31C
:10545000067406E226D24B980F00000005001601E4
:105460001000320058008E00BE002F730300263754
:1054700057310C7004272637B823040020B38A7BE9
:105480000000F12004C1992E0300F26A2F7303007B
:10549000263757310C70202C2637B823040020B350
:1054A000826CF120992E03007724992D010004C20B
:1054B000F2572F730300263757310C70582A2637BE
:1054C000B823040020B3825BF1200672992E0300FA
:1054D0007774997D010006727778772C997D0200A8
:1054E000992D030004C4F23C2F7303002637573173
:1054F0000C7090252637B823040020B38242F12097
:105500008632824110C3062D2431064C2B9E0F009B
:10551000C4C092260420F23E2F7303002637573171
:105520000C701C2A2637B823040020C3822EF120D9
:105530008632822D18D30100107357D466D7DCD081
:10554000FF3F82270422044291CE262E77C4264DA7
:1055500099CE01002B9E0F000424262DF21B91BE34
:10556000042377B499BE010099CE0200262CF212D2
:105570000420F2100420F20E0420F20C0420F20A9F
:105580000420F2080420F2060420F2040420F202AF
:10559000042058C1040030B12C101400E1F00000C8
:1055A0003C102400D9C11400D981040006D3B141B4
:1055B00006C204E00480FA7B0000182C0100107C75
:1055C00057246627CC20FE7F248292600CA00627F9
:1055D00004B00C904200107AC47192082F2E0D0076
:1055E000133B0440CB22020026E2B49124B124AC48
:1055F00092F30CA0222C04B00C901200107AC4710B
:1056000092082F2E0D00133B0441CB22020026E20C
:10561000B49124B124AC92F30CA05A2A04B00C909B
:105620001A00107AC47192082F2E0D00133B044209
:10563000CB22020026E2B49124B124AC92F30CA058
:10564000922504B00C901F00107AC47192082F2E7E
:105650000D00133B0443CB22020026E2B49124B197
:1056600024AC92F30CA01E2A04B00495107AC471E5
:1056700092082F2E0D00133B0444CB22020026E299
:10568000B49124B124AC92F3F21106B277B6063B82
:105690002B1C0200CC20FF00063282082F2E0D00AA
:1056A0001333064BCB22020026E224C23071C68798
:1056B000AA85FFFF062E58C11400588104002C1043
:1056C0002400E1F03C101001D9C10001067506D29A
:1056D00006C306E44B980F0000000500BC00100054
:1056E0002A004C007E00A6002F74040026E70C70F0
:1056F000042757E126E7B87E0800824D1022F1709A
:10570000F24A2F74040026E70C70202C57E126E79C
:10571000B87E080018220100106D823D57246626CD
:10572000F170F2392F7E0E0026E70C70582A57E1EF
:1057300026E7B87E080018220300184D0200185D05
:105740000100106D822857246624572466255724AB
:105750006626F170F220064C0621063D2B9E0F00B6
:105760002F7E0E0026E70C70902557E126E7B87EC5
:10577000080026C1910C820F0621F170F20C2F74E3
:10578000040026E70C701C2A57E126E7B87E0800C3
:105790008202F17058C100012C101001E1F00000EC
:1057A0003C102400D9810400D9C1140006A306C20C
:1057B0009900AF3004D00C901C2AF2602F7D0C00B1
:1057C0001827010010675724662606B277B6063BF5
:1057D000B1712B1C0200C4B406E22F680C003071BA
:1057E00082071837020006262FD80300F20C042285
:1057F000262D262C10361072573466375C30FF3F4A
:1058000024D426D3CCE0FF008239134E065BCB367E
:105810000200067B4B980F0000000500620010009C
:105820001E002C003A004A002F6E0E0026E60C7077
:10583000042757E1F2152F7E0E0026E757E10C7082
:10584000202CF20E2F7E0E0026E757E10C70582A0E
:10585000F2072F7E0E0026E757E10C70902526E711
:10586000F2062F7E0E0026E757E126E91870AF30CA
:10587000186E030066769970AF300483268DC68A51
:10588000A29E9870C60092049900AF30F205C471D0
:1058900092039970AF30047258C11400588104000B
:1058A0009970C6002C102400E1F000003C10180094
:1058B000D9C10800C1A10CD0082704E004B00CA095
:1058C00034380CC04200B87D0400820BB07D8209E0
:1058D0002F2E0A00133B0440CB22020026E223EEC7
:1058E000B4C124B123BB24DC92EF0CD0242C04B02F
:1058F0000CA034380CC01200B87D0400820BB07DBF
:1059000082092F2E0A00133B0441CB22020026E21B
:1059100023EEB4C124B123BB24DC92EF0CD05C2A6B
:1059200004B00CA034380CC01A00B87D0400820BFF
:10593000B07D82092F2E0A00133B0442CB220200C5
:1059400026E223EEB4C124B123BB24DC92EF0CD0B9
:10595000942504B00CA034380CC01F00B87D04009E
:10596000820BB07D82092F2E0A00133B0443CB2209
:10597000020026E223EECCE0B503D206B4C124B186
:1059800023BB24DC92ECA9E0803058C1080040A180
:105990002C101800E1F000002830803034140C2066
:1059A0003438B1F1AB3D020030F12414E1F00000D5
:1059B0003414B1F10B7E0000C421922418701C44F1
:1059C000C471921C0C70D03F18670200C46192131E
:1059D0001867D500C46192051877D400C474820E8C
:1059E0000C70D03F1867E100C46192051877E000A1
:1059F000C474820499008F30F207047199708F305B
:105A0000F20399008F3030F12414E1F00C70683605
:105A10000460063704472F56060026565751245473
:105A2000B4412653A107B9570800B95704002461AF
:105A3000247C92F2085000802C50602106760C7075
:105A4000B43FB950B43F086001802C609C6CB967CA
:105A50000400086001802C609CE5B96708000860BC
:105A600000802C600821B9670C00086000802C6061
:105A70003421B9671000086001802C60505DB9675F
:105A80001400B9671800E1F006725C70F000CC7089
:105A9000F000920B542F34211322C42AD2080C7028
:105AA000842326271022F2040420F2020420E1F0CD
:105AB000987096303418C1E106E28205EB5402007A
:105AC000C421920399E0963040E12418E1F00000EF
:105AD0001870A4343418C471B9F10400821198709C
:105AE0009630820E3820A0000C30B004B171EBC4A7
:105AF0000F006B0F000099009630EB10000038F19A
:105B000004002418E1F0000018609B303414C461D4
:105B1000B1F1920B17A10C70183826761027B372CA
:105B20002212AB2C0000F20F0BB00000C42192092E
:105B30001820B430CC20FF0082046C208000F203D7
:105B4000CB29000030F12414E1F000003418C1E149
:105B500006E2CB290000062EEB58020040E1241893
:105B6000E1F000001870293E9970B3309970A330AD
:105B70000C60BC37047E9900C1309900C230B4710A
:105B8000A106246292FDE1F0045A34149950BF003A
:105B90000455B1F106760C7014359950143504642F
:105BA00099670100185060439907040099070500A0
:105BB0009907020099570300B900004606760C7059
:105BC00000460C60100099009A309900A9309900A5
:105BD000BE30A9007E309900AA30B9002430B90047
:105BE0004830B9070400A9070800A9670A00CB5B81
:105BF000020030F199009F309900AE309900923048
:105C00009900C330990097302414E1F03C108000D3
:105C1000D9C17000B9215400043006210C40540051
:105C200004C4D981600026C1AB9D0F00067C046EC0
:105C30001057B46164519157247692FB0CD0FDFF4C
:105C40000C90FFFF04BE04E00C80D4040C60BC3751
:105C500004AE105CD45106570C50043E82221855F5
:105C60002500C65E82370446264D4334C43D435D5D
:105C70000202044D4334C34532020450135504401C
:105C8000F2092F250500262610222451264213440E
:105C90001355C65302F7C649B215069406BEF21252
:105CA00018552500C65E920E3830A0000628B9614E
:105CB0005C00B97158000BC30F003871580038618F
:105CC0005C00B4A124E124D113EE24C623DD92C2EA
:105CD000F20206BE38715400062B910758C17000BD
:105CE000588160002C108000E1F000003C10100092
:105CF000D1C11C70600006E206D4917299020100C5
:105D00006B480100062E0C301C430B490100062E87
:105D10000C30E845AB49010099DE180077D499DED4
:105D2000190050C10C201E002C101000E1F00000E2
:105D300017A10470F2092F57030017221055247180
:105D4000C645242192062357C656A2F60421F20224
:105D50000420E1F00C601435067218560400F77147
:105D60005C70FF00F750C675542718660100A20A40
:105D7000144326462645C64712063665266713662F
:105D8000F20204600C501435247526751037184241
:105D900078016643914799650100E1F03C101000DD
:105DA000D1C186D406E28233C431921238702430D5
:105DB000042026D738704830B9D024302471B97007
:105DC00048304BAB000004214BAB0000F220C45024
:105DD000920527E8267DA7E8F20E38723803267D63
:105DE000B9723803182249034B1C0100C4218203F5
:105DF0000470F202047138604830C47126D6B9D0FC
:105E000048309205282E0C004B6B020050C12C101C
:105E10001000E1F00662F7615C60FF000C50143581
:105E2000542734142465B1F126651875040018321E
:105E30007801184501001026F770153356322F24CB
:105E4000070034249136C67204652667265614630B
:105E500006372664020A0461F20810F52431C4F002
:105E6000245182031352F205B461432392F7045084
:105E700034442674044526470C6014352664F20B1E
:105E800010463461C4408205367524741377F206D7
:105E900034714377C47032F504740C6014351846BD
:105EA00004005C50EF00265566549956040099761C
:105EB000010030F12414E1F03C101000D1C106E2E1
:105EC00006D306C606351C603000916299020100B7
:105ED0006B480100062E0C30E8450B490100062EE8
:105EE0000C301C43AB4901000C7011000461997E19
:105EF0001800996E1900187D1A0099CE1B00997E22
:105F00001A000C703F00186D1C00B471996E1C00D3
:105F100024D124E192F950C10C205F002C10100014
:105F2000E1F000003C101800C1A114A4D9C1080080
:105F300026A406E206C30CD01C00F24D2FBD0C00B7
:105F4000062B8B690000C421924224D813DD26CD94
:105F5000990E4803107CD47182040473997E48031F
:105F6000107CD4728206187E4803647C997E4803B4
:105F7000107CD4748208186E48031C70400066764A
:105F8000997E4803107CD4788207187E48036C7091
:105F90003000997E4803187E4803997E4903107C9F
:105FA0005C706000F772C472820AC473820AC471A2
:105FB0008204990E4A03F2080472F2040474F20295
:105FC0000476997E4A03990E3403F207187B010088
:105FD000247226D7C6DAA2B30C701000B90E3803AB
:105FE000B90E3C03B90E4003A90E4403A97E460333
:105FF00058C1080040A12C101800E1F03C102C0002
:10600000D9810C00B0B4D9C11C00B9310400910190
:1060100006E206D406C50686826A049004A00870CB
:10602000000F302B06315627772CB7D24B67000074
:106030001061375137D2C665922D285D0A00C49091
:106040002F650B0030669203B16DF2032659B165DE
:10605000C4609203B99D0400286D08003461A96DE5
:106060000800286C0A002F560B00B105B85C04002C
:106070009203B1BCF2032665B1B6286C0800C49047
:106080002461B9BC0400A96C080024A1920430BDAD
:10609000F206069B286D0A00266930B6C4B092C28B
:1060A000C481286E1000387E38039215366A236644
:1060B000C46026A7A96E1000B9AE38039218182E36
:1060C00049034B1C0100C4209212282E0C004B7176
:1060D0000200F20DC4A0266A367AA96E1000B97EBD
:1060E00038038205282E0C004B6B020058C11C009F
:1060F00058810C002C102C00E1F000003C10100026
:10610000D1C118E2490318F248031564566E564F80
:10611000666413E6064E56F556451565566EC64F2F
:10612000666F996249038213C6450C603C030C50AC
:106130003000266226529206064604608B800200DA
:10614000F2060645065604618B80020050C12C10F1
:106150001000E1F0341CC9E1040006E20623063118
:1061600091014B67000010714B980F000000040074
:1061700034000E00160020002A00182E4903F723D1
:10618000F211182E4903F7225421F20C182E49035C
:10619000F7215421F207182E4903F7205421F20267
:1061A000042048E10400241CE1F000003418C1E19F
:1061B00006E3EB59000017E15471C4719203247F88
:1061C000F202047426721077D471823FA870823074
:1061D00082483471386024302377A9708230A676E3
:1061E000924004204BAC000004214BAC0000F2397B
:1061F000B90E140010720667546CC4689232B377FB
:10620000320918321800062E54374B8B0200C42175
:10621000821F990E0900F20B187E35033471137733
:10622000C470997E35039203990E3403A87E120040
:1062300082043471A97E1200286E1200287E10009C
:106240002676C470820AF20DC4E092D3F20A187E58
:106250003403C47192ECF2E1282E0C004B71020061
:1062600040E12418E1F00000341CC9E1040006E21A
:106270000623063191014B67000010714B980F0007
:106280000000040034000E00180022002C00182E1C
:10629000490377235421F210182E49037722542101
:1062A000F20B182E490377215421F206182E4903C8
:1062B0005421F202042048E10400241CE1F0000013
:1062C00018609C300672D462823E06640C50100046
:1062D00090269206B451246192FC0440F237106774
:1062E000DC60FC0092040C501C00F2280C502200D0
:1062F000F2252F6507001026CC2030009219185681
:10630000080057512452135524582F750600107752
:10631000577124725C70FE002472267518560100B5
:10632000C65722132667907692110440F20F186622
:106330000100246226562355F2023434C65322DA71
:106340000440F2040440F20204400624E1F000009C
:1063500018704C423414C472B1F18268046126632F
:106360002F7302000C403D00236691470C5016002D
:106370002F76020091570C70043E246118476C0080
:1063800023662F560200914518776900C471820375
:106390000470F202047418506742C4519202647887
:1063A0002F560200997501000C504C4218751A00C6
:1063B00018552000C4519202647498509F3092097D
:1063C00018509730C45192071850BF30C4539203ED
:1063D0006C7010002F560200997502009905030099
:1063E00018706A42C47182030470F2030C7080005A
:1063F00018506B42C45192036C70000218506D42E9
:10640000C45192036C7000042F56020024669975E3
:1064100004002626777404300C401000997505009E
:106420006B1002000C201800F202042030F124143A
:10643000E1F0000018708F303414C471B1F192048F
:106440002B9B0200F202042030F12414E1F0000042
:106450001870B5303414B1F128507A300C30240063
:106460005771F211382714302F6302001046CC40C8
:106470003D0092042B9B0200F20818660100246282
:1064800026362333C635A2EF30F12414E1F00000A4
:106490003C103C00D9C12C00D9811C0018750A00A1
:1064A00006D2C47306C592091875D803C471920543
:1064B0009905D80304A1F20204A018709040C47298
:1064C0008A10010006933444FA0901002F790D0067
:1064D0001067CC602D009AFD0000047226792377A6
:1064E0000667266D0451995CD803B7D4187601006D
:1064F000106657746676437723E7138E06685461F7
:10650000996CD903066ED462921EC4A08205186CE1
:10651000DA03C461921B1860C900C463920B9860CF
:10652000664292080422B7D6CB6D000004B137D67C
:10653000F20204B0990CDA031860AE30246199605D
:10654000AE30F2050451995CDA0304B0D48C9203A6
:106550000461F20AC48492050452995CDB03F206DA
:10656000C48C92040463996CDB03066EDC6010003B
:106570009219C4A08205186CDC03C46192160C60E9
:106580004C4218562000C4518205045104B199565A
:106590002000990CDC0318609230246199609230DD
:1065A000F2040461996CDC03066E5C602000F76203
:1065B000996CDD03066E5C6040007763996CDE03C6
:1065C000066EDC600008990CDF0392060C50FF0E8B
:1065D000A95CE603F2050C60FF1EA96CE6035CE013
:1065E0000010C47077E699ECE4032219C4A0820578
:1065F000187CE003C47192160C704C4218671F009F
:10660000C4628205046204B199671F00990CE0031B
:106610001870C33024719970C330F2040471997CEE
:10662000E0031870C700C47192111870C500C471DE
:10663000920D18706C42C47192099870AD30045478
:106640009950C5009203EB460000379424952462CC
:1066500023662F760D0010575453995CE103107791
:1066600024617771547704E423990C80043E997C6B
:10667000E203236626E1269D06AC2C808A00047A7C
:106680000424044B26210638B795B7D62B9E0F005D
:106690001049105E24915654995AE80337D624E1E4
:1066A000B47124A1379592ED187CF1032C60100091
:1066B00023665C701F0026D6997CF103187D0100CB
:1066C0005774DC700004820E0461996CE303F20AD3
:1066D00018770100247226972399C6942AF8FEFFA2
:1066E00004B0987CD80392241870C9000C203300A1
:1066F000C4719AA7000018706642C473820704230D
:1067000004B1CB6D00006B6E000018709F302471D7
:1067100099709F301870C700C471920A1870C50034
:10672000C4728206C473820404739970C500C4B134
:1067300092032BA302003830A0000C2008050BC3E5
:106740000F00187CD8033820A0000C302005B17150
:10675000EBC40F00187CD9033820A0000C30400592
:10676000B171EBC40F00187CDB033820A0000C30A3
:106770006005B171EBC40F00187CDC033820A00069
:106780000C308005B171EBC40F00187CDD0338209C
:10679000A0000C30A005B171EBC40F00187CDE0323
:1067A0003820A0000C30C005B171EBC40F00187C7C
:1067B000DF033820A0000C30E005B171EBC40F00FE
:1067C000187CE1033820A0000C300006B171EBC446
:1067D0000F00187CE2033820A0000C302006B171B5
:1067E000EBC40F00187CE3033820A0000C304006F7
:1067F000B171EBC40F00287CE6033820A0000C30F8
:106800006006B171EBC40F00187CDA033820A000D9
:106810000C308006B171EBC40F00187CE403382003
:10682000A0000C30A006B171EBC40F00187CC000B2
:106830003820A0000C30C006B171EBC40F0004205A
:1068400058C12C0058811C002C103C00E1F00000C5
:106850009870BF303414B1F1824818709730C47109
:1068600082440C602400045004703434F2162FF675
:106870000200104FCC403D009206187F0400777252
:106880005471F204CC402D00920204512F460200B4
:106890001701244226642366C66322EAC450820399
:1068A000C47192230471042199709730CB6D00005C
:1068B0001870BF30C47192041870A230F2101870B2
:1068C000C700C471920A1870C500C4728206C473EE
:1068D000820404739970C50018706742C4719203F2
:1068E0006B6E00002BA3020030F12414E1F00000D5
:1068F000C430821D1853DB0330720860FCFF2C602B
:10690000FFFF567606655768083003005663C4518A
:106910006676B172920CB364320ACC408700C2072B
:106920001C6001FF56676C600087B162E1F00000F7
:1069300018708F303414C471B1F192032BC8020067
:1069400030F12414E1F000003C101000D1C1990393
:10695000010091031872D80306D2C47106E3927342
:10696000917398724C03820304739173987DE303CF
:106970008204107E6474917E287DE603CC70FF1E35
:106980009204107E6478917E18CDE103107E57C288
:1069900066C713CC062D0C30180091CEABB20000A8
:1069A000C4211C704000820A062D0C301000ABB2CE
:1069B0000000C42192051C70800066C7F209062DF4
:1069C0000438ABB20000C42192046CC0400091CEE8
:1069D000987DDA038206187E01006471997E0100B9
:1069E000987DDD038206187E01006472997E0100A5
:1069F000987DDE038206187E01006474997E010092
:106A0000987DDC038206187E01006478997E01007F
:106A1000987DD9038207187E01006C701000997E62
:106A20000100987DE0038207187E01006C70200051
:106A3000997E0100187DDB03186E0100577366769E
:106A4000997E010050C12C101000E1F03C1018009C
:106A5000D9C10800C1A120C206E228B2020006D3B3
:106A6000062C043706A46B880F002322C6B2D21F5F
:106A7000C4CAC21D287E0400286E06002471C461A9
:106A80002377A97E04009203A96E0800286E0800EF
:106A9000C667D20AC4D092080471A97E0600A90E66
:106AA00004000421F228A90E0600F224062C043367
:106AB0006B880F002322C6B2C21DC4CAC21BC4A069
:106AC0009213A87E0600820B287E08002677236793
:106AD000C463C2020473A97E0800F2040461A96EB3
:106AE00008000422F2020420A90E0400A90E0600E8
:106AF000F2020420207EC47AD203C4208204A10EB4
:106B0000A90E020058C1080040A12C101800E1F0A5
:106B1000C4213418C1E106E592093874C400B17586
:106B20003874C800B97E0400F21306234B3100000C
:106B3000C423D2036424132206720662577C57686A
:106B40006676667257246672B17EB97E040040E1B3
:106B50002418E1F03C101000D1C137E306D2B7F49D
:106B600027E206E3A7FD17E299031400A7FCA90397
:106B700016000623383D28006B0D0000383D2C0020
:106B80000426262E6B0D000050C104212C1010008D
:106B9000E1F000001C7064009900603099006130E1
:106BA0009900623099006330990064309900653033
:106BB0009900663099006730B9005430B900303020
:106BC0009900B2309900B8309900903099009E3009
:106BD000A970B600B9001C30B900EC2FB9004430E0
:106BE000B9004C30E1F000003C101400D9C10400A1
:106BF00006D2062C0C202E43B1B106B38B9A0F009F
:106C000013E20422262B2F7B0D00262D063C0C3090
:106C10002E43064E99E7010091072B9E0F00042298
:106C2000262E58C10400132230B12C101400E1F0BC
:106C30003C101800D9C10800C1A12F7302000461E3
:106C400091670C70F02E18B7010018770200267BB0
:106C50001367C468C202047804D22F63020026D3EB
:106C600016CB13A79976010026D213CC04E0F210BC
:106C7000C6EBB205062E8B260000F204062C2B284C
:106C8000000024E124C1912D13EE24D113CCC6EAD7
:106C9000A2F00422262A58C10800132240A12C1079
:106CA0001800E1F03C102000D9C11000D1810C6027
:106CB000F02E1876010018D6020006E226D713DD62
:106CC000C4D806C3C228049804A234D8369726A391
:106CD0002F6302000C50320013DD139926A204B07A
:106CE0009156062924B12B28000013BBC6BD912A5A
:106CF0002491139924A1A2F618708F30C4719205C3
:106D00001870C900C471920E26EC99DE010024D2DD
:106D1000132DF202042058C1100050812C102000C5
:106D2000E1F02F7D0E00267C0C607F0024D1996756
:106D3000020013DDF2EA00003414B1F110725C704D
:106D4000FC00CC7078008263CC7078001231CC707B
:106D50002800825FCC7028001215CC7010008A9237
:106D60000000CC7010001206C4708A8C0000C47839
:106D7000F21DCC701800824DCC7020009253FA8224
:106D80000000CC7040008241CC7040001207CC70F3
:106D900030008278CC703800F209CC705000823517
:106DA000CC7068008234CC704800923CF232CC70D7
:106DB000B400822BCC70B4001213CC70A00082629D
:106DC000CC70A0001207CC708000821FCC709000A5
:106DD000F21BCC70A400821BCC70B000F215CC70FA
:106DE000D0008213CC70D0001207CC70C000820D8E
:106DF000CC70C400F209CC70E4008207CC70F400BF
:106E00008204CC70D400920E0420F2470422F24592
:106E100017E1D47192392B170000C4208237042265
:106E2000F23CCC70A8008225CC70A8001210CC7067
:106E30008800821FCC7088001204CC708400F21687
:106E4000CC7094008214CC709800F209CC70C80009
:106E50008210CC70C8001205CC70B8009219F209EB
:106E6000CC70E8008204CC70F80092120422F21573
:106E700017E1D471920F2B170000C420820D042259
:106E8000F20C0421F20A0422F2080420F206042083
:106E9000F2040422F202042030F12414E1F0000094
:106EA00034142F640300B1F110560672CC50320036
:106EB000921DC47024421826010023448218C42065
:106EC0000461263404502662920E0461F20C1847C5
:106ED0000C002FF50700264F10F324515CF07F00C3
:106EE000243191F4B46192F4F202042030F12414BC
:106EF000E1F000003C101000D1C11C70400006E21F
:106F000006D49172990201006B480100062E0C30E4
:106F10001C430B490100062E0C30E845AB4901002B
:106F200099DE180077D499DE190050C10C201E009C
:106F30002C101000E1F000000450047004662F458E
:106F40000200B46110442451267492FA0627542F8B
:106F5000E1F00000862282109072820D06670657CB
:106F6000F7615457047153751856003015775675EC
:106F7000997600309102E1F034140C60D8370C702F
:106F80001000B1F1B471B106246492FD0C20003000
:106F9000043004426B100200047130F1997000302B
:106FA0001472997001302414E1F00000341404705C
:106FB000B1F11837003013270460045893F6920398
:106FC000C420820E06436346D441920A04515356AC
:106FD000D7216653262F995700301322F208B45157
:106FE000246192ED2471C47292E5042030F12414DE
:106FF000E1F000003C101000D1C1107206D2D47133
:1070000092186BFA020057210C70D837262730E20D
:10701000F20C062E063D6BAE0100C4219204382E00
:107020000800F20838EE0C00C4E092F40420F202EA
:10703000042050C12C101000E1F000003418C1E110
:107040004B00030086E28207902E92060BFE0200A0
:10705000912EF202042040E12418E1F03C101400CB
:10706000D9C1040006D206234B00030006E20C201F
:107070001C00262D0B6C00001822010006315C203C
:107080003800F72191014B67000010714B980F00F9
:10709000000004004A003A0028001C000E00062EE2
:1070A0000433044104528B880200F218062E043285
:1070B000044404588B880200062E04310C40100052
:1070C0000C5020008B880200F209062E04300C4080
:1070D00040000C5080008B880200990E340358C188
:1070E00004002C101400E1F038506C303418C1E169
:1070F00006760C702C32B9502C320C606400B967E3
:10710000040008E00030086001802CE0849D2C60C1
:107110007C4DB9070800B9670C00B9705430307E57
:1071200014625676B17E307E14635676B17E2B4B58
:107130000000307E1C6041005676B17E307E1C60BF
:1071400001045676B17E40E12418E1F00672D47154
:107150009205D42282050422F2040421F2020423BF
:10716000E1F000003C101000D1C106E2062306D376
:107170008B9A0F00187E19001322C67292110460B8
:10718000F20A2F560D00184E1A0060552461C645AC
:1071900024E1920A1356C657A2F50421F2061421DF
:1071A0002627F72FF202042050C12C101000E1F026
:1071B0003418C1E106E20B0B03000C701C43186786
:1071C0003300C66292141860D23FC46182121877ED
:1071D00000015CE01000C4729207C4E00421820246
:1071E00004201322F207162EF72FF2040420F202D5
:1071F000042140E12418E1F03418B9F104001073BF
:10720000D4718206042438F104002418E1F01870C7
:10721000B2300634064191718BA800001021F2F4BF
:10722000B3723C101000D1C106E206C3221504D08F
:10723000F20D2F7D0C00182722006B2F00004B3120
:107240000000C62E821424D113DD187C2E00C67DCA
:10725000D2F10420F20D0623063E5C307F00ABB273
:107260000000742113223421F72FF202042150C1AF
:107270002C101000E1F000003C101400D9C10400F3
:1072800018E0A530B1B106C20CB0183806DE34E102
:1072900013EE2F7E0B001027063CAB110300C42118
:1072A000920499EC0300F203B4D192F258C10400A5
:1072B00030B12C101400E1F03C101000D1C106D206
:1072C00004E00CC018382F7E0C001027063DAB11CF
:1072D0000300C421920499ED0200F20724E1187022
:1072E000A53013EEC67ED2F050C12C101000E1F094
:1072F0000C50D83704400C6010003075F20BB837D2
:107300000800820A1033C63292030647F205387726
:107310000C00C47092F5B461245492F00624E1F09C
:107320003418C1E1107206E2CC70FF0092101822EE
:1073300001002B18030086328205062E6B0D00001B
:10734000F206062E04300446AB9D0F0040E12418DF
:10735000E1F000003C101800D9C1080004300C40D6
:10736000CC02062E0C201C43B101A90104006B10B5
:1073700002000C20343006316BAE0100C4219213A0
:107380003830A0000C20E0060BC30F0018709E30B0
:10739000C4718209062E0C201C430C307001044677
:1073A0002B9E0F000CE01C430C706400A97E0600AD
:1073B0000472997E08000C70D007B97E0C0004722C
:1073C000997E10000C707700997E12000C70690095
:1073D000997E13000C706600997E14000C70690091
:1073E000997E15000471997E33000C706400A97EAB
:1073F00042000473997E440004300C70D0070446A8
:107400000C206A43B97E4800990E0900A90E0A00B3
:10741000990E1600A90E4C006B10020004300446B1
:107420000C207243A90E54006B1002000C207A430A
:1074300004300446A90E5C006B1002000472997EB1
:1074400067000471997E68000472990E6600997E47
:107450006900990E6A00997E6B00990E6C00997E06
:107460006D00990E6E00997E6F00990E7000997EE6
:1074700071000CE08E4304D4062E04300C401B0037
:107480006B100200B4D10C702800917E2CE01B0020
:1074900092F404300C401B000C2001446B100200DD
:1074A000043004460C20FA436B1002000CE01C432D
:1074B0000472997EE400997E0001047AB97E040189
:1074C0000430047104460C203244997E0801997EF0
:1074D0001000990E0101B90E0C01B90E1001A90E90
:1074E00014016B100200043004460C203A44A90E2B
:1074F0001C016B1002000C20424404300446A90E0B
:1075000024016B10020018709E30C47182090C2097
:107510002C01262E0C30700104462B9E0F000CE02F
:107520001C430C702B09A97E32010477997E34012B
:107530000474997E35010C702A09A97E36010C204D
:10754000BC440C70000204300C402500B97E3801A8
:10755000B97E3C01990E4001990E5001B90E6001AF
:10756000B90E6401B90E6801B90E6C01B90E700153
:10757000B90E7401B90E7801B90E7C01B90E800103
:10758000B90E8401B90E8801B90E8C01B90E9001B3
:10759000B90E9401B90E9801B90E9C016B1002004E
:1075A0000C705349A97EC6010C60E4440C70800045
:1075B000B4719106246192FD0CE01C430C706131A2
:1075C0000C2066450C300807A97E48020B9B0F0073
:1075D0000472997E6500997E640058C108002C10E1
:1075E0001800E1F03418C1E1062E0C20E845043003
:1075F0000C4018006B100200062E0C20E8450430E9
:1076000004466B1002000C20EE450C30FF000446CF
:107610006B10020004610CE0E8450473996E0D00E4
:10762000997E0E000462996E140018606043990EF2
:107630000C002666C46802031366F20204680C702C
:10764000E8459967150004619967160040E1241820
:10765000E1F000003C1018000C701800D9C10800BF
:10766000267106E20623C1A106D406C506A630B7D8
:107670004B310000C423D20857D154D466D21860CD
:10768000CD00132DF208B37232041860C930F20332
:107690001860C830307E1C4001FF572456745C20AF
:1076A000FFFF662708700FFF2C70FFFF562757CA91
:1076B0000870F00056C7662CB12EB9AE0800307BBA
:1076C0000850FF00B97E8400387B04002C50FFFF77
:1076D0005675385E8800083000FF56536675B97ECF
:1076E00088000676386E0400577456646676B97E54
:1076F000040058C1080040A12C101800E1F000005F
:107700003C102000C9A1080006A64860D000D9C1DD
:10771000100006E206B506C4C16106D3EB550000B1
:10772000062E133BEB570000062E133C2B57000090
:1077300026CB062E0631064BB1D1A9A10600A9C160
:1077400004006BB3010058C1100048A108002C10C0
:107750002000E1F03414B1F11C60780091629902CC
:107760000100EBA7000030F10C201A002414E1F016
:10777000C4513C1010000C701000D1C1267106E2FB
:1077800006C610D792234B3B0300C4C192152F723B
:107790000E0091079907010099070200990703005D
:1077A000187E01001C6080005C707F0024246676D7
:1077B0001322997E0100C4D1920F186E18001C701C
:1077C00080006676997E1800F2070478917299021B
:1077D00001000C20180050C12C101000E1F0000036
:1077E000147126721377C477D20618220B30162232
:1077F000F72FF2020420E1F01870B7303414C4718E
:10780000B1F19208AB3F0300742113223421F72F0A
:10781000F202042030F12414E1F0000018704F430C
:107820003418C471C1E106E2921606236B400300CE
:10783000C42082252F6E0E003870143F26E657E1D3
:1078400026E7287E08000421CC702000D202042004
:107850001322F2181870B730C47192132F6202000D
:107860003870143F26E657E126E7287E08000421F9
:10787000CC702000D20204201322F2040420F20271
:10788000042040E12418E1F03C101000D1C199031C
:10789000010006E29103102206D3AB3F0300C4218E
:1078A000920D0471917D187E4A035C70FE00647134
:1078B000917D187E4803997D010050C12C10100065
:1078C000E1F00000C4303C101000D1C106E206C354
:1078D00006D48276C420920606234B00030086E27B
:1078E000827104300C401000062D6B100200042140
:1078F000262D063C04462B9E0F00187E0C000C2003
:107900001000917D187E0A00C473925D185ED80342
:10791000187E0400C451186E2E0092030475F20EF6
:10792000C464D205C47BD2070473F208C468D205CC
:10793000C475C2030472F2020474997D0700987E34
:1079400005008206187D08006471997D0800987E04
:1079500007008206187D08006472997D0800187E71
:10796000C000C4738220B86E300382121876000201
:107970001866EE01D771C4646471137792046C7059
:107980002000F20FC462920D6C704000F20AC470C5
:107990008205C47482050471F2040473F202047750
:1079A000997D0900043A062E263DEB440300043C71
:1079B000062E263DEBCA02000C201000F204042023
:1079C000F202042050C12C101000E1F03C10200005
:1079D000D1811CB01000D9C11000069204E004D07F
:1079E0000CA0D83726B3067D5771267A30C7F20E21
:1079F000382C08002F4E0900063CCB46030026E237
:107A000023EEC6EB320638CC0C00C4C092F2F2036F
:107A10000CD0100024D113DDC4DFC2E6062E58C1FD
:107A2000100050812C102000E1F0000034140C20D4
:107A3000BE360C30FE00B1F10B4F030030F106767C
:107A40000C70BC369920BC36990701000627241417
:107A5000E1F000003C102000D9C1100006D206E37E
:107A600006C4062334D10631C9A10800B10106B508
:107A7000A901040013DD0B4B010034C4F20D2FAB40
:107A80000E00062A8B690000C421820A187A0100C0
:107A9000247226B723BBC6BC22F30470F231987D52
:107AA0000C30922D10610471997D0C3017D1576400
:107AB000666717D2175357746675175457746675EF
:107AC000175557746675085000302C50049CB165EA
:107AD000086000302C60089CB176187D0C30066D73
:107AE000C471576492030474F2020470646366679D
:107AF000087000302C70009CB167F2040471997D0D
:107B00000C3058C1100048A108002C102000E1F0F2
:107B1000C43034180478C1E1267110E7821506726A
:107B200006F2D77157F336F70C70C046267F38F748
:107B3000B800C43124F1B9F7B800C20638F7BC0068
:107B400024F1B9F7BC000672D771572336270C70A1
:107B5000C04626273872CC00C4E126373872C400EC
:107B6000B932CC0026573872C800B952C400264733
:107B70003872B000B942C8002667B962B0009207F7
:107B80003872D4002471B972D400F2063872B4008D
:107B90002471B972B40040E12418E1F0CC3000083F
:107BA000923317EF5C70FC00CC7080008234CC7094
:107BB0008000D210CC7020008221CC702000D20333
:107BC000C478F206CC7028008226CC704000921A4D
:107BD000F215CC70B8008214CC70B800D208CC700A
:107BE0008800820ECC70A000920DF215CC70C000FF
:107BF0008207CC70E0009206F2030421F20F042603
:107C0000F20D0420F20BCC300081920718220E00F6
:107C10005427F2040424F2020420E1F03C103C005A
:107C2000D9C12C000C40240006E306D20430062102
:107C3000C9A12400AB9D0F00907E38CE040018BE71
:107C4000010028AE020092040C702200F2020470BF
:107C500026B72FEB0C0004262621063E6B0D0000F4
:107C60000436263E06216B0D00009901180099018B
:107C70001900183E0C00187E0D0057346637CC30C2
:107C80000608A9312200820DCC300008820ACC30CF
:107C90008E888207CC3000818204CC30D98892173C
:107CA00024B626BCB9B10C001C705600917B997BA0
:107CB00001000473997B0200990B0300990B0400E7
:107CC000990B050034A6A9A11600F20824BE34AE13
:107CD00026BCA9A11600B9B10C0017D6B9C1100075
:107CE000D47182240474997115001870B730C4716E
:107CF0009205062E8B5D0300F2020426107D992169
:107D000014002F670700266757613F7706005771F9
:107D1000267D38771800062D0631F17058C12C00E9
:107D200048A124002C103C00E1F01870B230F2DCC5
:107D30003418C1E104300C409C04062E0C20C046CF
:107D40006B100200043004420C20582F6B1002000C
:107D5000067E0C70C0460C4032000461A9470E003C
:107D6000A9671600A9471A00A9672000044A04223F
:107D7000A9471C000C605433044799270100992738
:107D800002009927030099270400992706009927E4
:107D90000700992708009927090099270A009927C1
:107DA0000B0099270C00B94748009920C046184697
:107DB0006C000431045104211866680099370500ED
:107DC000A9571400A9271800045A04250431A957FB
:107DD0001E00A9272200B9373C00B94744000422FD
:107DE000A9071000A9071200B9072400B907280045
:107DF000B9072C00B9073400B9073000B967400053
:107E000099275400992770000422B92774000C2088
:107E1000F401B92788000C20C00BB9278400042284
:107E2000B9279C000C20F401B927A40004330422D4
:107E3000B93764009927A80004320C20E0050C50E3
:107E4000F401B9476000B937800099378C00B92731
:107E5000A000B9473404043304210442B957500048
:107E6000B9576C00B9379000B9272C0499474404DE
:107E7000042704431451143226562636B9273804F1
:107E8000B94754040C20F4010442B9675C00B96797
:107E90007C00B9577800B9579800B9379400B96792
:107EA0003004B92740042646B9074C00B9075800EA
:107EB000B9076800B9073C04B9074804B94750043A
:107EC00004220C40F40199276004B9475C040422A1
:107ED0000441B9674C04B9276404B9477004B96711
:107EE0006C040C20F40104620C40C00BB957680408
:107EF00099677C04B9277804B94774040463B957B7
:107F00008804B93784040C50E005042104320C4085
:107F1000F401B9678004B9579004B9075804B92728
:107F20008C0499379804B94794040C706C4704503A
:107F3000246DB4612451B157B9070400B907080092
:107F4000B9070C00B9071000B9071400B9071800E9
:107F5000B9071C00B9072000B9072400B907280099
:107F6000B9072C00B9073000B90734002C7038006D
:107F700092E140E19900582F9900592F2418E1F01F
:107F8000CC301F003C104C00D9C13C00D9812C00E2
:107F900006D2D207CC301700C207047C04C6F20612
:107FA000047E04C8F203047A04C4C4C004A126A752
:107FB000B97DE00157A1068D066D067C9202047121
:107FC00018340100174257345758102426351743E8
:107FD0002632575CB4712653B1562444246492F17E
:107FE0000431263C1471C63A267C5771267D066DF5
:107FF000065C04910CB084223F4C0A00D203C4A05A
:1080000092020441B9A1100006A506580686066D25
:1080100006D730ED062A063CB717B759B79ADB9654
:108020000F00862237173759379A922C062E063EB4
:10803000572C773466320623772C262B10E2062342
:108040005C20FF00262B102257EC66E206237724E3
:108050005C20FF007738262B5C30FF001022263B87
:1080600010335724573866E266E376E91399B3393B
:1080700032040C301B00F2020430269913997693D7
:10808000F21FC4C6C21DC424921B063E062E773CB6
:10809000263B5C20FF001033262B1022573C663213
:1080A000062E77245C20FF0077E8262B5CE0FF009B
:1080B000102226EB10EE5724663257E866E330387C
:1080C000B441763EB93D040024A124D4248492A274
:1080D00038A1100006851454265A0675577106D625
:1080E000267604C0046430283037B461B928F00023
:1080F000B937F00024C12484247492F60C703C003B
:10810000267C5771069C267D5791B7D4269D04A0E6
:108110000464F242064ED741063B73341333042EF7
:10812000B759B79AB7D8EB0B010024E1064ED741F7
:10813000063B7334B92114001333042BEB0B0100FD
:108140000431263E0642D731062B73230632133301
:10815000042DB717EB0B01000432263EB92118009D
:10816000D731062B7323063213330429EB0B01009E
:108170003717383114007643383118007643764289
:10818000914837D82481B4713759379A92C4B46171
:1081900024A124948208068A578130B9268104E0FC
:1081A0000474F2B9379406E10444B106107E183E17
:1081B0000100667057346673183E0200B4415738A8
:1081C0006673183E030024E4573C6673B17624645A
:1081D00092ED24C4C6C5A29358C13C0058812C001E
:1081E0002C104C00E1F000003C104400D9C13400D8
:1081F0000CC0100006D226C1B7180623064C063D57
:10820000D9812400CB0D01000CA0100026AD04B1D3
:108210000C9054220CE0441E068CF23F387520006E
:10822000B43157712671187713002F24010057714C
:10823000267E307706675764777C6667387510004E
:1082400057712671187712005771267E307776673E
:1082500006765774776C66763065245457612661CC
:10826000186611005761266E306676760667576489
:10827000777C66672F740800107724445771267E38
:1082800030777667B16292CB063A0621064C24B16C
:108290002CA010004B100100383DE001C6B3B20520
:1082A000065904400434F2BB0CE01000046026E1DF
:1082B00008F0FF00082000FF04542F760E0010C7BE
:1082C0003849100030795741577126712641387767
:1082D000100037045C7000FF564F66743849200068
:1082E000667C574126413704B45156422FC60100DF
:1082F0006674B17C2464249492E106E10C608422CB
:108300000444305EB44106750625777C26765C20F1
:10831000FF00107726261022577C667206257724E8
:108320005C20FF00775826265C50FF00102226565E
:1083300010555724667257586675B17E24E492E250
:10834000371857320621263D8B11010058C13400E1
:10835000588124002C104400E1F000003C10200063
:10836000D18106A60C602400D9C110002661309688
:108370000C6028002661067330360C602C002661E4
:1083800030C60C602000266120B60C6030002661EB
:10839000106606E4C46206D58204C46192031462C6
:1083A000916C06627764996C0100C430066777644B
:1083B000992C0200996C03000425997C0400262C5A
:1083C000820504482B9E0F00F205043004486B1010
:1083D0000200C4D0042D262C8207063D0C4020004C
:1083E0002B9E0F00F20604300C4020006B100200A0
:1083F000C4A00C202D00262C8207063A0C40100049
:108400002B9E0F00F20604300C4010006B1002008F
:10841000C4E00C203D00262C8206063E04482B9E1C
:108420000F00F205043004486B1002000C204500D8
:1084300004300448262C6B1002000C204D00262C22
:1084400004300C4010006B100200067BC4B077743F
:10845000997C5D0099BC5E0082080C205F00262C90
:108460000639064B2B9E0F000C205F00262B58C1AF
:108470001000232250812C102000E1F01C705600C7
:10848000917297E1047397E2C4521C70780097E6EA
:108490001C70720099020300990204009902050001
:1084A00097E79204047297E8F205C45192030471AD
:1084B00097E8067477749932090097EA972BE1F0F0
:1084C0003C101000D1C10CF0140026F110EF0CF09C
:1084D000180026F110DF0CF01C0026F10C701000C3
:1084E00010FF26711077C4F2D7716672920557D6C5
:1084F00066D723EDF207C4F1820323E7F20357E2C4
:1085000066E75744D7346643D75366455763664694
:10851000664E50C123242C101000E1F03C101000D6
:10852000D1C1243406D2993401001C7023000422E6
:1085300006E4917426240C30D43F04432B9E0F0094
:1085400099DE050050C12C101000E1F0C4403C1031
:108550002000D9C11000D18106E206A306D430C2A2
:10856000824B37E106640654D761F75E26752F5CAF
:108570000600C656B7E1B152B2032471B7E1F7C1A4
:10858000DCC03F00821E2F7C0D00CC704000C20575
:108590000CB0400036BCF20206BD0C901800269EBE
:1085A0002F2C0900063A064B2B9E0F0026CBCCC081
:1085B0003F00C222062E063926AB36DBEB4E010009
:1085C00006CD77C306BA24C1F207063B062E2CB0AF
:1085D0004000EB4E0100B4C192F9064D5C403F00F3
:1085E000C44077D357D32F3D0A0082060C201800D1
:1085F000262E2B9E0F0058C1100050812C102000F9
:10860000E1F000003C101800D9C10800047006E237
:1086100006D30468065777515751265E0637305502
:10862000D731B4612F47010073539154247192F3F1
:10863000307E0C403700F77136475C403F00062E15
:108640000C30202D24410BAB0300062E06310448CC
:108650000BAB030004700C501000066777612462B6
:108660005761266E06373066D731B4512F470D005B
:1086700073639164247192F258C108002C101800A1
:10868000E1F000000C70D03F1867ED00C461920764
:108690001877EC0076723471F77FF20204700627C7
:1086A000E1F000003418C1E118E0F4451870D23F41
:1086B00024E1C47113EE92070421CBB40300C4215A
:1086C000920264E4062E40E12418E1F00C70D03FE1
:1086D0001867D500C46192051877D400C672820D60
:1086E0000C70D03F1867E100C46192091877E00070
:1086F00076723471F77FF2040471F2020470062777
:10870000E1F0000018701C443418C472C1E1824EBC
:108710000C70D03F18670200C461924018771400B3
:1087200018E09C30C471D7E164E113EE8204C47593
:108730009226F2136CE0820004220BB70300C420DF
:1087400082046CE0400013EE04240BB70300C42045
:10875000822E6CE02000F22B6CE0860004220BB726
:108760000300C42082046CE0400013EE04240BB725
:108770000300C420821C6CE02000F21904220BB715
:108780000300C42082036CE0400004240BB7030004
:10879000C420820D6CE02000F20A98709D30920394
:1087A00004E2F20204E664E1F20204E0062E40E193
:1087B0002418E1F01870D23F3C102400C471D9C1D4
:1087C0001400D981040006E29AC600001072DC7021
:1087D000FC0092050CC01C00FAAF00000CC0220087
:1087E000FAAB000018709C300667D46282082F6CC8
:1087F0000E001066CC6030008AB80000D4718A90F8
:1088000000002F2C0E00AB640000C4219A890000E8
:10881000FAB0000024C423CC2F7C0E0010673870FF
:10882000DC3F0C202C00C6679A99000024C223CCA0
:108830002F2C0E00EB780000C4208AA500000463F2
:10884000266C23662F760E00246123662F560E00B9
:1088500010451097C44106745771247213870CC0D9
:10886000FF00920318C50500268623882F780E0086
:1088700010670CA0FF00C461B161920318A7050046
:10888000C4C0920206C918B0E43F0C202900C6B942
:108890009265062ACBB40300C4208A780000062C17
:1088A0000BB70300C4208A750000C4949205C4C2AB
:1088B0000C202E008253C4D292273071577124723B
:1088C000137726870C70D03F186701002388C46196
:1088D000920B18770300C47192072F780E0010775F
:1088E000D471825AF2062F780E001077D471925705
:1088F000C4B18203C4B5920826E8107ED472820403
:10890000C4C2920206CB0C70D03F99A7BF0099C792
:10891000C00099B7C10099D7C2000420F21F2F7C74
:108920000E001067CC603000823D18770100247281
:1089300026C723CCF20314D426D3C6CD2A54FFFF76
:108940001870E43FC4718203C47592079970904017
:108950000420F2040420F202042158C114005881BA
:1089600004002C102400E1F00C30D43F04D2F204B7
:108970000C30D73F04D1C4D124C223CC9A4EFFFF80
:10898000FA4AFFFF0C202800F2E90C202B00F2E647
:108990000C202A00F2E30C202D00F2E00C202D0028
:1089A000F2DD0C202800F2DA0C70D03F1867D400FA
:1089B000C66292039937D5000C70D03F1867E0006B
:1089C000C66292039937E100E1F000003C10180004
:1089D000C1A1D9C1080006A204E004D00CB0D03F68
:1089E00004C92F2E0E00262E5721362E57212C205B
:1089F000F400262B063A04468BA30F00C4208208FD
:108A0000B4C124D113DD24E192ED0CD0FF00062D7A
:108A100058C1080040A12C101800E1F00C70D03FA4
:108A20001827D5001877E1007421C4713421F72F7D
:108A3000920324211322E1F03C102800D9C1180030
:108A4000D98108000CC0D03F187C020006E2C47235
:108A500006A306B48A1F01008BD10300187CED0029
:108A600006D2C4719A190100267AC4B21377B7D11D
:108A7000920B2F7A0E000C50300024A2915723AA9B
:108A80000CC0D43FF21CC4B192192F7A0E0024A25C
:108A900023AA0CC0D73F1C6023002F2A0E00063CDF
:108AA000044324A3916723AA2B9E0F002F7A0E0064
:108AB000045124A1915723AAF20204C02F7A0E0078
:108AC00024A1046123AA91672F7A0E0024A123AA6E
:108AD0002F2A0E00063C044391072B9E0F000483AF
:108AE000268A0C70D03F238818571400C4D02F68F2
:108AF0000E002481238891562F680E00248192163F
:108B00000471238891762F780E00248123D82F2D8D
:108B10000E00063C044324D39107238D2B9E0F00A7
:108B20002F780E0091072481F262238891D62F6856
:108B30000E009106990102001867D5002481C461D6
:108B4000A101238892061857D40004D19151F20252
:108B500004D00C70D03F1867E100C46192082F6DFB
:108B600001001857E00024D113DD9156C4D18216BC
:108B7000C4B210619216C464821117510471F204D8
:108B8000C45482070472C67DA2FCC67D8207F2022D
:108B900004710454915126719167069804A0F22241
:108BA000C46282FC17510471F204C4528207047239
:108BB000C67DA2FCC67D82F2F20204710452F2EB81
:108BC0002F290E00063C04432B9E0F0004732679C8
:108BD0002F6A0100237710562494267E239924A11E
:108BE0009157137AC67DA2ED57D1268D23882F7811
:108BF0000E0024812388046191670CA0D03F2F7858
:108C00000E009107187AED0004D1C47126D823DD37
:108C100092102F2D0E00063C044324D32B9E0F00F0
:108C200023DD2F7D0E00185AEC0024D123DD91574F
:108C3000C4B292250C70D03F18670100C46192073E
:108C40001877030074713471F77FF20204700C60BE
:108C5000D03F3856CC003866A400575257615C505C
:108C60003000546C2F4D0E00266524D1267623DD6E
:108C700091742F7D0E0024D123DD91073791062DAD
:108C8000362613221471267226E62421917E1322A1
:108C9000F2040420F202042058C118005881080090
:108CA0002C102800E1F0000018709C303C101000DF
:108CB000D472D1C106D206C3820604426BD203002D
:108CC00006E2F20204E018709C30D471820A2F3C54
:108CD0000E00062D233304416BD2030026E223EE5F
:108CE000132E50C12C101000E1F000003C101000B9
:108CF000D1C12FD2020026D257D106E236D257D1A7
:108D00000C20C040262D04300C402C006B100200BB
:108D10000C70D03F38670C0026D7B9EDF000B96D64
:108D2000FC0050C12C101000E1F000003C101000BD
:108D3000D1C1062E0C20D03F04300C407C026B10B9
:108D40000200067E0C70D03F0462996701009967AB
:108D500002009967030004510C601C4399561000EF
:108D60009950D03F045299560001046F996705004D
:108D70000C6050001C50540099670800046199571A
:108D80000600B9670C00145E18609C309957090002
:108D90000452B95710000656D45299070400990797
:108DA00007008205046499671400F206D461820406
:108DB000045299571400087001000CE0D03F2C7049
:108DC000805104620452B97E1C000C2018070C70FC
:108DD0001E000438B96E1800B97E2000995E240088
:108DE000EBA401000C20F53F04300C4020006B1078
:108DF00002000473B97E9400187E14000463C472E8
:108E0000B96E900092060C500001B95E9800F2070E
:108E1000C47492050C608000B96E98000C70D03F4D
:108E20000C604600B967A0001860B7300C50C0A8AD
:108E3000C461B9579C0092050452B957A400F203CB
:108E4000B907A4000CE0D03F0C603C00B96EA8004C
:108E5000186E14000472045404300C4010000C20EE
:108E60007F40997EAC00995EAD00996EAE006B10AC
:108E70000200047104540C608000B97ED000995E39
:108E8000D400B96ED800997ED500045204620C70EB
:108E90000001B95EDC00996EE00004510461B97E06
:108EA000E40004200472B96EE800990EBF00990E28
:108EB000C000990EC100B90EC400B90EC800B90EA9
:108EC000CC00995EE100997EEC00995EED000BE824
:108ED00003000C20C4400C30FF0004466B1002005D
:108EE000186E140004D1996E000104E8132D0BE8EC
:108EF0000300B4E124D192FB50C12C101000E1F02A
:108F0000C4220C70D03F9927140092060C60000117
:108F1000B9679800F207C42492050C608000B96715
:108F20009800E1F00672D4713C101000D1C106E245
:108F30008A7400000672D472820DB372220B04612F
:108F400099601C4454E4046299E09D309960D23FDA
:108F5000F269046199601C449960D23F066EDC603E
:108F60001000067EF771547182030462F2020460FD
:108F700066760422043299709C30EBCD0300042401
:108F80000432EBCD0300B37E3219067E547413779E
:108F9000C47099709D30820504D50CC06800F2043D
:108FA00004D10CC02800062DABF803000C70D03F94
:108FB000B9C7980099D7AE00F220067EDC70400059
:108FC000820C0422ABF803000C6000010C70D03F4F
:108FD000B96798000462F20F067EDC702000820DF3
:108FE0000424ABF803000C6080000C70D03FB9671C
:108FF000980004649967AE00067EDC70200082054C
:1090000004240431EBCD0300DCE04000820B042299
:109010000431EBCD0300F206046299601C449960B0
:10902000D23F50C12C101000E1F000000672C47154
:109030003418C1E106238204C472920FF20428207E
:10904000B800F216C43028E0B800821128305E4320
:109050002B970F00E720F209C43028E0B800820700
:1090600028305E432B970F00C62EB202062ECC206E
:109070003601B2030C20360140E12418E1F0000073
:109080000C70C83399070900B877040082110C707E
:10909000A8340468B05782071845CC01C441920334
:1090A0009945D401B461247492F6B900CC33E1F04F
:1090B0001872CC01C471920A0C60C833387604006F
:1090C0009902CC013471B9760400047197E20C70F6
:1090D0001000A972FE0104719172E1F03C102000B1
:1090E000D9C11000D18117E517A45774667617B55A
:1090F0001893040057646669C67610B2172118A247
:10910000020018C2030010E3177118D3020018F30D
:1091100003009211574457A8575457D8664A665DC2
:10912000664B57CC665E57FC664C665FC645A2052B
:109130000420F20FC676B20A3F770600C47ED2083A
:1091400004462B9E0F000421F2040420F2020420A6
:1091500058C1100050812C102000E1F0C441B1052D
:10916000B90504008204C4429233F21D067208401D
:10917000FF005774562406635C70FFFF77285C601D
:10918000FF0057686672667606635C6000FF57688A
:109190006676B175087000FF667456737778B97596
:1091A0000400F21606735C70FF00577823226627CE
:1091B00006735C7000FF57786627086000FF087030
:1091C000FF00667656737778B125B9750400E1F033
:1091D000343143332623F20A107224711377C4709A
:1091E00091723421920534314333C43032F6E1F0C8
:1091F00034140438B1F12B0F040030F12414E1F0E1
:109200003C101000D1C10CE0C83306D22CE0100095
:109210000CC020000C201100063E064C262D2B9E73
:109220000F00062E063C2B0F04000471990D04005C
:10923000997D010050C12C101000E1F03C10180085
:10924000D9C10800B8C2E40106E2823218DC060087
:109250001862EF01067D5477C667922C062CEB95B9
:109260000000C4219205067DDC7030009225DCD020
:10927000C0009224187C05000667D4618221D47452
:1092800092210439263C044806212B9E0F0006211A
:109290002B1004000C30C4010621263E04488BA389
:1092A0000F00C4200471820204701327F20C042002
:1092B000F20A0420F2080420F2060420F20404203A
:1092C000F202042058C108002C101800E1F0000040
:1092D00034211322C424D20418226801F202042388
:1092E000E1F000003C103800D9C1280006E306C2B6
:1092F00006D404300C4024000621B9B1240006B580
:10930000AB9D0F0004262621063C6B0D00000621B4
:109310000C301C436B0D00000C701A00267EB7D376
:109320001C707277A97122001870B230A9D1160092
:10933000997115001870B730B9E11000C47192042A
:1093400099011400F2050C70100099711400C4B05A
:109350009205047199711800F203990118000471C3
:109360009971190006270C201C3C18701C3C063112
:109370002F670700266757613F77060057712672EF
:109380003877180099011A00F17058C12800182187
:109390001A0038B124002C103800E1F03C102C00E9
:1093A0000C702C00D9C11C00D9810C00267106E379
:1093B00030370C7030002671307714A1B1710C7009
:1093C00034002671B0B7068206D406C526A4825B97
:1093D000287E040023AA309ED7A126AE347E26978D
:1093E000286A0600287A040004262667307A044694
:1093F0002667047E267523772629B791B7D22B9E40
:109400000F003031062904462B9E0F0099C90D002C
:1094100077C499C90C0037D237910657D4538206C6
:1094200004443F5504001355F20204500440F20571
:109430002441910613442461C645A2FB286E040012
:10944000346EA96E0400286E0600246EA96E060014
:10945000286A06002665A96A0600286B0A0018CB50
:10946000030026762675A97B0A002F7D0C00997BC8
:109470000300187B0200995B06002471997B0200AF
:1094800004B0F21F24C426C623CC063C6B55000052
:109490000628133DAB580000063C0628D7A1EBB2C6
:1094A000010026AE287A060004C02474A97A0600BA
:1094B000F2E8063E062824B16B5C000023BB24E8DA
:1094C000C6BD2F4C0B002344A2F558C11C00588187
:1094D0000C002C102C00E1F03C102400D9C1140029
:1094E000D981040037E306C2E06706D306E43205FB
:1094F000E87718002A8C0000062C063D4BDB0200A2
:10950000F27F987E0B00921338BC1000062BB1BE80
:109510000B330000187B1400B92E0400997E0A005A
:10952000187C02002C701000A97E0800288E08000C
:10953000387E04002FB80700186B0C0018AB0D0024
:10954000576426A623AA046E266AD463820504946F
:1095500036961399F20204900436263B0446062DF3
:10956000B1712B9E0F000426262D063B04462B9E30
:109570000F003071248EB97D1000A9AD1A00A98D9D
:109580001800990D1400A90D1600187E0B00186E16
:109590000A0024711377C676997E0B00B20B287EE1
:1095A000080004222C701E0026A7269AA99E0800F7
:1095B000F227C6769224182E0C00187C0300242172
:1095C0001322C627992E0C00B216302EAB330000A2
:1095D00006D2B12E0B330000187D1400B92E040002
:1095E000997E0A000C701000A97E0800990E0B00ED
:1095F0000422F20676273421F72FF202042058C104
:109600001400588104002C102400E1F03830A00030
:109610000C2024070BC30F00987E0C008A73FFFFF9
:10962000F286000018704C423C103000C472D9C160
:109630002000C9A1180006E28A85010004B126B302
:109640002F7302000C602D0023BB91672F7B02005B
:109650000C601A00916718708F3024B1C47123BB5D
:1096600092690C60043E18767C001866680074717C
:10967000C4613471F77F9203647223771860584293
:10968000C4618208C46292036474F204C4639202E7
:10969000647C18607A3EC46192036C70100018609C
:1096A0007C3EC46192036C70200018607E3EC461F1
:1096B00092036C7040001860823EC46192036C702B
:1096C00080000C60043E18568000C4519208186651
:1096D0007400C46492020463576466761860C246DC
:1096E000C46192046C700004237728605A42CC60F5
:1096F000FF1E92046C700008237718609530C461D7
:1097000092046C700010237718607642C461920452
:109710006C700040237718605E42C46192055C70F3
:10972000FF7F6C7000802F6B0E00917677749976B6
:1097300001000C704C4224B21857130023BB2F6B4E
:109740000E0091561877140004AB0CC0043E26A1FD
:1097500057710C3095006675263C044B062A9176AD
:1097600024B12B9E0F00063A044B23BB06212B9EEF
:109770000F002FDB0E00062D0631044A2B9E0F0032
:10978000287C8400997D0A005C7000036774997DD1
:109790000B00187C8600C4719211187C8700C4717C
:1097A000920F186C8900187C8800C461577164732B
:1097B000137792076C701000F2040470F2020471C7
:1097C0000C504C42997D0C00990D0D00990D0E0026
:1097D000990D0F0018751600186517002677576445
:1097E0006676186515002CB0100074613461F76F4F
:1097F00066761865180023BBC4612F4B0E009203D8
:109800006C70000418606542C46192036C700008BB
:109810009174777497C11870A43E24B2C47123BBAD
:109820002F3B0E0082030470F20204721860A53E02
:10983000C461920264741860A63EC46192026478A6
:109840001860A73EC46192036C7010001860A83EB7
:10985000C46192036C7020000C50043E1865A50092
:10986000576366671875A600C47192036C600001A7
:109870001870AB3EC47192036C6000020C50043E41
:109880001875AC001845AB00D77AD74966741845EF
:10989000AD0024B4D74B66741845A80023BB5443CD
:1098A000D74566741845A90026EB5443D74666741D
:1098B0001845AA005443D7476674667606677764EE
:1098C00097B10860FF00566791737768777C97B20D
:1098D00097F3910E18750C00C4719202917E187066
:1098E000113EC4719204107E6472917E1870123E13
:1098F000C4719204107E6474917E1870133EC4711A
:109900009204107E6478917E1870143EC4719205A2
:10991000107E6C701000917E1870153EC471920517
:10992000107E6C702000917E1870163E0C201C007A
:10993000C4719209107E0C201C006C704000917E56
:10994000F202042058C1200048A118002C10300059
:10995000E1F0000018708F303414C471B1F192043A
:10996000CB310400F202042030F12414E1F00000B5
:1099700018704C42C4728230CC4080008204CC40CB
:109980005000920518706C3EC47282282F7302003A
:1099900024310C603E00233391672F730200046171
:1099A00091670C70043E186769002431C462233348
:1099B0002623920491020423F2123867700038774C
:1099C0006C00C667C205047191720423F208046337
:1099D00091620423F2040420F2020420E1F000006A
:1099E0003C101000D1C11C60300006E39162990266
:1099F000010038334C0106D206C46B480100062D25
:109A00000C301C430B490100062D0C30E845AB49D6
:109A100001000473997D1800990D1900186E020059
:109A200057C1996D1A00287E0A00186E03005773FB
:109A300026666676B86E3C01667C2377820CAC6045
:109A4000D80382091066C46192060462916E990E71
:109A50000100F204910E990E01005C70FEFF997DE9
:109A60001B007774997D1C00187E10000C202500C7
:109A7000997D1D00287E10007774997D1E0050C1CD
:109A80002C101000E1F000003C101400D9C10400BB
:109A9000B1B11C70300006D39172990201003833C5
:109AA000140006E206B506C46B480100062E0C3011
:109AB0001C430B490100062E0C30E845AB49010060
:109AC0000473997E18000471997E1900187D0400B2
:109AD00099BE1B00997E1A00990E1C00187D050086
:109AE000286D0800267757636676186D010057C108
:109AF0006676667C2377997E1D007774997E1E00BA
:109B0000187D0A000C202500997E1F00287D0A0080
:109B10007774997E200058C1040030B12C101400D5
:109B2000E1F000003C101400D9C10400B1B106E21C
:109B30001C70300006B6917206D406C59902010069
:109B40006B480100062E0C301C430B490100062E09
:109B50000C30E845AB4901000473D7C157D2997E58
:109B6000180066DC0472997E1900990E1A0099DEBD
:109B70001B0099BE1C00990E1D0058C104000C204A
:109B8000220030B12C101400E1F000003C10100055
:109B9000D1C11C707C0091729902010006D3383348
:109BA0004C0106E206C46B480100062E0C301C4333
:109BB0000B490100107D57C6C4725CC000F09203CF
:109BC00064C4F204C473920264C699CE100077C4D0
:109BD00099CE1100187D1A000C2018005772997E3A
:109BE0001200287D1A007772997E130050C12C1044
:109BF0001000E1F01870C146C471920B9900882FD3
:109C00009900892F99008A2F990098309900BC30CB
:109C10000C605C4B0C702000B4719106246192FDC5
:109C2000E1F00000E87218003232C430820F0C708C
:109C30004C4238673400C4312461B9673400C2062D
:109C4000386738002461B96738000C704C423867B7
:109C50004400C4512636B9374400921438672C00AA
:109C600038573C002461B9672C001564C665B206FC
:109C7000386740002461B96740002645B9408842F2
:109C8000F206386730002461B9673000E1F0000067
:109C90003C103400D9811400D9C12400306238D27C
:109CA000680006E238926C0006B3B792B713EB591E
:109CB0000000067D5C7000FF777426D70C701C4393
:109CC0003867780113A9266A06895C8000FFB967A6
:109CD000780138677C017784266813DDB9677C01D9
:109CE000386780013F580D00C4D02665B9678001F0
:109CF00006C2820D38676C01C4D12461B9676C015A
:109D00008206386770012461B9677001062EEB5333
:109D10000000C4238A990000C4B17798B991040067
:109D2000069C923D284E1800385E1400067E0460A2
:109D3000F233CC601000823406455443C441820C97
:109D4000C443922406320C301C4338436001244142
:109D5000B9436001F21B0C501C4338756801247133
:109D6000B9756801E07C3A7E0000182C1800063DA9
:109D70000648065A5427B1012B5903003711062C07
:109D8000063D0450CB610400F26D246128471C009D
:109D9000136677512474C44092CDF2020460187C9B
:109DA0000400D47182080C701C4338576401265B90
:109DB000B95764010C701C4338579001062B265B81
:109DC000B9579001B794AB940000379404C006488B
:109DD000065AE079320F1829180004715427063DFD
:109DE000B1712B59030037110629063D0451CB618F
:109DF000040024C113CCC6CBB213062ECB540000F2
:109E000086E28230EB5900000C606E00266E206600
:109E10000692B7910440045004D00461F2DB18703C
:109E20001C3CC471921837920870F0005676777A0D
:109E30001377C4758210C476820E38210C00063D5B
:109E40006BAD0000F2080C601C4338769801247159
:109E5000B97698010C601C4338769C012471B97660
:109E60009C0158C12400588114002C103400E1F0EA
:109E7000E872180032150C704C42386748003857A9
:109E80004C002461B96748001563C665B20638679F
:109E900050002461B96750002635B9309842E1F08E
:109EA0003C101800D9C1080006D2063D0621B101B8
:109EB000A90104006B0D00000621AB190300062167
:109EC0004B00030086E28261987ED803825E102EEA
:109ED000AB3F0300C420825918CD06000C702D0141
:109EE000267C5771267EB067920D2F2C0C00262CF5
:109EF00057212C20F403262E0430044CB1276B107C
:109F000002002CC02D0157C126CE186D0700307CF1
:109F10009167186D0900A9670200185D0800576471
:109F20006665285EE603A9670200C665C204A957F4
:109F30000200F208CC60FF00D2050C600001A967A6
:109F4000020098670600820A28670200CC60FF0FB3
:109F5000C2050C60FF0FA9670200186EE303C4611D
:109F60002867020092043C603200F2033C602E003D
:109F7000A9670200186D0B00A9670400185D0A00AC
:109F800057646665A967040058C108002C101800C2
:109F9000E1F000003C102000C9A1080006B2063B19
:109FA0000621D9C11000B101A90104006B0D000008
:109FB0000621AB19030006214B00030086D28AB0AC
:109FC0000000987DD8038AAC000098AB0A0018CB3B
:109FD0000600921218708F30C4719AA200000C70A3
:109FE000E600267C5771267DB0778A9A0000987724
:109FF0000E008A9600000C702D01267C5771267D7C
:10A00000B0E7920E2FEC0C0026EC57E12CE0F403A5
:10A0100026ED062E0430044CB1E76B100200987E4A
:10A0200006009206187DF2032471997DF203987E52
:10A030000600920C0C205C4B0C3020000C40FF0002
:10A040002B3600002421992E0A00987E0A00106EFB
:10A050009209C46092652CC02D0157C126CDB10C68
:10A06000F25F182B0700C460992E06008211286E3B
:10A070000200CC60FF0FC20C186DE303C4619204B0
:10A080000C60CD0FF2030C60D10FA96E0200186BAB
:10A09000090008F00030A96E0800185B080057643A
:10A0A0006665A96E080099AE0B00185DE203184DB5
:10A0B000E103383FA89A0CB0A89AD43126BF92FA8F
:10A0C000083080005771243154436673D746545783
:10A0D00066745755D72766756672B17B987E0B00FC
:10A0E000921F18708F30183E0600C47192192CC050
:10A0F000E60057C126CDB07C821328470C000653DA
:10A100002324C632C202065428471E00A9570C0059
:10A110002334C6630656C2020654A9571E0058C10E
:10A12000100048A108002C102000E1F03C101000A5
:10A13000D1C118E0BA300C402100062D0C20BC36ED
:10A1400004306B1002000C30210006CD0CC0BC3670
:10A150009930BC360C70200004F704340C202830F1
:10A16000997C010099FC0200993C0300AB190300A3
:10A170000C2028304B00030086D28A9900000C2066
:10A18000C0360C3028306B0D0000066E5762136627
:10A19000996C0A00987DD8038A8A00000C702D0102
:10A1A000267E5771267DB07782329057820464688C
:10A1B000996C0A009867060082080C60BC36185635
:10A1C0000A00645499560A002847020028570400E0
:10A1D0000C60BC3610F799460C0099560E00774477
:10A1E000775499F60B0099460D0099560F002857A1
:10A1F000080018470B0018370600995611007754CD
:10A200009936100099561200994613000C70E6001A
:10A21000267E5771267DB067822A18760E00C4719B
:10A2200092260C70BC3618570A00645299570A00DF
:10A230002846100028561E0018260A0018360C0062
:10A2400018F603009947160099571B007744775476
:10A2500099F71400992715009947170099071800D6
:10A260009907190099371A0099571C002CE0D6005D
:10A2700057E126EDB06E821B18761C00C471921750
:10A280000C70BC3618570A00645199570A002856BA
:10A290000A00184608001836050099571F00775421
:10A2A00099371D0099471E009957200050C10C2076
:10A2B000BC362C101000E1F03C101000D1C1987297
:10A2C000D8030C50D80310D22652824F067204E0F5
:10A2D000042004F8B845DC00821790648209046108
:10A2E0002662266310C664C891C60461F202046047
:10A2F00098440600820A046126622663104664447C
:10A3000091460461F2020460B8479803820B170E6D
:10A31000C441920804612662266310466442914655
:10A320000461B8475803820C18441C00C4419208C9
:10A33000046126622663104664419146F203C461BB
:10A34000920E044126422F620300264391D6066EE8
:10A3500010C457622422666C13229164B4F124E184
:10A360002454247492B8F202042050C12C1010001E
:10A37000E1F000003C101800D9C10800062E0C20A6
:10A38000BC3604300C400001C1A16B10020006AEC7
:10A390000CA0BC369900BC36046704750CB0D837E5
:10A3A00004E40CC01000990A0100996A0200997A2D
:10A3B000030030DBF20EB82D0800820DCCE0FF0068
:10A3C000D20A2F3E0A006B96040038DD0C0026E20C
:10A3D000C4D092F2B4C124B492ED13EE14610627F6
:10A3E0000C20BC36266E97A199E0BC3658C10800F7
:10A3F00040A12C101800E1F018708E303414C47491
:10A40000B1F192040B8A0400F2034B9C040030F17A
:10A410002414E1F03418C1E186E282050C70D803FF
:10A42000267EF20204702C30370057312637B07385
:10A430008229906799070600A90708009202B103D4
:10A4400018670A00084000303854A89A0C30A89ABF
:10A45000D451263492FA57616461B16398370A0087
:10A46000820734310C205C4B13336B3800000C70C6
:10A47000D803267EC4708206187EF2033471997E5A
:10A48000F20340E12418E1F03C101000C9E108009B
:10A4900006E2063E0621B101A90104006B0D000091
:10A4A0000621AB19030006214B000300C4208205DE
:10A4B000183E06004BA1040048E108002C101000D3
:10A4C000E1F000003418C1E1062E0C204C420430AB
:10A4D0000C40D0006B1002000462067E0C704C42EF
:10A4E00099604C42046399670C00046299670D00FF
:10A4F0000C60FF0EA9670E0004629967100099674F
:10A500001100996712000463996713000467996743
:10A5100014000462996715000463996716000462C9
:10A520009967180099671900046199671B00046214
:10A5300099671C0099671E0099671F0099672000A2
:10A54000996721000C603C00A9672200A9672400DC
:10A550000C602800A9672600A967280004629907F3
:10A56000170099071A0099071D0099672A00B90773
:10A570002C00B9073000B9073400B9073800B90713
:10A580004400B9074800B9075400B9075800B90793
:10A590006400B9076800B9077400B9077800B90703
:10A5A0007C00B9078000B9078400B9078800B907A3
:10A5B0008C00B9079000B9079400B9079800B90753
:10A5C0009C00B907A000B907A400B907B000B907FB
:10A5D000B400B907B800B907BC00B907C000B90793
:10A5E000C400B907C800B907CC00B9073C00B907D7
:10A5F0004000B9074C00B9075000B9075C00B90723
:10A600006000B9076C00B9077000B907A800B90766
:10A61000AC0040E12418E1F034140420B1F14BE423
:10A6200000000420EBE4000030F12414E1F000000D
:10A630001870A63034142471B1F19970A6306BB142
:10A64000040030F12414E1F0C4303414B1F1922A42
:10A650000C702200267218F71700183722001847CE
:10A660002300185724001867250018722E0018229E
:10A670002F0057746672CC7000089216CCF011004F
:10A68000921506735774667443771C40B03CC674C9
:10A69000920F062557246626762723223421F72F8A
:10A6A000F2080420F2060420F2040420F20204203E
:10A6B00030F12414E1F0000006633414F760B1F1C6
:10A6C000065204702461F2081845010010F5574441
:10A6D000264F26742452B46192F80663D431F76091
:10A6E00026662626820310622676066777685C70E7
:10A6F000FFFF267606277728267230F115272322BA
:10A700002414E1F03C101000D1C106E206D30C3055
:10A7100078006B0D00000426262E0C3080006B0D97
:10A7200000000C701C000468267D996E0C002377D5
:10A730000C604500996E0E00066777640C201A00C5
:10A74000996E1000997E11000C6011001C70800041
:10A75000262E0C309800997E1600996E1700990EDF
:10A760000D00990E0F00990E1200990E1300990E0C
:10A770001400990E1500990E1800990E19006B0E11
:10A7800000000C201E00262E0C30880004CE6B0E1C
:10A79000000026CE062C0C3014006BB604000672A6
:10A7A0007774997E19000C705000997E2300997E71
:10A7B00025000478267D1C603D002377996E2200D9
:10A7C000996E24000667992E180077640C202A00E1
:10A7D000262D996E2600997E2700990E2800990E45
:10A7E000290050C123222C101000E1F0C440341481
:10A7F000B1F19204CBB80400F202042030F1241429
:10A80000E1F000001860293E9960AB30E1F00000F3
:10A81000086000302C60205830761C5001035675BB
:10A82000085083FF6C7000022C50FFF35C201F0067
:10A830005675572966271C7001305627B126307689
:10A840006471B1760860003038762058D47192FD7A
:10A850000421E1F03C1014000C703C1404240C3072
:10A860008804B171D9C10400CBF90100CB3A0000D2
:10A870002B390000087000302C70049830670850A5
:10A88000FFFB2C50FFFF5665B1673077DC70000886
:10A89000820A04D004E8062D2BC10400B4E124D1BF
:10A8A00013DD92FA087000302C70049830671C5049
:10A8B00001085665B167087000302C703858306751
:10A8C00014535665B167306714555665B167087003
:10A8D00000302C70849D1461B167087000302C70BA
:10A8E000009A146208D0003004E5B167387D889D75
:10A8F000387D949D0420AB4D0000387D989D042147
:10A90000AB4D0000B4E192F3087000302C70809DD4
:10A910001461B1670C703C1404240C309404B171C0
:10A92000CBF9010058C104002C101400E1F0000024
:10A930003C1018000C701800D9C108002671C1A184
:10A9400030F70C701C00267130E70C702400267163
:10A9500006B630670C702000267110A70870003012
:10A960002C70385830D7573364D4B1D708D0003062
:10A970002CD0205830CD1C70390056C7067B547738
:10A98000D771667C1CC0C1005C30FF00567C6673CA
:10A9900054231C30010F56735725083083FF66720D
:10A9A0002C30FFFF5C401F00574956736674084007
:10A9B0007FFF2C40FFFF5674D7AB1C400130667AF6
:10A9C0005453567457566675B17D107F185F030057
:10A9D000577C6675185F0200084000305754667552
:10A9E000185F01002C400058575866750454B17424
:10A9F000265F187F040018450300577C66741845CD
:10AA0000020018550100574466745758084000303A
:10AA100066752C4004580458B174265F187F0800EE
:10AA200018450300577C667418450200185501004C
:10AA30005744667457580840003066752C400858D3
:10AA4000045CB174265F187F0C0018450300577C26
:10AA5000667418450200185501005744575866742B
:10AA60006675C460085000302C500C58B1758A854A
:10AA70000000C4B504F40428043C0850003010461B
:10AA800018D6030018C602001876010026F62626FE
:10AA90002636923A574C664D57C45778664C6647EF
:10AAA0000C703C582675B14718760400184F030007
:10AAB000577C6674184F020057446674184F0100A3
:10AAC000574866740C4040582645B1741876080003
:10AAD0001723577C6674172257446674172157480A
:10AAE00066740C4044582645B17418760C0017B3B0
:10AAF000577C667617B22C5048585764667617B163
:10AB000057686676F239577457C8667C667457DCA6
:10AB10000C4048582645667DB174187F0100184FD7
:10AB20000200577457486674184604006674184F3C
:10AB30000300574C66740C4044582645B17417E125
:10AB4000172257745748667418460800667417230E
:10AB5000574C66740C4040582645B17417F11732B3
:10AB600018660C00577457486674667617B32C50F5
:10AB70003C58576C6676B175107E186E010057749C
:10AB80006676086000302C601858B176187E040094
:10AB9000186E0300577457686676186E050066765F
:10ABA000186E0200576C6676086000302C601C58E6
:10ABB000B176087000302C70205830676461B1673E
:10ABC0000860003038762058D47192FD087000304B
:10ABD0002C7004983067DC600008820858C10800B7
:10ABE000042140A12C101800E1F030676C600008CF
:10ABF000B167087000302C70385830676462B167F4
:10AC0000F2EE00003C102000D9C1100086E2825014
:10AC100004202BC1040098709D309225062E043527
:10AC2000CB760000063E0C20F80004450BA701007F
:10AC30000CD01C43182D0101063E0C402800EB42AD
:10AC40000100182D01010C70EE450430044004523F
:10AC50000460B1E1B7D1B9010800B9010C002BCAF9
:10AC60000400F226C4749224062E043DCB76000024
:10AC70000C200001063E044D0BA701000CD01C4324
:10AC8000182D0101063E0C406800EB420100182D12
:10AC900001010C70EE450430044004520464B1E13B
:10ACA000B7D1B9010800B9010C002BCA040058C182
:10ACB00010002C102000E1F03C103800D9C1280011
:10ACC00006E20C201800043026210C401000AB9D39
:10ACD0000F002F7E0E00267E0667D7612676046160
:10ACE00026670C308E4326360C601C432676187778
:10ACF0007200B9011000CC706800A9011400820430
:10AD000004600445F2030464044D0C501800047000
:10AD100026512FF7030010DF2F270500247191D251
:10AD20001327C624A2F70C701000B1512671062E0D
:10AD3000043004400452B7D1B9010800B9010C0035
:10AD40002BCA040058C128002C103800E1F0000084
:10AD50003418C1E106E2EB420100062E6BE6040066
:10AD600040E12418E1F000003C103400B9B12000AB
:10AD700006B20C201000D9C12400262106D306C437
:10AD800004300C401000AB9D0F002F7D0D00267D80
:10AD90000667D7612676046126670C508E432656D7
:10ADA0000C601C43267618777200CC706800820411
:10ADB00004E00465F20304E4046D04702F37050019
:10ADC0000C4010002641102326472471912413477C
:10ADD000C646A2F5062C0C30EE456BAE0100C42130
:10ADE0009206087000302C703458B1E70C701000D7
:10ADF0002671062D064B066E04300451B9C10400BD
:10AE0000B171B9010800B9010C002BCA040058C186
:10AE1000240038B120002C103400E1F03C10100068
:10AE2000D1C10CE01C4318DE01014B1B00002F7D3B
:10AE30000D00267D0667D7612676267E18477200AC
:10AE40000632062D2BEB0400183E010104200C40B5
:10AE5000EE45EBEB040050C12C101000E1F00000B7
:10AE6000087000302C7028583057087000302C7053
:10AE70002C5830670675777497E50676777C97E3EC
:10AE80000870FF005676777897E2067677749764B5
:10AE900097E19162E1F00000087000302C703058AA
:10AEA000306714575665B16730676464B1673067BF
:10AEB0006468B16706570C501C4318601C43187532
:10AEC000010057646667187502001845030057743F
:10AED0006674184504005774185505006674577455
:10AEE0006675085000302C501058B165086000306D
:10AEF0002C601458B176E1F018208D300C601C43A2
:10AF000004761056B47126251322246192FB9920F1
:10AF10008D30E1F0087000302C7028983067646143
:10AF2000B16708700030F2033867009838672898D6
:10AF30000C502898D461265792F830251322F72018
:10AF4000E1F000000870003034142C703C98B1F12E
:10AF50003067042A7461B1676B18020030F1B900E0
:10AF600044302414E1F000000C70C0461867380427
:10AF70001857540457665754666518578C0466650D
:10AF80001857700457526665085000302C500099CD
:10AF9000B165186734041857300457626665085065
:10AFA00000302C500499B1651867500418574C04B0
:10AFB00057626665085000302C500899B1651867D3
:10AFC0006C041857680457626665085000302C50AE
:10AFD0000C99B16518678804185784045762666530
:10AFE000085000302C501099B16528675804285734
:10AFF0003C0457686665085000302C501499B165C0
:10B000002867900428577404576866650850003014
:10B010002C501899B16528675C042857400457687C
:10B020006665085000302C504499B1652867940437
:10B030002877780457686667087000302C70489944
:10B04000B167E1F0CC20FF00920AC4309204B9004D
:10B05000DC2FF2100471B970DC2FF20C3870DC2F89
:10B060000860000C2C70850557742676262757211A
:10B07000B132E1F03870DC2F0860000C2C708505CF
:10B0800057742676267257713077B173E1F000005D
:10B09000CC20FF00341CC9E1040006E282190C2018
:10B0A000FF000631B1014B040500B0719208CCE0FD
:10B0B000F0000421C20204201322F20DC471920A8E
:10B0C000CCE041000421C20204201322F204042136
:10B0D000F202042048E10400241CE1F03418C1E12C
:10B0E00006E21820C2002B050500C4219206182094
:10B0F000C200063ECB02050040E12418E1F000004A
:10B100001820C2003418B9F10400B1012B05050064
:10B11000C42192061820C20006314B04050038F104
:10B12000040030212418E1F008700F002C70F0FFAB
:10B130005672063277725772543F26373418573793
:10B140000C20BC00B131B9F10400CB0205000C7039
:10B1500049000C20BD000637B171CB0205000C2060
:10B16000BD0006314B0405003071D47192F938F1FD
:10B1700004002418E1F00000087000302C70001E5C
:10B180003037087000302C700810306704516C6044
:10B190008001B167086016302C6034080870FEFF2B
:10B1A000B1562C70FFFF0850163056732C50001CFF
:10B1B000B175087016302C70041C0C40001EB1478D
:10B1C000085001000870163066532C70081CB157E7
:10B1D000087016302C700C1CB147087016302C709B
:10B1E00044080452B157087016302C706808B10733
:10B1F000087016302C705408B107087016302C7087
:10B200004C080451B157B106E1F000003C10AC000D
:10B210000C30FC1D0C4048000621C9E1A4002B9E07
:10B220000F000CE0480026E1062E0C30A01D0C405B
:10B230005C002B9E0F00086016300C701700305E0B
:10B24000B471B956281124E492FB06E10860163067
:10B250000C701200305EB471B9562C1124E492FBCC
:10B2600048E1A4002C10AC00E1F00000341C0434D0
:10B2700004212631B9F10800B9010400B1014B04E1
:10B280000500042206314B04050037D130615774A4
:10B29000267606677766546FC469B970F42FC204C6
:10B2A0002C603700F2032C6030000C50003599659B
:10B2B00001000C602E009965020006677764546FE8
:10B2C000C469C2042C603700F2032C6030000C50BB
:10B2D0000035996503000C602E009965040006672F
:10B2E0007762546FC469C2042C603700F2032C608B
:10B2F0003000547F0C500035C479996505000C600E
:10B300002E0099650600C2042C703700F2032C70E1
:10B31000300006560C5000359975070038F10800CA
:10B32000047799700035241CE1F000003414B1F169
:10B3300010721451043104680645544706F353F45F
:10B34000B461064F66471374345192F7917230F12D
:10B3500004282414E1F0000004573C101000067685
:10B360000C70043ED1C19950043E0C601000045191
:10B37000B967040004629957080099570900996752
:10B380000A0099570B0099670C0099670D0099679F
:10B390000E0099670F00996710009967110099676F
:10B3A00012000458046699571300A96714000C5042
:10B3B00016000C602500A9571600A96718000C504C
:10B3C00031000C603400A9571A00A9671C000C500A
:10B3D00038000C603C00A9571E00A96720000C50E3
:10B3E00040000467A95722009967260004510C60A9
:10B3F000100099572700A9672C00045299072400D0
:10B4000099072500B907280099572E0099572F0052
:10B41000995730000C60353E047CB471910624616C
:10B4200092FD9900413E0C60423E047CB47191064D
:10B43000246192FD0CE0043E04620471990E4A00FE
:10B44000990E4B00B90E4C00990E5000B90E5400E5
:10B45000996E5800996E5900996E5A00990E5B00CA
:10B46000997E5C00996E5D00996E5E00996E5F003A
:10B47000990E6000996E6100996E6200996E63008A
:10B48000996E6400997E6500997E6600996E6800E9
:10B49000996E6900B90E6C00B90E7000996E740057
:10B4A000996E7500996E7600996E7700997E780096
:10B4B000996E7900996E7A00996E7B00996E7C0086
:10B4C0000430044A062D0C208E3E996E7D00996E44
:10B4D0007E00996E7F00996E8000996E8100996E52
:10B4E0008200996E8300A90E8400996E8600996E81
:10B4F0008700990E8800996E89006B100200062D56
:10B500000C208E3E0B1A0500992E94000430062D57
:10B510000C20993E044A6B100200062D0C20993E27
:10B520000B1A05000452992E9F00995EA000995EA7
:10B53000A100995EA200995EA300995EA400990EF5
:10B54000A500995EA600995EA700990EA800990E25
:10B55000A900990EAA00990EAB00990EAC00990EA5
:10B56000AD00B90EB00050C1995095302C101000AC
:10B57000E1F000003C102400D9C11400D98104007E
:10B58000CB2900001870CC00B121C4719257046817
:10B5900006B70CB0F02E9960F02E04730465997B09
:10B5A0000100996B020004760C6018000CA0FE2BC1
:10B5B00004E004D00C90FC2B1C80800004CC997B10
:10B5C0000400996B0300107A2F2E0E00C4762F3DD5
:10B5D0000D00262E263D262B263924258206C47CE6
:10B5E0008204CC701800920E04432B9E0F002F7E15
:10B5F0000E00267E267B18670500666899670500A1
:10B60000F212C479820DCC701200820ACC70240030
:10B610008207CC7030008204CC703600920904435B
:10B620002B9E0F00107B24E1C6E78ACC0000B4C13A
:10B6300024D124A392C9FAC60000C47092460464BF
:10B6400006B70CB0F02E9960F02E0CA0FE2B047201
:10B65000046104E004D00C80FC2B04CC997B010035
:10B66000997B0200996B0400997B0300107A1461A6
:10B67000266713662F9E0E00C4612F3D0D00269E87
:10B68000263D2F290B0026382425D20D04432B9E5E
:10B690000F00269B187905001C608000667699795A
:10B6A0000500F208C4758203C47B920904432B9EF3
:10B6B0000F00107B24E1C6E78A850000B4C124D1C5
:10B6C00024A392D5FA7F0000C472923A046C0697C4
:10B6D0000C90F02E9960F02E0474046899790100A2
:10B6E000996902000471046B0CB0FE2B0CD0F52E8E
:10B6F00004E00CA0FC2B1C80800004CC9979040091
:10B70000996903002F3E0E00263E2F2309002425B1
:10B71000263A04432B9E0F00107B146126671366A4
:10B72000C461C205C4758203C47B9204107D66782F
:10B73000917DB4C124E124B324D392E5F243C473D0
:10B740009241046C06970C90F02E9960F02E0477CD
:10B750000465997901009969020004710C60180070
:10B760000CB0FE2B0CD0F52E04E00CA0FC2B1C80A2
:10B77000800004CC99790400996903002F3E0E00E3
:10B78000263E2F2309002425263A04432B9E0F0032
:10B79000107B146126671366C461C20CC475820AEB
:10B7A000C47B8208C4768206C47C8204CC701800F4
:10B7B0009204107D6678917DB4C124E124B324D332
:10B7C00092DE30210B2B000058C114005881040078
:10B7D0002C102400E1F00000045206760C70543363
:10B7E000B950543304690454B9670400B9570C00C4
:10B7F00024670C503800B9670800B9571000B967C2
:10B800003C0004520468B9571400B9573800B967AE
:10B8100040000454B96748000464B9574400B9575C
:10B820004C00B967500004580C60FFFFB957540032
:10B83000B9675800045A0468B9575C00B9676000DA
:10B840000C502000046AB9576400B9676C000C50B2
:10B85000FA000464B9071800B9071C00B9072000F2
:10B86000B9072400B9072800B9072C00B907300030
:10B87000B9073400B9577000B9676800E1F00000FB
:10B880001870603EC47292050672DC702000921D32
:10B890001870613EC47292050672DC704000921707
:10B8A0001870623EC47292050672DC7080009211BC
:10B8B0001870683EC472920F5C200020C42004718E
:10B8C000820204701327F2080420F2060420F20416
:10B8D0000420F2020421E1F09870BE0092072F7359
:10B8E000020010676C60200091671870613EC4719F
:10B8F00092072F73020010676C6040009167187008
:10B90000623EC47192082F73020010571C608000C1
:10B91000666591670C70043E18676600C461920A00
:10B9200018776500C47192062673267210676464E6
:10B9300091671870683EC4719207243126231072F3
:10B940006C7020009172E1F034180461C1E12F7332
:10B950000200916718601C44C46192040C601100DD
:10B96000916704E126E326E2910E6B47050018700B
:10B97000C146C4719206106E1C7080006676917E7E
:10B9800040E12418E1F000003C1020000C70200081
:10B99000D9C11000D181267120870C70240006E2E5
:10B9A000267106D3043A1097263D916E06C406B55B
:10B9B0009902010006A66B480100062E0C301C43BC
:10B9C0000B490100062E0C30E845AB490100062E5C
:10B9D0000C301800EB4A050099CE1C0077C499BEC4
:10B9E0001A0099CE1D000C301E0077B4062E0CC034
:10B9F0001E0099BE1B002BE2020026C223CC063C8F
:10BA0000062ECBE502001870B73026C2C47123CCD5
:10BA1000922B0C601C003484F2252F760D001057F9
:10BA2000CC50DD00923D98570200923A185703001F
:10BA3000CC505000923518570400CC50F200923090
:10BA400018570500C452922C98570600922918776F
:10BA50000700C4719225062E063CCB9E00001322DF
:10BA6000F204C66822DB0420C4912FDC020023DD2F
:10BA7000920E063D064A062E4B4B040026D223DDCD
:10BA8000063D062E4BA2020026D223DD0424262DDD
:10BA900058C11000232250812C102000E1F02F7695
:10BAA0000D0018770100247226672366F2DB000080
:10BAB0002F73020004639167046199670100187095
:10BAC000293E2432C47D2623D20424711377F20246
:10BAD000047D91720423E1F02F7302000C602A00B0
:10BAE000916724320461996701002623910218703E
:10BAF000CC00C4728203C47392139870A93082037D
:10BB0000047191721870C500C4729204107264724C
:10BB100091729870BE308204107264749172042322
:10BB2000E1F000001870B5303414B1F128507A30CB
:10BB30000C3024005771F212382714302F630200A2
:10BB40001046CC402A00920513336B570500F208CB
:10BB500018660100246226362333C635A2EE30F182
:10BB60002414E1F03C101000D1C10C70500006E22A
:10BB7000243A9902010091726B480100063D0C3095
:10BB80001C43062E0B490100062E0C30E845AB493C
:10BB900001000CD01C43287D4200062E997E200017
:10BBA0000C3022007774997E2100EB4A05000C309E
:10BBB0002400062E0CD02400EBDF020026D223DD69
:10BBC000063D062E2BE2020026D223DD063D062E80
:10BBD0002B56050026D223DD133D062E6B5705009C
:10BBE00026D223DD063D062ECBE5020026D223DD3C
:10BBF000063D062EEBE503001870B73026D2C4715F
:10BC000023DD9206062E063DCB9E0000F2020420A4
:10BC100026D223DD063D0C405000062E4B4B04007F
:10BC200026D223DD063D062E4BA2020018708F306F
:10BC300026D2C47123DD9208062E063D0C4050002A
:10BC40002B4C0400F202042024D4262D50C12322C0
:10BC50002C101000E1F000003C101000D1C118724F
:10BC6000160006E21C5080005C70F0000C30EE45BF
:10BC700091529902010099020200990203009972FF
:10BC800016006B480100063D0C301C43062E0B4984
:10BC90000100062E0C30E845AB4901000CD01C43D6
:10BCA000287D4200062E997E20000C3022007774F9
:10BCB000997E2100EB4A050098709030920A062E7A
:10BCC0000C302400EBDF02002C20240023D2F207EA
:10BCD0000CD02600990E2400990E2500063D062E54
:10BCE0002BE2020026D223DD063D062E2B56050050
:10BCF00026D223DD133D062E6B57050026D223DD09
:10BD0000063D062ECBE5020026D223DD2F7D0E0058
:10BD1000046591670454995701009907020018506F
:10BD200060439907040099570300990705001870AC
:10BD3000B73099D0B030C47124D623DD9206062ED8
:10BD4000063DCB9E0000F202042028707E3026D2F1
:10BD500023DD2627063DA9207E30062EEBE50300D5
:10BD600028707E3026D223DD2627063DA9207E308E
:10BD70000C408000062E4B4B040028707E3026D2EB
:10BD800023DD2627A9207E30063D062E4BA2020089
:10BD900028707E3026D2262718708F30A9207E305A
:10BDA000C47123DD9208062E063D0C4080002B4C0A
:10BDB0000400F202042028707E3024D42672262D3E
:10BDC00050C12322A9707E302C101000E1F0000039
:10BDD0009870BE303414B1F192114B3100008622BC
:10BDE000820FC423D20F1820BE00C422920C182048
:10BDF000C30074211622F72FF2060421F204042155
:10BE0000F202042030F12414E1F000003C1028007C
:10BE1000D9C1180098E09B30D9810800A10199018F
:10BE2000020006C206A39207B37332050BB00000EE
:10BE3000C4208270C4E199A1020099A1010091A1DE
:10BE4000339A82071860A5300C70183804D0F20AB3
:10BE500018DC0100F20910572471C65A820524D15A
:10BE600013DDC6D6A2F91870A530C67D822D0473E5
:10BE700006E126710C801838F79FF21D186C02003D
:10BE8000C66D920391AEF21D34D113DD2F6D080003
:10BE900010B6066BF763C696920E062B063CB7D11A
:10BEA000AB110300C42137D19206C4D091BE8206E3
:10BEB00006ABF207C4D092E3F20206AB04D091AE17
:10BEC00024E1C6E792F804B306E126B110DE062DA0
:10BED0002B6F0500C4D3D2045721542466D291DEBF
:10BEE00024E1C6EB92F4175110610675577C575840
:10BEF00066756676576466761792B97CC4000656F6
:10BF00000676577C57586675667657646676B97CB0
:10BF1000C80058C11800588108002C102800E1F012
:10BF20003C101400D9C104000CC0D8370CD010004C
:10BF3000B1B130ECF20FB8BE0800820E062B0B5BDD
:10BF400002004B3100000632062B0B71050038EE63
:10BF50000C00C4E092F1B4D124C492EC58C10400A6
:10BF600030B12C101400E1F098709B303414B1F112
:10BF7000920B147826721377CC70F600C2039920C6
:10BF8000B430AB79050030F12414E1F03C101C0012
:10BF9000D9C10C00B9B1080018E2010006D20CB0FA
:10BFA0001838C4E0821234E113EE2F7E0B0010C764
:10BFB000063D062CAB110300C42192F4062D063C6D
:10BFC00099ED01000B71050057E10C70702E26E70A
:10BFD00030EE38D0A000C4E90212062E043ACB8617
:10BFE0000F00043AB121062E8B960F00B9210400F0
:10BFF0000C305409062DEBC40F00F207062D0C304F
:10C000007409B1E1EBC40F0058C10C0038B108004D
:10C010002C101C00E1F000003C101C00D9C10C00E9
:10C02000B9B1080018E2010006D20CB0183824E1BA
:10C030001870A53013EEC67EC2102F7E0B0010C7FD
:10C04000063D062CAB110300C42192F2062D063CDE
:10C0500099ED01000B71050057E10C70702E26E779
:10C0600030EE38D0A000C4E90212062E043ACB8686
:10C070000F00043AB121062E8B960F00B92104005F
:10C080000C309009062DEBC40F00F207062D0C3082
:10C09000B009B1E1EBC40F0058C10C0038B1080081
:10C0A0002C101C00E1F000003418C1E117E1183237
:10C0B000030017227637764706E2343134410C20EC
:10C0C0001800262EF73FF74F0BD30200C42192052C
:10C0D000062E6B810500F206C4229204062E0B7D0B
:10C0E000050040E12418E1F03C101400D9C104001F
:10C0F0000CC0D8370CD01000B1B130ECF220B8BE73
:10C100000800821F062B6B140300062B6B1603001E
:10C11000186B0200187B0300062B2676E770997BCC
:10C1200001000B7D0500062B0B5B02004B3100006C
:10C130000632062B0B71050038EE0C00C4E092E0CD
:10C14000B4D124C492DB58C1040030B12C101400C7
:10C15000E1F00000107234141367CC601C00B1F1E0
:10C16000C2030C701C009970A53013770C6018384E
:10C170002471F204176191562461B471242192FB59
:10C18000EB87050030F12414E1F000003C101000B2
:10C19000D1C106E306D44B310000B372323A5C20C1
:10C1A0007F00C427C208C42FC208CC201700D207C2
:10C1B0000427F2060421F2040423F202042FC4D05F
:10C1C0000870010057282C70460166278232ACD0D7
:10C1D000D803822F187D0400C471920618707B3E2C
:10C1E000C47192026427187D0100C471920718700F
:10C1F000813EC47192036C200004187D0500C47157
:10C20000921818707D3EC47192146C200008F211CF
:10C21000C423D208C4E00820010092092C20400168
:10C22000F208082001002C204201F2032C204101D9
:10C2300050C12C101000E1F0341404400451B1F14D
:10C240000B8D050030F12414E1F00000087000307F
:10C2500034182C70889AC1E106E230271322B362A9
:10C26000221A0662D4688210F21630676464B167DD
:10C27000AB2C0000063E6B920500087000302C705D
:10C28000A09AB127F20830671455C4E05665B1672B
:10C2900092EDF2EF40E12418E1F000003414045074
:10C2A000B1F10B8D050030F12414E1F03C102800B1
:10C2B000D9C118002B390000087000302C70049888
:10C2C0003067085002006C600040B167306738305A
:10C2D000A0006665B16730676C6080000C20CC09F7
:10C2E000B1670BC30F0018701C4306ED0CE01C4334
:10C2F000B171187E0100B7D1187E02003820A0006D
:10C30000B7D2187E0300063C0C30E001B7D3187E8C
:10C310000400B7D4187E0500B7D5EBC40F00187021
:10C3200034303820A000B17118703530063C0C3024
:10C33000E001B7D118703630B7D218703730B7D3A4
:10C3400018703830B7D418703930B7D5EBC40F0037
:10C350000C203430063E6BAE0100C42092151860EC
:10C36000343018703530576466671870363018509E
:10C37000373057746675185038305774667557746F
:10C3800018503930F21418601C43187E01005764AD
:10C390006667187E0200185E030057746675185EA3
:10C3A000040057746675185E05005774667508506A
:10C3B00000302C500C98B165086000302C6010984B
:10C3C000B176EBAF010018504F43087000302C706D
:10C3D0000498306714435664B16730671445C452FB
:10C3E0005664B167920730676462B167306764640E
:10C3F000B167087000302C7020980464B167087031
:10C4000000302C7004983067085000026665B167F0
:10C410003067085000046665B167306708500080D7
:10C420006665B1671870CA00C47192030B500000B2
:10C43000087000302C700498306708D000306C60B1
:10C440000004B16730676468B16718608F30C461F9
:10C45000920F3067085000016665B1672CD0989E36
:10C460000461B16D3067085000086665F2113067ED
:10C470000850FFFE2C50FFFF5665B1672CD0989EE8
:10C48000B10D0850FFF730672C50FFFF5665B167BC
:10C4900018709B30C471920418E0F32EF204CB297B
:10C4A000000006E2062E4B310000087000302C70B0
:10C4B0002C98B1270430062E6B92050008700030CE
:10C4C0002C703098B1271870B73008D00030C47184
:10C4D0009213EBFB04006BF8040006E257E46BF8E0
:10C4E000040066E257E46BF8040066E257E46BF878
:10C4F0000400662EF2140C700099267D0462B16768
:10C500000C60543318766C001866680057726676B3
:10C510000C601099266DB1766BF804002CD01C9835
:10C52000B12DCB4B00006B4C000008700030086050
:10C5300003002C7080982C60FFF6B1670870003003
:10C540002C708498B107B8601C3F8205087000A069
:10C550002667F2020460087000302C708898B1677A
:10C56000B860283F8205087000A02667F2020460C8
:10C57000087000302C70B498B167087000302C70CF
:10C5800090980C603C06B167087000302C70B89829
:10C59000046FB167087000302C70B09830570CE011
:10C5A0001C431C400004286E3C015654B1573057C0
:10C5B0005C60FF036665B167087000302C70BC9842
:10C5C00030671C5000015665B16730676C60100021
:10C5D000B167087000302C70C0980C603C06B167E1
:10C5E000087000302C70009A1462B167286E420007
:10C5F000087000302C700C9AB16708700030186E0B
:10C6000044002C70109AB1670B420000286E320172
:10C61000282E3601087000302C70849AB167EB43E5
:10C620000000282E3601CB44000018E0F42EB37E23
:10C6300032030CE01800062E4B3100000870003069
:10C640002C70889A6C200014B1270430062E6B924F
:10C650000500087000302C70A09AB12708700030D7
:10C660002C704C98306708E0003064682CE0A49A85
:10C67000B1670CD04C42B10E182D1A000B460000C9
:10C68000306E187099301C5019005665B16ED77114
:10C69000306E5C7018006676B17E307E6474B17E58
:10C6A000187D1B00C47192081870C400C4719204F4
:10C6B0002B480000F203CB4800001870C500C4747A
:10C6C0009204EB460000F2038B4700001870933091
:10C6D000C47192036B490000087000302C70A49A5A
:10C6E00030671C5001405665B16730676C60008050
:10C6F000B167086000303876A89A0C50A89AD471B7
:10C70000265692FA0471B175087000302C70049BA3
:10C710000C600A10B167087000302C70009B0C6030
:10C720001205B16718706A3EC4719AC700000B4ABF
:10C7300000001870CC000C609400C47182030C607F
:10C740004001087000302C70089BB1673860B0332E
:10C750000870003057652C700C9BB1670870003072
:10C760002C70149B0C6064A0B167087000302C70B2
:10C77000189B0C605000B1670C701C4318573501B2
:10C78000086000302C60809BB1560860003018575C
:10C7900034012C60849BB156386738010870003032
:10C7A0002C704099B167087000302C70849D0C602B
:10C7B000FF7FB167087000302C70249EB1070870AD
:10C7C00000302C70289E0C603403B1670870003074
:10C7D0002C702C9E0C60B40BB167087000302C706C
:10C7E000309E0C60281EB167087000302C70409E8F
:10C7F000B107087000302C70349E30670850FEFF7F
:10C800006C600001B16730672C50FF015665B1675D
:10C81000306714526C60003CB167087000302C70B7
:10C82000489E0C602800B167087000300860201432
:10C830002C704C9E2C600020B1670870003008609E
:10C8400074002C70509E2C602674B1670870003004
:10C8500008601B222C70549E2C60CF6FB16708704B
:10C8600000300860070F2C70589E2C600103B167E0
:10C87000087000302C70009D30675665B1673067D6
:10C8800014555665B167087000302C700C9D0C6013
:10C890002000B16718705842086000305473577414
:10C8A0002C60189DB1760B8200006BF5040058C116
:10C8B00018002C102800E1F0AB4A0000FA3BFFFF03
:10C8C0003C105800D9C14800D981380018731900AC
:10C8D00018631800577466764377235706E20625D7
:10C8E00006D30684B7D7B7512B0E0300C4208A861F
:10C8F000020038210400AB440500C4208A810200F4
:10C9000037D1DC701000187EC000820AC473920B0D
:10C9100018201D446B740000992EC000F204C473EB
:10C920009A710200186D1A003820A000A96E0E003E
:10C93000187D1B0057746676A97E0E000C30E00946
:10C94000B171EBC40F00287E0E00C47AC204046AE1
:10C95000A96E0E00107D5C70FC00CC702000920F60
:10C960000C201C00262D0C301C436BAE0100C42093
:10C970008A4B02000C702200B7D2F2040C501C004B
:10C98000B752187E0A00C47392070C602E00266E00
:10C990001066B793F2030470B7D31454265838A125
:10C9A0000800B759F20618770100247226A723AAB7
:10C9B0003799C6A632072F7A0D001067CC60320077
:10C9C00092F30C702200267E38C10800049204B055
:10C9D000B7DAFAD800002F7C0D009067921818473C
:10C9E00001000C202E43B71B8B9A0F00371BC64249
:10C9F0009A0D02000422262C262D0C302E438BA3E8
:10CA00000F00C4208AB60000FA030200C4619AB382
:10CA1000000018B701000452C4B0265C23558AFAFE
:10CA20000100047199BE2E00265D066E267BF2077A
:10CA3000104524515C407F0099462100B471246167
:10CA400092F8C6A8B20838212800063D064AABF580
:10CA50000200F2020420187E2E0026B2262713229E
:10CA600013BBB9211000992E2E0037D4C4B03471F5
:10CA70000451997E0100064E0460265B92390451F0
:10CA8000F2370C7022002674107704312636B7D89E
:10CA9000C63B5C707F00B7D51376B7D6266E3F7362
:10CAA0000B002C60230006F32471D203C4B0921152
:10CAB0000471F20F102637555C207F00C652020623
:10CAC0001322135FB9211400B75624F12461F20236
:10CAD000B75DB47192F037D6375D267E18672200B5
:10CAE0009964220037982441996722000663B45163
:10CAF00092C937D4C47C9213187E270006675C6005
:10CB00007F00CC601600920B185E2600186E250080
:10CB1000995E2700996E2600997E25000C70F02EF4
:10CB2000185701000471C4500460267592200471E6
:10CB3000F21E1326B79BB7DC8B260000C4B004415D
:10CB4000063E264B379B37DC920B0441F209185303
:10CB50002200243176525C507F00C4508207B441D9
:10CB600092F70CC01200FA5F01002461B47192E2E6
:10CB7000349113992F7C0D0018770100247226C779
:10CB800023CC37D9C6C72A28FFFFC4909A46010094
:10CB9000062D06384BBE030086C29A450100187068
:10CBA0008F30C471920B38310800062D0648065E9E
:10CBB0002BA5020086229A330100A87E0C00920B5E
:10CBC000042A262D8B020300C420A92E0C008A29DA
:10CBD0000100912E286E0C001C7000406676A97E24
:10CBE0000C002F7B0E00182721005C207F006B2F8C
:10CBF0000000992E040037D1186E0A00DC70000482
:10CC0000921DC4639205187E0700C4719239990E73
:10CC1000070018709A300452247199709A30995014
:10CC20006A3EAB4A00001870B5300C3022005771D4
:10CC300038271430EB4A0500F223C463921E987E15
:10CC40000700921B18709A3034711377C470997072
:10CC50009A3092131870CB00C471920F04619960DE
:10CC60006A3E0B4A00001870B5300C302200577134
:10CC700038271430EB4A05000471997E0700C4B4CC
:10CC8000186E0A00D213C46392043753C454C226E8
:10CC90001870A93024719970A9301870C700C47138
:10CCA000921D04629960C500F215C463921737D3D0
:10CCB000C474D2141870A93034711377C470997089
:10CCC000A930920C1870C700C47192080452995090
:10CCD000C5000B4200000471F20204703791DC6061
:10CCE0002000186E0A009214C4639205186E0500A5
:10CCF000C4619225990E05001870BE30042124717C
:10CD00009970BE309900C3000B930500F21AC463FA
:10CD10009213986E050092101860BE30346113664D
:10CD2000C4609960BE309208046104209960C30019
:10CD30000B93050004710451995E0500C4719203C0
:10CD4000CB5905001870B730C4719206062E063D07
:10CD50000648CB790200B8611C0032050471997E47
:10CD60004C03F203990E4C031870B730102EC471A7
:10CD7000920D3752063D06484B5303000C60C046E7
:10CD8000387628002471B97628000C501000062E41
:10CD9000990E0800990E0900A90E1000A90E1200A4
:10CDA000B90E3000B90E3400A90E3800A95E3A0061
:10CDB000EB5802004B3100000632062E0B710500C5
:10CDC000062E6B160300062E6B140300186E02006D
:10CDD000187E0300062E2676E770997E01000B7DF3
:10CDE00005000461A90E1800A90E1A00A90E1C0066
:10CDF000A90E1E00A96E2000F21604CAF21404CA7D
:10CE0000F21204C1F21004CBF20E04C1F20C04C100
:10CE1000F20A0CC01200F20704C1F20506C2F203C6
:10CE20000CC01100062C58C14800588138002C1045
:10CE30005800E1F018709430C471824E046199601A
:10CE4000943006760C701838990018380461996788
:10CE50000100046299670200046B996703001C607B
:10CE6000800099670400046F99670500046399675F
:10CE70000600046A996707001C607F009967080034
:10CE8000046E996709001C607E0099670A000469B6
:10CE900099670B001C607D0099670C00046D996711
:10CEA0000D001C607C0099670E00046899670F00F4
:10CEB0001C607B0099671000046C996711001C606E
:10CEC0007A00996712001C607900996713000C7052
:10CED00014009970A530E1F0C4203414B1F1820B34
:10CEE000087000302C70481EB07722070421EB1523
:10CEF0000100F203EB15010030F12414E1F0000011
:10CF00003418C1E108E00060062E04300840020039
:10CF10006B100200B9E0D42F0C70C8340468F2071B
:10CF2000A107A9070200B90704002478B46192F9A7
:10CF30000C707C4BB970D82F0C70B83E046CF207A3
:10CF4000A107A9070200B90704002478B46192F987
:10CF500040E12418E1F000003C102800D9C118007D
:10CF600006E306D2D98108006B0F0000C4D0820707
:10CF70000CB0CC2B04F70C70C834F2060CB0A02B0C
:10CF800004FB0C70B83EC4F004213840D42F385054
:10CF9000D82F04300CA07CCB089002601484262F7C
:10CFA000925E0421F25C206BC6E6D256B8C704003C
:10CFB0008206B940D42FB950D82FF232C4D024649D
:10CFC000820C266406C6D4C3820324645668C669EC
:10CFD000D20A06C40646F2082665C66AD20406C509
:10CFE0000656F20214C11461C6C692130461266388
:10CFF000C66FA2323820A0000C30FC09B940D42FF3
:10D00000B950D82FB1E1B9D10400EBC40F00F22D13
:10D01000B940D42FB950D82FB13CB90C0400386CAA
:10D02000040078570200B967040020672461436652
:10D03000C656A1673203A9670200307C6C700001FC
:10D04000B17C24C4EB100000062C0430064E6B109B
:10D050000200062CF20D2431247824B2B42192A4CB
:10D06000B940D42FB950D82FEB100000042058C17C
:10D070001800588108002C102800E1F03C10240012
:10D08000D941080001610170C121C9611C00B9F1D9
:10D0900018006B0F00000420043C6BFB0500862287
:10D0A000820904719970A030B10204312424EB1973
:10D0B0000200087000302C707810306714535665E9
:10D0C000B167EB10000048611C0038F118004021E6
:10D0D00011161107584108002C10240061000000AF
:10D0E0003C103000D941080001700161C96128007D
:10D0F00008700040D9C118002C700002C12138E727
:10D1000014006B0F0000387068300CC0243226E722
:10D11000B9E0683038E0283238DE0400F2243CE020
:10D120002C00386E080038706830C667B2190420C9
:10D130000C3014006BFB05008622820B307EB1E2BE
:10D14000B7E1387E04000430B7E2242CEB1902006A
:10D15000387E2C00386E3000B176B967040006EDD9
:10D1600038DD0400C6EC92DC087000402C70000230
:10D17000B9070800EB100000486128004021111693
:10D18000110758C11800584108002C1030006100E8
:10D190003C101000D1C106E2AB4D0000C4E106C254
:10D1A0008208087000302C70989D30D713DDF20291
:10D1B00004D104200C3010006BFB05008622920580
:10D1C0000471997EAC2FF225087000302C708C9879
:10D1D00030770C601C43B9768C01087000302C70DD
:10D1E000949830772377B9767401B9C2040099D244
:10D1F000020099E20100187EAC2FC4719205917271
:10D20000990EAC2FF202910224280433EB1902008C
:10D2100050C12C101000E1F03418C1E1042006E3E5
:10D220000C3010006BFB05008622820A0C70510046
:10D23000B9E20400A17204342428EB19020040E191
:10D240002418E1F03418C1E1042006E30C3010008A
:10D250006BFB0500862292060C20E2002B56020092
:10D26000F20C0C704100B902040099E20200A172B4
:10D2700004342428EB19020040E12418E1F00000F6
:10D28000341404200C301000B1F16BFB0500862231
:10D2900092060C20E2002B560200F20A0C7061008C
:10D2A000B9020400A17204342428EB19020030F101
:10D2B0002414E1F03C101000D1C106E306D20C307A
:10D2C000100004206BFB0500862292060C20E20071
:10D2D0002B560200F20EC4E0B9D204000C704600D6
:10D2E00092030C704500A17204342428EB1902004B
:10D2F00050C12C101000E1F01870D23F3C101C00FF
:10D30000C471D9C10C00B9B1080006E206D306B455
:10D3100006C59270147126731377C471D26D0624FA
:10D32000B101A90104002B7F0000C4E08267B87E30
:10D3300030038266CC20180082030C201C00C4D26B
:10D3400026B204340422107B2621263B8205186B6A
:10D3500002009161F2049171187B0100044497D19D
:10D360002B9E0F001795CC60FF00921617D4C6763F
:10D3700092131793C667921017D2C676920D179123
:10D38000C667920A1071CC70F0009206382E3003F6
:10D3900004304B160600062C06318B070400C4210E
:10D3A0008231C4D20C40D03F387E300392121867CD
:10D3B000F40104202F560600265657513F660500FB
:10D3C00057612664385610012451B9561001F21BDA
:10D3D0001877F40104202F570700265757513F773D
:10D3E000050057712674385718012451B957180190
:10D3F000F20A0421F2080421F2060420F2040420B7
:10D40000F202042158C10C0038B108002C101C0095
:10D41000E1F00000C4403C101000D1C106E306D288
:10D420000C30940082030C300C0104216BFB0500CE
:10D430008622823638726C000860FFFFC4D15676AF
:10D44000B9726C00B9021800B902680030520C7051
:10D450001000820204706C70200054EF0860FF001E
:10D46000667E2C6000FF5665577C6676B172086058
:10D47000FF0F37E32C60FFFF5676086000306676BA
:10D48000B7E31474B7E50C708C002672C470820583
:10D49000086000A02676F2020470B9727C0050C1C8
:10D4A0002C101000E1F000003C101C00D9C10C0051
:10D4B000C9A1040006A30C30880406C20CD0501485
:10D4C0000424B1D1CBF9010004200C3010006BFB17
:10D4D000050086E2821A062A6BFA0200063A06B2B4
:10D4E0000446062E2B9E0F000C70D83757B126B776
:10D4F000307BB97E0C00B9CE0800B1EB04240C30AF
:10D500009404B1D1CBF9010058C10C0048A104002A
:10D510002C101C00E1F00000341406320421B1F19B
:10D520006BFB050030F12414E1F000003C1010000A
:10D53000D1C106E20C20100006D306C46B290600F8
:10D5400086228230B870D02FB102B9D20800B9C299
:10D550000C00B9E204009204B920D02FF2233867FE
:10D560000400C66EC2123FEE0600B9E70400B172B5
:10D57000B920D02FF21738460400C645D20E0676E1
:10D58000F204B162B127F20E3867040037613656F3
:10D59000B067B76192F1F2F63F550400B956040046
:10D5A000F2F150C12C101000E1F00000B870C42F4F
:10D5B0003414B1F19213B870282F9204B870742FFC
:10D5C000820D0830018004710C20FA002C30EC37F9
:10D5D0000440B970C42F0B2A060030F12414E1F086
:10D5E0003C101000D1C19872180006E206D39231A7
:10D5F000C44092052BF500008642822D0C50902BE2
:10D60000046430753077F20F28371A00C634920957
:10D61000B0278223C4D08223B03D8223C623822335
:10D6200038770C00C47092F1B461245492EBC4D0EA
:10D630008204B07D8202B17E38705C2FA94E1A0040
:10D64000B97E0C00B9E05C2F0B2E06000420F20C12
:10D650001426F20A1422F2081428F2061428F204FE
:10D660001428F202142850C12C101000E1F0000020
:10D6700034180C202000C1E16B29060086E28209E3
:10D6800004300C402000AB9D0F001471997E0A00FD
:10D69000062E40E12418E1F03C101400D9C104002A
:10D6A00086D306E292083830A0000C20180A0BC37B
:10D6B0000F00F244C4208210086000A0266D08709C
:10D6C0000200C667C2193820A0000C30300AB1D160
:10D6D000EBC40F00F2330C707C4BC6D7A2050C7064
:10D6E0007CCBC6D7C2093820A0000C30540AB1D177
:10D6F000EBC40F00F2236B0F000034D4306D1356CF
:10D70000776493668216B4619214C4E00645D741EB
:10D7100082040C70C834F2030C70B83E267438478B
:10D720000400B94D04002047B9D704003441A14793
:10D7300057646665B16DEB10000058C104002C10F1
:10D740001400E1F03418C1E106E20B330000863228
:10D75000820404216B350600063E04216B35060069
:10D7600040E12418E1F000003C101000D1C106E2B5
:10D7700006D3F20DC4E034D113DD820B062EAB3399
:10D78000000006C2062ECB3A060006ECC4D092F387
:10D79000062E50C12C101000E1F000003C101000CB
:10D7A000D1C106E20CD02000187E3000C47192096D
:10D7B000382E3400183E3800EB3B0600990E30003E
:10D7C000B4D12CE0140092F150C12C101000E1F003
:10D7D0003C105800D9C1480006E306C404300C4090
:10D7E000400006D20621C9A14000AB9D0F00187E63
:10D7F000100099C1010099711400287E0A0038BEFA
:10D800000C00A7D3387D2800B9B10C00B7D204733F
:10D810009171387E0400062BB7D4187E08000CC026
:10D82000150097D3107B26C15C70FC0099713900FC
:10D830002B17000099213A00187B0100062B547128
:10D84000063C99713B000CA01B004B4A010038219B
:10D850000C0026A1063A0B4B01000CB0210026B1AA
:10D8600038210C00063BCB4B010098613B0018713E
:10D870003A009213C4709208B9A12800B9C12C00D3
:10D88000B9B13000F214C4719212B9B12800B9C113
:10D890002C00B9A13000F20BC4619209C470920748
:10D8A000B9A12800B9B12C00B9C130000C701B001F
:10D8B0002671B7DD1871150038310C0018211400DD
:10D8C0000446045454712641265199713C006B88DA
:10D8D0000000183114009921020037133821080084
:10D8E0000C50B002265D6B180600C4219218382136
:10D8F0000C00283104002B74040006270C201C3C6B
:10D9000018701C3C06312F670700266757613F7768
:10D9100006005771267238771000F170382E040017
:10D92000183E0800EB3B060058C1480048A14000E3
:10D930002C105800E1F000003C105000D9C140000C
:10D9400006C206D306E404200C304001D981300021
:10D950006BFB05008622B92108008A60010004697A
:10D96000266D0676DC603F00065DD7517773820234
:10D97000247106475743C6D43F6D0400063D246119
:10D98000D203C44092070461F2052F230C00243116
:10D990009102B46192FB26DC1C608000916D2F64C3
:10D9A0000C0014412646915406351442264677341D
:10D9B0009134063514432646773891343464775CC5
:10D9C000915637520461C4703C5040002667B9C17B
:10D9D0000C0008D0D2C308C0321008B0BA9808A012
:10D9E000CDEF08904567B757B7912CD0F0E12CC028
:10D9F00076542CB0FEDC2CA089AB2C9001239AA38A
:10DA000000000471B7D1FA9F0000C4CFD217107D77
:10DA1000577CB97E4000186D010057686667B96E83
:10DA20004000187D020057746676B97E4000186D7C
:10DA300003006667B96E4000F212386E3400387E1B
:10DA40002000303E7676386E0800042176767637F0
:10DA5000B71B6B130100371BB92E4000B48124C1E2
:10DA600024D424E492D337D230610C50500006EB1A
:10DA700006DAB9B12000B9A12400B715068904C09F
:10DA8000B75406B706A6F207B9E11400068A06EDF8
:10DA900006A506D20425063AB71B6B130100CCC0BD
:10DAA0001300371BD20B15780668566D567E7676B6
:10DAB0000860825A2C609979F220CCC02700D209E4
:10DAC0000678767D0860D96E767E2C60A1EBF21523
:10DAD000CCC03B00D209067D767E066E5678566D28
:10DAE0007676FA9200000678767D767EFA8D0000D2
:10DAF00008601B8F2C60DCBC375506382625305B50
:10DB0000B71B2652265726560C201E00B75A6B13F9
:10DB10000100379424C1B46124B4371BB794375A39
:10DB200092B43071066A2675375338B1200038A197
:10DB300024002C504000B171269626A226BD264E08
:10DB4000B753F208B191064D069A06AB06BCB9E18F
:10DB500018003791B461B791924E06CB06BA06A968
:10DB6000309138E1180006797774997E02000679C1
:10DB70007778997E0100067A7774997E0600067A96
:10DB80007778997E0500067B7774997E0A00067B7C
:10DB90007778997E0900067C7774997E0E00067C62
:10DBA0007778997E0D0006747774997E120006D4FA
:10DBB0000674999E030099AE070099BE0B0099CE9A
:10DBC0000F00779C77AC77BC77CC777877DC919E29
:10DBD00099AE040099BE080099CE0C00994E13002E
:10DBE000997E110099DE10003831080004206B3551
:10DBF0000600F21438E11C0038D10C0004C00C807F
:10DC00005000FA04FFFFCCC03B00CA73FFFF08605E
:10DC100062CA2C60D6C1FA71FFFF58C1400058811A
:10DC200030002C105000E1F03414B1F13833100002
:10DC300004216B35060030F12414E1F0CC303C06B1
:10DC40003C101000D1C106E206D306C4C20DC44088
:10DC500082060420063E6B350600F2240421063EAF
:10DC60006B350600F21F04200C3010006BFB050022
:10DC70008672920CC4C08205063E6B350600F21215
:10DC80000421063E6B350600F20D042826270432D7
:10DC9000B9E70400A9D70200990701009107EB1921
:10DCA000020050C12C101000E1F000003C101000E8
:10DCB000D1C1067306E30430F20528670A00307705
:10DCC0002636C47092FB04212C3022006BFB050029
:10DCD00004D006C2F20F0C202200262D383E04008C
:10DCE000284E0A00262C8B980100287E0A0030EE70
:10DCF00026D7C4E092F1062C063D04408B62060054
:10DD000050C104202C101000E1F000003C10100065
:10DD1000D1C106E306D23830A0000C20780A0BC32C
:10DD20000F00062D063E04408B62060050C1042001
:10DD30002C101000E1F000003C101000D1C128E2CE
:10DD40000C0006D206C3063E5C301F0006735771F6
:10DD5000573226372F730D009867300082172867D7
:10DD60003200C66E92132C303000062D263D064C34
:10DD7000990730002B3F0600287D120024E1347102
:10DD8000A97D12005CE0FF0FF2DF062E50C12C10BF
:10DD90001000E1F03C101800D9C10800C1A106D262
:10DDA00006A306B428E20C0004C0F224063E5C3050
:10DDB0001F0006735771573226372F730D0098676F
:10DDC0003000821528673200C66E92112C30300068
:10DDD000062D263D064A990730002B3F0600287D78
:10DDE000120024C1347113CCA97D120024E15CE03F
:10DDF000FF0FC6EB92DC062C58C1080040A12C1086
:10DE00001800E1F03C101000D1C130D20672B02DE4
:10DE1000821C98621C008219A8621200821628E2F5
:10DE200010001837040024E15CE0FF0F064E4B6D34
:10DE30000600307D28670800A9E70C00346126E65B
:10DE40005CE0FF0FA9E70E0050C12C101000E1F0BC
:10DE50003C101000D1C1376237A3C4508238187209
:10DE60003900CC708400923318D611000C70D600A3
:10DE700077D2267D57712675B0E71846120018C66E
:10DE800013008225187E1C00C471922106747772DB
:10DE900057C266C7282E0C00063C2B710000C42117
:10DEA0009216063D064C062E4B6D0600062E063DCC
:10DEB000A9CE0C006B6A0600287E0800A92E0C0073
:10DEC000347126275C20FF0FA92E0E0050C12C10A4
:10DED0001000E1F03C102000D9C11000D18108C031
:10DEE000FF5F0CE0A43604D00C9068362CC0FFFF16
:10DEF00004A526AD2F8A0A006B0F0000268A387E03
:10DF000008005781248438B704002689F21E1CA01B
:10DF1000100026A73067B83A040038770400B167CC
:10DF2000B97604008208C63CC2030421F202042030
:10DF30006B3506000420063A6B350600207E3471EE
:10DF4000A17E067B38BB0400C67892E2EB1000008D
:10DF500024D1C4D224EC92CD58C1100050812C1091
:10DF60002000E1F0C4313414B1F1067292060420AD
:10DF700006376B350600F205042106376B350600BF
:10DF800030F12414E1F000003C102000D9C1100051
:10DF900006E206D304200C300001D18106C406B588
:10DFA00006A66BFB05008632825E04700C600001E1
:10DFB000B4612F5703009175247192FB06530460DE
:10DFC00004700C4000012F260E0010F52461102271
:10DFD000C66D267F26725C70FF00A20204602F27A8
:10DFE00003001092B441919591F2245192EDC4C076
:10DFF000045104600470265C92110451F20F2471E4
:10E000005C70FF002FF70300102F26625C60FF009A
:10E010002F46030010E491EF9124B45192F1C4A073
:10E020000451265A921B0451F21924715C70FF00AE
:10E030002F270300104226645C60FF002FF60300C8
:10E04000109F9192914F102226425C40FF00264380
:10E050001024104B7642914B24B1B45192E7042026
:10E060006B35060058C1100050812C102000E1F0E3
:10E070003C102C00D9810C00B121068304200C3007
:10E080004000D9C11C00B712B75106A66BFB0500B2
:10E0900086E28AF4000004200C3040006BFB05008F
:10E0A00086D29206063E6B350600FAE80000042090
:10E0B0000C3040006BFB050086B2920A063E6B35C1
:10E0C00006000420063D6B350600FAD80000042047
:10E0D0000C3000026BFB050086C2920E063E6B35CB
:10E0E0000600063D04206B3506000420063B6B3518
:10E0F0000600FAC4000004200C30D4006BFB0500BD
:10E1000086929212063E6B350600063D04206B3562
:10E110000600063B04206B3506000420063C6B35E8
:10E120000600FAAC0000066E0C704000B471910657
:10E13000246192FDCC8040008226CC804000D20435
:10E1400004702481F21D30210638064A6B4A06000D
:10E1500004700C6014002F470A001034B4612F576C
:10E160000E009135247192F804700C604000F21694
:10E1700030512F670E002657104524719146B48107
:10E1800092F8F2F304703051B481265710352F679E
:10E190000E009136247192F8F2E82F470E001044D9
:10E1A000B4612F570D007C4036009145247192F6E2
:10E1B00004700C6040002F470D001034B4612F57DD
:10E1C0000C009135247192F8B841040037D1065CF7
:10E1D0000460247192090471F20737122646103444
:10E1E000246199353F00B471245192F8383104000C
:10E1F000062C2C304000064A6B4A060004700C6066
:10E2000040002F470E001044B4612F570B007C4094
:10E210005C009145247192F604700C6040002F4719
:10E220000B001034B4612F5709009135247192F816
:10E23000065A06690C7014001045B47199464000E6
:10E240002451246192FA064A06290C3054006B4A84
:10E2500006000420063E6B3506000420063D6B35A3
:10E2600006000420063B6B3506000420063C6B3597
:10E270000600042006396B35060058C11C00588181
:10E280000C002C102C00E1F03C1028000C70280031
:10E29000D9810800D9C11800267130970C702C0064
:10E2A0002671307706C206A304200C3024000684B1
:10E2B00006B5B791B1716BFB050086E2826C042054
:10E2C0000C3014006BFB050086D28204066C0470CF
:10E2D000F210063E6B3506000420F2621056CC5058
:10E2E0001F00C25BCC507E002461D2592471237779
:10E2F000C67AA2F5064B0638062E2B9E0F0006693D
:10E300002F7B0E00776C916706697768996701002B
:10E3100006697764045499670200265B062C063A66
:10E32000064E066D999703002B8406003021063DAA
:10E330000C4014000C9014002B9E0F0004B1269E7C
:10E34000F21D0C501400066E062C063A064D2B8466
:10E350000600062D063E0C4014002B9E0F00307167
:10E36000065E3F6E090010351047B4617643914751
:10E370002451247192F924B123BB37D1C6B7A2E24C
:10E380000420063E6B3506000420063D6B35060072
:10E390000421F2060420F2040420F202042058C1F1
:10E3A0001800588108002C102800E1F03C101C00D7
:10E3B000D9C10C00062E0C202E43B9B108008B9A4F
:10E3C0000F0018708B30C672921C18608C30187059
:10E3D0001D40C66792160C20B431063E0C302E4309
:10E3E0000C4021008BA30F00C420920B0C20743131
:10E3F0000C301E400C4040008BA30F00C420823F15
:10E400000CB074310C301E400C404000062B2B9E8B
:10E410000F000CD0B4310C302E430C402100062DDF
:10E420002B9E0F00062D8B9A0F0018C01D4013E283
:10E43000CCC0400099E08B3099C08C30D220CCE029
:10E440002000D21D0471B1710C704C31062B063CBA
:10E45000064D065E0C600010B7D1EB940600C42098
:10E46000820E0472B1710C706031062B063C064DB1
:10E47000065E0C600010B7D1EB9406000C20F53F4F
:10E480000C304C310C4020002B9E0F0058C10C006A
:10E4900038B108002C101C00E1F000001870BB30EF
:10E4A0003414C471B1F192030B9E060030F12414B0
:10E4B000E1F000003C1050000C705000D9C1400049
:10E4C000D981300026713077B9210C00B1710C7000
:10E4D000540026713077B9311000B7D10C70580054
:10E4E0002671307704200C308002B71506B5B79638
:10E4F000B7D76BFB050086C28AAA000004200C3047
:10E5000014006BFB050086D29206063C6B350600B4
:10E51000FA9E000004200C3080026BFB050086E2AE
:10E52000920A063C6B3506000420063D6B3506005A
:10E53000FA8E0000382104000C30A0002C209F002F
:10E540006B880F003061063E0471263B267B2676E1
:10E55000B9310800063E2637B93120002471066E15
:10E560000C301400C4202667263D0491B799B931B8
:10E57000280006AC04802692923F0491F23D383187
:10E5800014002F450E002635102324519124B46128
:10E5900092F73831080004509103B02130613712EE
:10E5A000246192090461F2073831180026351023DE
:10E5B00024519124B461244192F838312000064E50
:10E5C00091833799065C910638210C003831100090
:10E5D000066DB7DB2B840600379A37DB064D065AEB
:10E5E000366D1024B46191252441245192FB24817D
:10E5F0002CA01400F2040667067C06C6B4918208BB
:10E60000C4B004610450266B92C30461F2C1375157
:10E6100006C7F751C450047104602675920A04714C
:10E62000F20837572F460C001034265624619135D6
:10E63000B47192F80420063C6B3506000420063DB8
:10E640006B3506000420063E6B35060058C14000BD
:10E65000588130002C105000E1F000003C104C00BC
:10E66000D9C13C0006E2042C06C306D40635262197
:10E670000446C9A1340006B62B9E0F000CA0200052
:10E680000C201200063B064A26212B9E0F00046C2C
:10E690000C702600062E063A26610C408C0A0C509F
:10E6A0001300B9D10400B9C10800B1714BA606002E
:10E6B00058C13C0048A134002C104C00E1F000008F
:10E6C0003C1078000C707800D9C16800D9815800DE
:10E6D000267130A70C707C0006E2267106250683A1
:10E6E00006D40636044630B706C506962B980000B9
:10E6F0000632042C262104462B9E0F000639062CD8
:10E7000004468B96000006320C2012002621044697
:10E710002B9E0F00063B062A0C4020002B98000081
:10E720000CC0200006320C201800064C26212B9E1F
:10E730000F00063B064C062A8B96000006320C2082
:10E740003800064C26212B9E0F00046C0C704C00E8
:10E75000062E063C26610C40A00A0C501600B9D1CA
:10E760000400B9810800B1714BA6060058C16800C9
:10E77000588158002C107800E1F000003C10E000B7
:10E78000B921B8000C205800D9C1D000B931BC0063
:10E7900006E404300C4058002621D981C000B9613C
:10E7A000B40006B5AB9D0F0004200C3041006BFB9C
:10E7B000050086D28ACD000004200C3041006BFB9E
:10E7C000050086C29206063D6B350600FAC10000C0
:10E7D00004200C3010006BFB05008672B971B0008C
:10E7E000920A063D6B3506000420063C6B35060098
:10E7F000FAAF0000CCB04000C22904300C405800F1
:10E800000621AB9D0F00087045672C700123B7D21D
:10E810000870CDEF2C7089ABB7D30870BA982C7004
:10E82000FEDCB7D4087032102C707654063E064BCE
:10E830000621B7D50BAB03003831B0000621CBB0B1
:10E84000030038E1B0000CB0100004300C4041006F
:10E85000062D6B10020004300C404100062C6B109A
:10E860000200063E064B062D2B9E0F00062C063E90
:10E87000064B2B9E0F00066D067C0C504000104688
:10E88000B4517C4036009146104724617C405C00C6
:10E890009147247192F50CE0580026E108904567F5
:10E8A00008A0CDEF08B0BA98088032102C90012350
:10E8B0002CA089AB2CB0FEDC2C807654062E063DB5
:10E8C0000C404000B9015C00B9015800B9916000EA
:10E8D000B9A16400B9B16800B9816C000BAB030049
:10E8E0003841BC003831B800062E0BAB030038317C
:10E8F000B400062ECBB00300062E063C0C404000B0
:10E90000B9015C00B9015800B9916000B9A1640077
:10E91000B9B16800B9816C000BAB03003831B400A9
:10E920000C401000062E0BAB03003831B400062E4D
:10E93000CBB003000420063D6B3506000420063CE6
:10E940006B3506003831B00004206B35060058C125
:10E95000D0005881C0002C10E000E1F03C102800ED
:10E96000D9C1180006E206D306C4062104300C40C3
:10E970001400B9B1140006B5AB9D0F00C4B1920CE0
:10E9800014240434262E263D064C0C50100006613B
:10E990008BBC0600F20DC4B2920B14440454062C36
:10E9A0000C301000264E265D06612B8406000C20DC
:10E9B0004D00262E06310C4010002B9E0F0058C132
:10E9C000180038B114002C102800E1F0C4203C10CD
:10E9D0004000D9C13000C9A1280006E206D306C410
:10E9E00006B582350CA0510026A20C201400063A70
:10E9F0000C40100026212B9E0F00062A04300C40EC
:10EA000010006B100200C4B1920A062E063D064C9F
:10EA10000C50100006618BBC0600F20BC4B29209C8
:10EA2000062C0C301000064E065D06612B84060095
:10EA30000C301400062126310C4010008BA30F006F
:10EA4000C4200471820204701327F202042058C10A
:10EA5000300048A128002C104000E1F03C104C028E
:10EA6000D9C13C020CC0100026C1D9812C02B93199
:10EA700014020682043006B4062C0C402000AB9D24
:10EA80000F000C20300004300C40E4012621AB9D27
:10EA90000F00042004386BFB050086E28A1D01008C
:10EAA00004200C3010006BFB050086A29206063E87
:10EAB0006B350600FA11010006DC04900468064C70
:10EAC00004200C306400B9412002B96124026BFBC0
:10EAD0000500C420B12D384120023861240292186B
:10EAE000063E06D46B3506000420063A6B35060058
:10EAF000C49004E126E9920804E1F206303D0420C6
:10EB000024D46B350600B4E192FAFAE60000B46151
:10EB1000249124D492D6042AB921100206D40C20C0
:10EB200030003841140226210C301000AB7C030069
:10EB30000470046818374801B4612F570E009135EE
:10EB4000247192F9C4B0047106580460267B920DBA
:10EB50000471F20B30F31092B44126F6919F2434E5
:10EB6000242192F924612458B471826C0625063C54
:10EB70000448F2F1045004482F250E0010F2B4416D
:10EB80002F35010091F3245192F804382631065CA8
:10EB900004483025B441262D10F291F38207382124
:10EBA00028022454C652243192F50C203000064A23
:10EBB00026210631B9612402B9712002EB8F0300CE
:10EBC0003861240238712002045004482F250A00BD
:10EBD00010F2B4412F350E0091F3245192F83821F0
:10EBE0001C02065E262D04300444B92118020623B7
:10EBF00038F11802D72173F2062F18F50700B44137
:10EC0000762F992507002431345192F2063A064CAA
:10EC10000458302418F30800B451262D91F22444EE
:10EC2000243192F824D1B48192A638211402269B73
:10EC3000B421B9211402921206D606870468047022
:10EC4000F21804600C30300026310446069606782F
:10EC5000066DB9312802B94114020451C4B02659D5
:10EC60000481B9511C0204D0268B92DE0481F2DCAF
:10EC70002F470E001094B4612F570800919524710E
:10EC800092F8C4B00C90300004712488046026917E
:10EC9000267B920D0471F20B3024B451262610F21B
:10ECA000244491F3243192F924612488B4718205BB
:10ECB0000638064C0458F2F10420063E6B35060077
:10ECC0000420063A6B350600303D04206B35060003
:10ECD00024D4C6D992FA58C13C0258812C022C1077
:10ECE0004C02E1F03C101400D9C10400B1B118721B
:10ECF000810008B0FF5FC47004D106E204C02CB0EC
:10ED0000FFFF26D7921404D1F212063C062ECB5EEA
:10ED100000003F7E0200CC708B000632C207F21961
:10ED20000421F20204206B35060024C1B4D192EE16
:10ED30000870FF5F2C70FFFFC6E7C2060421063E85
:10ED40006B350600F2090420063E6B350600F2041E
:10ED5000C62BD2E7F2E858C1040030B12C101400E1
:10ED6000E1F000003C101000D1C10CD0300006E2F0
:10ED700026D2F208CBE70600387048303471B970FB
:10ED80004830062D2B120000C42092F5F209CBE783
:10ED90000600387048303471B9704830F2040CD035
:10EDA0003C0326DE062D2B120000C42092F1B90E82
:10EDB0003803990E340350C12C101000E1F000000C
:10EDC0003C101000D1C186C506E206D39203C420D0
:10EDD0008222C4D08222B07D8222062D2B12000016
:10EDE0008622821FC4C19207387024303471B970F2
:10EDF0002430F206287E10003471A97E100038708D
:10EE000048303471B9704830CBE70600B07D920BC2
:10EE10000423F20A0424F2080421F2060421F20475
:10EE20000421F202042250C12C101000E1F0000075
:10EE30003C1034000C703400D9C12400D981140076
:10EE4000267110B706A64860D800B754C9610400FF
:10EE500018C0F32E04542651B9310C0006D2063CDA
:10EE60000420069404402BD9020004310440062CEF
:10EE70008B950500063B06820440062A4B210600BE
:10EE800086E2920F062A063B04414B21060086E2E9
:10EE90009208C4D082400421063D6B350600F23B47
:10EEA000C4D0820C107D5C70FC00CC708400920693
:10EEB000187D10005476C47482030450F202045684
:10EEC00004742671062E063C04410668B1714B336A
:10EED0000300C4D0820C3793062E3C601400063D1C
:10EEE00004400C5010002366AB380300383110008A
:10EEF000062E4B590000C49082050C30D8032639E9
:10EF0000F2020430062E064B065C6B920000062EC1
:10EF1000EB5F0000062E58C12400588114002C100D
:10EF20003400E1F03C101C00D9C10C0027ED065460
:10EF3000066757627772996262019972630138427B
:10EF40003C0106E2B1310420043004612BF20600DA
:10EF500086D2823D0CC030004860D00026CD0C30F7
:10EF600050010C401400263E062CC96104002B9E63
:10EF70000F00286E1800287D2C0057686676B97D32
:10EF80002C0008600FFF307D2C60FFFF5676086074
:10EF900060006676062D063CB17DEB550000062D1F
:10EFA0000C301000EB570000062D04302B570000EA
:10EFB000043404740C601000062D26310C4010003F
:10EFC000B9C10400A7D5A7946BB30100062D58C1A1
:10EFD0000C002C101C00E1F03C1028000C702800E4
:10EFE000D9C11800D98108002671307706D3B171D4
:10EFF0000C702C0026713087047338321000917425
:10F0000091059106307106E2B107B10817E606C412
:10F01000D47106B506968269910604A0F20E187A9C
:10F020000A00C473820604216B3506000421F256DF
:10F0300004719179107A917B0C60D03F18760200B0
:10F040001059C472823D06B70CB0C833184BDC00AF
:10F05000C4418240C451921AC4D09232062AB931B6
:10F060000400AB990000C42038310400823338DA40
:10F070003003182DEE012B170400C421912C92208F
:10F0800030712CD06100B1D7F21BC4509219987026
:10F09000C8338216182614002B170400C421912CA3
:10F0A000920F182B7000C423D20BEB6600000C707B
:10F0B0003A34D722262730712C201000B127AB8795
:10F0C0000000C421921F18201D446B740000912C75
:10F0D000F21904216B350600042158C1180058812B
:10F0E00008002C102800E1F00426262EB931040077
:10F0F0004B000300C420B12806A2383104009290CE
:10F10000F2933028183E14000C401500264E8BA8B0
:10F1100000000420F2E30000341406320421B1F1AF
:10F120006B35060030F12414E1F000003C1028009B
:10F13000D9C118003830A00006D20C20B80A0BC381
:10F140000F00107D3820A000B171187D0100B7D1EB
:10F15000187D02000C30D00AB7D2187D0300B7D357
:10F16000187D0400B7D4187D0500B7D5EBC40F0097
:10F170000C202C006B29060086E28A8400000430F3
:10F180000C402C006B10020006670C60D831385020
:10F19000D83104C00C702000B16E0665736CD46168
:10F1A00092070471537C6675B970D831F204B4715A
:10F1B00024C192F43860D8313820A0000C30F80A0D
:10F1C000B161EBC40F00CCC0200082571C7040001E
:10F1D000C4C0997E0A001C6058000472996E0B002E
:10F1E000997E0C0092050461996E0D00F2060C7078
:10F1F0006400267C997E0D0057C404243CC0004066
:10F20000262E063D0446A9CE0E002B9E0F000C7044
:10F210001C00267E0C60D831B97E2000B97E1C000F
:10F22000B87628008205382610000437F1700C608B
:10F23000D831387604002471B97604000C502400CB
:10F24000387608000C40E031265EB94E2800B97EC1
:10F250002400B9570400B8762C00B956080082057E
:10F26000382610000437F1703830A0000C20180B3D
:10F270000BC30F000420F207062E6B0907001421B0
:10F28000F202142158C118002C102800E1F00000EF
:10F290003C104800D98128000693D9C138000C7071
:10F2A0006C1406C206E404240C308804B171CBF956
:10F2B00001000461B16E0C60D831B876280004B644
:10F2C00026BC8205382610000437F17038D0E431AE
:10F2D0000CA0E031F2181C802400268D0434062B8B
:10F2E000263804468BA30F00C420920B0C60D83143
:10F2F000B8762C008214382610000437F170F20F13
:10F3000038DD0400C6DA92E80C60D831B8762C00FB
:10F310008208382610000437F170F203C480920F7F
:10F3200004210C30300BCBF9010004240C30500BBD
:10F33000064B0456EB010200FAA80300287C0C00DF
:10F3400004240C30600BB171CBF90100287C0C0057
:10F35000CC7086DD8A980300C4789A8C0300187CF0
:10F36000170004240C30780BB171CBF90100187C24
:10F37000170004DECC70110026DC9A660300387C8E
:10F380000E00547F577126D7207DCC7000449A72AE
:10F390000300B10E38AC0E000C70160054AF57A12C
:10F3A000267AB7D606B736970C705C1404240C3056
:10F3B0008804B17126BCCBF90100107BC4719A6539
:10F3C0000300187BEC00186BED00577C57686676DD
:10F3D000186BEF006676186BEE005764667608606F
:10F3E00082632C606353C6769A5003000C60F00071
:10F3F000266B3C90F000B797B99120000460F211A1
:10F4000037D72676104718570100CC4035009206B2
:10F41000989702008A3A0300F2090472267526675B
:10F4200037D8C667A2EEFA3103000C200C066B2910
:10F43000060086D28A2A030004300C400C066B10AA
:10F4400002000C2022003716262D063C2B9E0F00B2
:10F4500038E1180006792CE0220026ED4B980F00C9
:10F4600001000800DE051600DE057802DE05DE0577
:10F47000DE05DE055A013860940138709801B794B2
:10F48000B7D238609C010C70041404240C3088043A
:10F49000B793B171CBF90100063B0C40F000062E8A
:10F4A0002B9E0F000C201000043A0472262E2638E2
:10F4B0000444917E2B9E0F000C6035000471996E00
:10F4C000F000997EF1000462996EF2003890E43108
:10F4D000BC90240082130C20F500043A0C70360016
:10F4E0000464262E26390444997EF300996EF400B4
:10F4F0000CB0F9002B9E0F00F2030CB0F3000422B5
:10F500002F7B0E000461262B043C91672631046496
:10F510000444262E996701002B9E0F0004282F7BA0
:10F520000E000C603300262B0C301000996706008B
:10F53000263104640444262E996707002B9E0F0091
:10F540002F7B0E000C603A0024BE043899670C0033
:10F550002F2B0E0004642631044499670D002B9E66
:10F560000F00C4900474267B82220426267E046346
:10F57000262B249A916706392F7B0E0004640444DD
:10F58000262E996705002B9E0F002F7B0E00046628
:10F5900024BC99670A002F2B0E000464063904442A
:10F5A00099670B002B9E0F000474267B26E71471CD
:10F5B000917E0C700414FA85010038709001386057
:10F5C0008C01B7D20C70181404240C308804B1716B
:10F5D000B793CBF90100063B0C40F000062E2B9EA2
:10F5E0000F000C201000043A0462262E2638044432
:10F5F000916E990E03002B9E0F000C703500997EC2
:10F60000F0000475997EF2000461996EF100389063
:10F61000E431BC90240082130C20F500043A0C6005
:10F6200036000474262E26390444996EF300997E20
:10F63000F4000CB0F9002B9E0F00F2030CB0F300A5
:10F6400004222F7B0E000461262B0438916726319B
:10F6500004640444262E996701002B9E0F000428A1
:10F660002F7B0E000C603300262B043C99670600AC
:10F67000262E046426310444996707002B9E0F0050
:10F68000C490047C267B8222267E04639167249AA0
:10F690002F7B0E0024BE0464063904442F2B0E0079
:10F6A00099670D002B9E0F0004262F7B0E00046629
:10F6B000262B99670400262E0464063904449967B2
:10F6C00005002B9E0F00047A267B26E71471917E9D
:10F6D0000C701814FAF60000386088013870840144
:10F6E000B793B7D4386080010C70281404240C3010
:10F6F0008804B9010800B795B171CBF90100047C09
:10F700000498267B2691063706290444B7D98BA393
:10F710000F00C42037D9820406290637F20F04707F
:10F7200038311C002637105317B1CC503200920AE2
:10F73000C463C20804282621243204442B9E0F00EF
:10F74000F206246226763798C676A2EB042A04389D
:10F750002628263104448BA30F00C420920304956D
:10F76000F2020496063B0C40F000062E2B9E0F0082
:10F770000C201000043804720461262E2631044443
:10F78000917E996E03002B9E0F00C4959A8600000F
:10F7900004240C30900BCBF901000C703500997EDD
:10F7A000F0000475997EF2000461996EF1003890C2
:10F7B000E431BC90240082130C20F500043A0C6064
:10F7C00036000474262E26390444996EF300997E7F
:10F7D000F4000CB0F9002B9E0F00F2030CB0F30004
:10F7E00004222F7B0E000461262B0C30140091673D
:10F7F000263104640444262E996701002B9E0F00D5
:10F8000004282F7B0E000C603300262B043C9967E4
:10F810000600263104640444262E996707002B9EB7
:10F820000F002F7B0E000C603A0024BE0C3010003D
:10F8300099670C002F2B0E0004642631044499674D
:10F840000D002B9E0F00C4900474267B8222042698
:10F85000267E0463262B249A916706392F7B0E009F
:10F8600004640444262E996705002B9E0F002F7B0D
:10F870000E00046624BC99670A002F2B0E00046456
:10F880000639044499670B002B9E0F000474267BF5
:10F8900026E71471917EF21304240C30AC0BCBF9E3
:10F8A00001000C6035000471996EF000997EF10042
:10F8B00004661471996EF200997EF3000C7028149E
:10F8C00004240C309404B171CBF9010038B0E43158
:10F8D0000CE0220026ED3CB0240004260434262E41
:10F8E000263B04462B9E0F000436263C062E04467B
:10F8F0000CC030002B9E0F0026CD04EC26EC043A01
:10F90000263B0444062E2B9E0F000C204000043A98
:10F9100026380444262D2B9E0F00233A0C702C020F
:10F920000C602C02267A2663576477746676A97D6C
:10F930003200187D38000C6040003471062CA96D2F
:10F940003600997D3800A90D3A006B05010006725A
:10F95000577477246672A97D3A0026AC0C70004378
:10F96000A17A0C70022CA97A0400A87A06000C6017
:10F970000044A96A02008250A90A0600066A184DCE
:10F98000390004500C701701F209103618260100D6
:10F9900057342632233326532462B47192F7187DEC
:10F9A0003C00183E0100577426730C602C0226643C
:10F9B00023772676186D4000183D41005764266372
:10F9C00023662676186E0200183E030057642663ED
:10F9D00023662676186D4200183D4300576426635F
:10F9E000236626762675F2045C70FFFF267606678E
:10F9F0007768C46092FA1577C4709206CC40110003
:10FA000092030C70FFFF237706675764777466676D
:10FA1000A96A0600F203A90A0600307838311800F6
:10FA200038774400062D2C302402F1700C705C14E1
:10FA300004240C309404B171CBF90100F226062D98
:10FA40006B090700F222387D100038D0E43104241D
:10FA50000C30CC0BB7D1B171CBF901003CD02400F4
:10FA60000424043A2621263D04448BA30F00C4201D
:10FA7000920A0C706C1404240C309404B171CBF90C
:10FA80000100F203B10EF2F658C138005881280087
:10FA90002C104800E1F000003418C1E10CE0D8312E
:10FAA00004300C404800062EAB9D0F000C70E03176
:10FAB000B97E0C00B97E0800AB41010024210B0A7D
:10FAC0000700087000802C7020CDB97E440040E112
:10FAD00004202418E1F000003418C1E106E2063EDB
:10FAE00004440C20842F2B9E0F000434263E044433
:10FAF0000C20782F2B9E0F0004380C20602F263E00
:10FB000004442B9E0F00B07E9205047199706C2FF7
:10FB1000F20399006C2F043004206B550700042079
:10FB2000ABA10900EB22010040E104719970AC30F7
:10FB30002418E1F038702C2F3414C672B1F1920FF2
:10FB400037A3B9602C2FF20DB8670C008206C6628D
:10FB5000920437A3B9670C0038770C00C47092F593
:10FB60006B09070030F12414E1F0000086223418FC
:10FB7000C1E1821B38E2200018722D00C4E05C70E5
:10FB8000F70099722D008211B82E040082054B5A9D
:10FB90000700B90E0400987E0C008207990E0C0035
:10FBA000990E0D00A90E1A0040E12418E1F00000A2
:10FBB0003C101000D1C19872180006E292580C2037
:10FBC0001C006B29060086D28254386E1000287EF5
:10FBD0001A00B96D10000461A97D1A00996D180012
:10FBE000187E1900997D1900187E08006472997DAD
:10FBF0000800186E0A00996D0A00187E0900997DA8
:10FC00000900306EA87E1A00B16D821F38705C2F1B
:10FC1000C67E9206387E0C00B9705C2FF214B97063
:10FC2000482FF20D38670C00C66E9208386E0C0033
:10FC3000B970482FB9670C00F2060676C47092F3CB
:10FC4000B970482FB90E0C00062E6B0907003860FA
:10FC50003C2F087000802C70A01EB97D1400B96D77
:10FC60000C00B9D03C2F0B2E0600F20404D0F20297
:10FC700004D0062D50C12C101000E1F086223C105B
:10FC80001000D1C1821804E0F202062D27E734717A
:10FC90002377C470A7E7921017ED30D2D472820494
:10FCA00037E4F170F2036B090700C4D024E113EECE
:10FCB00092EDF20204E0062E50C12C101000E1F08B
:10FCC0003C101000D1C1067206D257D15772267D62
:10FCD0000CD08C3226D706E2B02D82048B6407004C
:10FCE000B10D067E577157E226E70C708C3226E77D
:10FCF000990E120050C12C101000E1F03C102400AD
:10FD0000D9C11400D981040006E20C708C32049031
:10FD100004FA04A004B00460045A04DA042A04CAF1
:10FD2000B131C45A184712009205C44092053356A7
:10FD3000F224C4408222C4E08208303E38870400A6
:10FD4000C63892033326F256C441920FB047184783
:10FD500013008206C649A21133F60694F20EC64B72
:10FD6000A20C332606B4F209C441C2071847130097
:10FD7000C64AA20333D606A4B4C1246113662C700C
:10FD8000140092D030310673D472922FC45A920468
:10FD9000D4319204F22C13D5F20FC4DA820313DDAE
:10FDA000F208C42A820313D2F204C4FA822213DFB7
:10FDB000062DAB660700C4E0820C066D067D577207
:10FDC000576126670C708C3230EE2676B9E7040056
:10FDD000066D067D5772576126670C708C32267649
:10FDE00099071300332DF2061421F2041421F202B4
:10FDF000142158C11400588104002C102400E1F093
:10FE00003418C1E186E2820AB82E100082038B64A6
:10FE10000700B90E1000B90E140040E12418E1F0FB
:10FE20003418C1E106E2B822140082038B64070093
:10FE3000062E6B09070040E12418E1F03C10140085
:10FE4000D9C10400B1B10CE0943206B204C004DAA6
:10FE5000987E0A008207307EC67B9204062CAB6631
:10FE60000700B4D124C12CE0140092F358C104005F
:10FE700030B12C101400E1F018722D003414065724
:10FE8000D451B1F1820A5C70FE0099722D00DC70D1
:10FE9000200082038B72070030F12414E1F000008F
:10FEA0003C101000D1C10CE09E3204C004DA906E08
:10FEB0008216187E010024711377CC70EF00997EB2
:10FEC0000100D205C4619207C471C209062CAB6659
:10FED0000700F205C46392030472917EB4D124C179
:10FEE0002CE0140092E550C12C101000E1F000004D
:10FEF0003418C1E127E4C637B21A3F77030006E29F
:10FF0000F2093636286E080023332667A96E0800EA
:10FF100030EE286E0A00C636D2F5B02EA93E0A0091
:10FF2000A93E080082038B640700B10E40E124184B
:10FF3000E1F000003C101400D9C10400B1B1067218
:10FF400006E306C44B980F000000040028010E00D1
:10FF50001C00140018000CD03600F20704DEF20575
:10FF600004D0F2030CD02200067C4B980F00000056
:10FF700004000601A200D800D8000E000C201004D6
:10FF80006B29060086B2827804632F7D0B00996B83
:10FF90000C002C7013001464567624D3B97B040033
:10FFA00056D60C7000043FDD0700C6DEB10BA9EB8E
:10FFB0000800020206DE23DD0461A9DB0A0036ED3B
:10FFC000A96B0E0006DBF2220C2010046B29060040
:10FFD00086229206062B8B64070004B0F24D047350
:10FFE00097EC237ECC70FF03B10299020D00B12D76
:10FFF000A7E4C2030C7000040C6010002662B7A1D5
:020000040001F9
:1000000036E7046106D2A7E5A7A7C4E012DEF22B0B
:100010000C201300047314C4262D267E567C562C07
:1000200026276B29060086B2822726DB2CD01300F8
:1000300056DCB9DB0400A9EB0800A9EB0A00B10B00
:10004000990B0C00F2100C2010006B29060086B2F0
:100050008213B90B0400A9EB0800A9EB0A00B10B4D
:1000600099CB0C000471A97B0E00990B0D00F204D2
:1000700004B0F20204B058C10400062B30B12C10B9
:100080001400E1F0C4203C101400D9C10400B1B147
:1000900006D206E306C48AEE0000C4308AED0000F2
:1000A00004200C30340104404B7A0700C420B92EE0
:1000B00010008AE40000987E0D00920638706C00F3
:1000C0002471B9706C0037E138506C00B97E1400AF
:1000D000B15E04619167387E140099670100387E33
:1000E0001400185D260099570200387E1400990705
:1000F0000300302E38BE1400EBEE01000672777458
:10010000997B0500C4C806720460992B04007778B7
:10011000772C997B0600992B0700996B0800996B47
:100120000900996B0A00996B0B00996B0C00996B95
:100130000D00996B0E00996B0F00820BC4C48209ED
:10014000C4C39217187E0C0034741377C471D21193
:10015000187D0400997B0C00185D0500995B0D006B
:10016000186D0600996B0E00187D0700997B0F0033
:100170000450995B1000995B1100995B1200995B28
:100180001300995B1400995B1500995B1600995B4D
:100190001700995B1800995B1900995B1A00995B2D
:1001A0001B000470065D0C601000182D260023470C
:1001B000C624383E1400C20418452700F202044049
:1001C000B461263799431C002471245192EF0460D6
:1001D0000C704000385E1400B471265699052C004E
:1001E000246192F904600C708000385E1400B471D0
:1001F000265699056C00246192F9387E14000C6033
:1002000063001C507E009967EC009957ED000C606C
:1002100053000C5063009967EE009957EF000C6093
:1002200044000470A90E1800385E1400B46126570B
:100230009975F000247192F9287E1800386E140028
:100240000C50350026679956F0002471386E140062
:100250002377266704519956F0002471386E1400F4
:100260002377266799C6F0002471A97E1800042020
:10027000F206142EF2041426F202142158C10400CE
:1002800030B12C101400E1F03C101000C634D1C184
:100290000C70100006D50C5014002671265106E390
:1002A00010771055B21AD472920E18761E00DC70B8
:1002B00040009213C4508207B8766C009204B8765E
:1002C0007000820B0C30B705263E14745637C634C6
:1002D000020206342333F202063E04404B7A070042
:1002E0008622820827E5367EA17DA9E20800A9E2E0
:1002F0000A0050C12C101000E1F000003C10140066
:100300002C301400D9C10400233306E206D40421A2
:100310000440B1B14B7A070086B2825A286E1A00A7
:1003200038CB040006765774776466762377917C21
:100330007774997C0100286E1C0099DC0400067615
:100340005774776466762377997C02007774997C7A
:100350000300067D7774997C0500067D777877DC4D
:10036000997C060099DC070038DE2800062DEBEEAC
:10037000010006727774997C090006727778992CCF
:100380000800997C0A000C6050000C701000772C5B
:10039000996C0C00992C0B00997C0D00287E2E0086
:1003A000066706575764775466652366996C0E0096
:1003B0007764996C0F000460996C1000996C1100BF
:1003C000996C1200996C130026D7B9DE300058C121
:1003D0000400062B30B12C101400E1F03C101C007E
:1003E000C9A10400D9C10C0006B206E4062306A385
:1003F00006340641B1012B150700B071821DA33EE2
:10040000821D042304434B7A070086D2821906ED2D
:1004100004C0382E0400284E0A002F3C0A002B9EF0
:100420000F00287E0A00B0EE26C792F4F212062DC5
:100430008B640700F20604E0F20414E1F20214E116
:10044000062E58C10C0048A104002C101C00E1F03D
:10045000387B1000062D063BF17086E282F2F2E84E
:100460003C102000D9C11000D18106D2069304238C
:100470000C302A0004404B7A070086C2825738ECC1
:1004800004000CA0270004BE26BE26AD047004287C
:10049000997E1400063A0471262B0446997E1500B5
:1004A0002B9E0F000C202000262E04300446AB9D0E
:1004B0000F00062E0C30B80104462B9E0F000426B8
:1004C000063A262E04462B9E0F00042E0434263DA9
:1004D000262B04442B9E0F000C20260006390444D2
:1004E000262E2B9E0F000470997E0E000471997BBE
:1004F00001000478997E10000470997E1100047642
:10050000997E12000474997E13000478997E0C0081
:100510000476997E0D00387D1800062D063CF1709A
:1005200006E2062C8B640700F20214E1062E58C185
:10053000100050812C102000E1F000003C1014004D
:10054000D9C10400066406E30634576257312636E3
:100550000C708C32B1B12FB30700186B120006D2A9
:10056000C46206C4920F186B1300CC60E300C20A89
:1005700024342637ABA30700C42092040473997B6C
:100580001200067C577157C226C724CC0C402700A6
:100590000C508C32062D063E264D265CEB9A01004F
:1005A00058C1040030B12C101400E1F03414B1F142
:1005B00018722D0006320667D461920C647199722C
:1005C0002D005C703000CC70300092042434ABA35A
:1005D000070030F12414E1F03C101400D9C10400EC
:1005E000B1B130E306C206B3062E063C06D4EBECEE
:1005F0000100C4209A870000067E5C70F000CC7079
:10060000E0008A820000C4E08A810000062B0431E9
:100610008B68070086E22A810000066E067E57720C
:10062000576126670C708C32267698671200920408
:10063000046199671200066E067E5772576126673D
:100640000C708C32267618771200C4718203C4D0E5
:100650009209062C063BABA30700C4D006629203A6
:10066000F2571461064E065E574157520C708C3299
:1006700026542F45070018441200C441C20E245CC2
:100680000C402700062C063D264C265799E08A3060
:10069000EB9A010006E2F241C441923C067DF2066B
:1006A00018670C00C46192053077C47092FAF23C6E
:1006B00028370800042304404B7A070086C2822CA6
:1006C000063DABC10100C4208207062C8B640700E5
:1006D00014E1F22306CD066E067E57725761266737
:1006E0000C708C322676B02782038B640700067E5E
:1006F000577157E226E70C708C3226E7B1CE04E042
:10070000F20C14EEF20A14EEF20814EEF20606E20F
:10071000F20406E6F20214E1062E58C1040030B1DC
:100720002C101400E1F0062D6BBF0100C4D092D351
:1007300014E1F2F33C101C00D9C10C0006D206C330
:10074000062306E4043EB9B10800CBBA0100C42078
:10075000927630BE063D062BEBEC0100C42092657C
:10076000067B5C70F000CC70E00092150471917112
:100770000C705E009901010097D2187E01000651AD
:100780005C707F0097D3187E020097D4187E030018
:1007900097D5F24D387D0400386D0800767BD6760B
:1007A000820C5CB0FFFFCCB0A9FE8207B87D0C00C4
:1007B0008248043C263DF202063E18408A30066418
:1007C00006745772576126670C708C32267618674C
:1007D0001200C461C20B306338770400C66792060A
:1007E000062D063C8BAA0700F22D0C7090320440B7
:1007F000046A18570E00C451C20D30233057C62565
:1008000092091344062D063C99408A308BAA0700B2
:10081000F219B461244133442C70140092EB062D7C
:10082000064C6BAF0700F20E0C50B8010C402700CD
:10083000062D063C264DEB9A0100F2041422F2022A
:10084000142458C10C0038B108002C101C00E1F031
:100850003418C1E138E22000187E0C00C478820808
:100860000478997E0C00990E0D00A90E1A000C3028
:100870002400263E04406BAF0700187E0D00247153
:10088000997E0D000471A97E1A0040E12418E1F060
:100890003418C1E186E28209B82E040082038B6419
:1008A0000700062E6B09070040E12418E1F0000064
:1008B0000676D4713C102400D9C11400D9810400FB
:1008C00006E206D306C406B5068682030494F20245
:1008D00004900678D4728203047CF20204700C2027
:1008E0001000B1716B29060086A230719205062DA9
:1008F0008B640700F2582697998A0A00287D080021
:10090000062D36790C301400B10AB9DA0400A97A40
:100910000800CBBA0100C4208206062A2BC50700B6
:1009200004A0F241387A0400286E1A0038D7040077
:100930000676577477646676B9DA0C002377917D72
:100940007774997D0100286E1C00062B067657747B
:10095000776466762377997D02007774997D03002A
:10096000EBEE0100067277745795997D05002C9087
:10097000005006727778669C997D06000679577458
:10098000779466792377997D0C007774992D04000C
:10099000997D0D00772C0470992D0700997D120028
:1009A000997D130058C11400062A588104002C10A8
:1009B0002400E1F03C101000D1C12872680006E26A
:1009C000CC70170006C3C20A18621E001C7080009B
:1009D000667699721E001421F25B06D3F7D0D4D14B
:1009E00082030434F2020430A87E660082500420A0
:1009F00004404B7A07008632920A186E1E001C7063
:100A000080006676997E1E001421F242385E5C00FA
:100A1000062E064C066D2BC607008622920A186E1B
:100A20001E001C7080006676997E1E001421F23034
:100A3000B87E6C009205B92E6C00F2050676B067A0
:100A400092FEB127C4D0A90E6A009204067CD4712C
:100A5000820B387E5C002471B97E5C00287E6600C3
:100A60003471A97E6600D4C18207187E1E006C70A6
:100A70002000997E1E0038220400CBBE0100287E93
:100A800068002672A97E68000420F202142150C179
:100A90002C101000E1F000003414B1F1B8726C00B9
:100AA0009203F21F0676B06792FE38670C00187644
:100AB0000D0018560C005774667506577754D457B6
:100AC00092106C70000199760C00777499760D0085
:100AD00018721E006C70200099721E000420F2042F
:100AE00004314BCE070030F12414E1F03418C1E199
:100AF000F20530E22BC50700062EC42092FB40E130
:100B00002418E1F03418C1E19872180006E2821D41
:100B1000C47A821BC4718219B822740082058B6466
:100B20000700B90E7400382E6C001471A97E3400D1
:100B30000BD80700382E70000BD80700B90E6C00D8
:100B4000B90E7000A90E6A0040E12418E1F000001F
:100B500086733C105800D9C14800D9813800B75479
:100B6000B9311800A901080006E206A42852620063
:100B7000286236008A9C010018721800C47482072B
:100B8000C4778205C4728203C4739222C4A08A9F70
:100B90000100287E6600C67AB20B186E1E001C701B
:100BA00080006676997E1E001421FA8A0100287E54
:100BB0006800CC701700CA8B0100186E1E001C70F4
:100BC00080006676997E1E001421FA7A0100142DA9
:100BD000FA77010006C7B07C92FE187C0A0006670F
:100BE000D46182030454F2020450D4728203047C60
:100BF000F2020470286C080037183646364536472E
:100C0000287E6A002344C470A7D4820CC6A706DAE3
:100C1000C20206D723DD367D364DA7D42344069C79
:100C2000F20304D00490C6DAB23FC440823DC460EF
:100C3000823B3F9D0A00C6940202069437D4239952
:100C4000D471821837940458B161047104230639B1
:100C50002651066EB7D1EB94070086B28A0C0100CC
:100C600038311800382B0400263D06492B9E0F0012
:100C7000F20D0423063904414B7A070086B28AFE3E
:100C8000000037D6267DB97B0400062BCBBE0100C1
:100C90003795269D262623992322068DB9211400F7
:100CA00006D9069CF203068D04B00470B7D337D87A
:100CB0000460B799A9712800236737D4B79B547192
:100CC000B7DCB9B11C00B9C13400F26E3FCD0A00E7
:100CD000379B237CC676C20328C12800B871300038
:100CE00023CC821E37940471B161B8610C0082027A
:100CF00004703718045813770420063C2651066EFA
:100D0000B7D1EB94070086928ABC000038311800F6
:100D100038290400263D064C2B9E0F00F21C0420AF
:100D2000063C04414B7A070086B28AAB000037D6F6
:100D30000420267D04300440B97B04004B7A070070
:100D400086929206067B062738B11C00F212063BFB
:100D5000CBBF01000629CBBE010037D526272322B1
:100D6000CC201800B9211400C20838B11C00062993
:100D70008B640700FA880000385E5C000639062E96
:100D80000440265D04602BC607008692827AB86113
:100D90000C00820437D9B197F203B9910C0026DC1C
:100DA00023DDB9912400C6DAA292C48038B11C00B8
:100DB00038C13400822238DC0400F218287D080093
:100DC0002678A97D0800B07D9210287D0A00382D74
:100DD000040038311800262706482B9E0F00287D76
:100DE0000A002678A97D0A0030DDC4D092E8287C6C
:100DF00008002687A98C08002794C4B0A96E6A0051
:100E0000820D382C0400063BCBBF0100286B080084
:100E1000287C08002676A97C0800C4C0920537D338
:100E2000B97E6C00F2033793B16C387E5C00C490DD
:100E3000267AB97E5C00287E66003FAA070037D577
:100E4000A9AE6600A97E68008234B8690C008233BE
:100E500037D4D472923218760D0018560C0057749D
:100E600066756C70000899760C00777499760D00A1
:100E70000420F2260460B793F2060470B7D3F2039D
:100E800038B11C00186E1E001C708000C4B066765D
:100E9000997E1E008204062B8B640700B8610C004B
:100EA000820E06260BD807001421F20A142EF2082F
:100EB0000420F2060420F2040420F202142158C196
:100EC0004800588138002C105800E1F00675F77082
:100ED0002357C656C20206762377B7D80C7068002F
:100EE000267E2077B8CE6C00B7D59A76FEFF0480B8
:100EF00004D00490FADAFEFF3C105000D9C1400043
:100F0000D98130003761B9311400B719B754187559
:100F1000070018650600577466760667576477748D
:100F20006667236606765C70FF1F5C6000202366A0
:100F3000B7D328732400B7971C6014002667289243
:100F40000800C4603C90140006E223993203146D3B
:100F50002667E7612366B796D76123663C70130066
:100F6000B79804800CA01400B7DAFAAE000037532B
:100F700037DA37975C50FF1FC6796665B79112075D
:100F800037586C600020B791B752F203B99108004E
:100F900004220C30140004404B7A070086C28A9960
:100FA0000000382C0400383110000C4014002B9E37
:100FB0000F00387E040038DC0400267AB97E040075
:100FC000287E0A003FAA0700A9AE0A0038A108003F
:100FD000F23E287E0A00068A2367C6A6C20206875A
:100FE000A38882340C2018006B29060086B2920672
:100FF000062C8B6407001421F26D386E040006384D
:1010000004230442065BB181CBB60100863292090B
:10101000062B6B090700062C8B6407001421F25A7B
:10102000062EB9312C006BBF010038312C0008604E
:1010300000802C6034EE062CB9EB1400B96B100064
:1010400036A8CBBF0100A3AA820430EEC4A092C28E
:1010500037D137915774776466762377997D060088
:101060007774997D070037920C3014002C601400BF
:10107000236606765774776466762377997D020037
:101080007774997D0300062D0470997D0A00997D7F
:101090000B004BE50100992D0A007724992D0B00D8
:1010A00037553719387514000625063CF170062CA3
:1010B0008B64070037D337923756369626752377D9
:1010C000239906A8B7D3C4909A53FFFF0420F202D5
:1010D000142158C14000588130002C105000E1F01C
:1010E0003C1028000C702C00D9C11800D9810800D0
:1010F0002671C44030B70C702800267106D206C392
:1011000006E506A610978A9900000C301400B71166
:10111000CBBA0100C42037119AB30000387D040017
:10112000C4C099E70800999709003064579406569F
:1011300077549957110006F6065699671000775CA8
:10114000669E77F806E60C6045009957130099F7FC
:10115000120099A701009167286D080057A4068620
:1011600057847764668623880668776499670300E6
:101170000460998702009967060099670700286054
:1011800078305CE0FFFF0626065677545724662524
:1011900023220652775499270400995705002461A9
:1011A000A96078306CA045008203B06C9210186B77
:1011B000040099670C00186B050099670D00186B07
:1011C000060099670E00186B0700F20C065677545C
:1011D00099570D00065699670C007758776C995708
:1011E0000E0018370D0099670F0018670C00573470
:1011F00018570E00663618670F0057586653576C1D
:10120000666506565C50FFFF26FE26F57768266F5A
:101210002686262826A2269A065977585C90FFFF34
:1012200026950669776826691566236699670A0018
:10123000776499670B00F212376106411875110047
:10124000186510005774667618651200576866674F
:1012500018751300577C6676B171A87B2400820A4A
:10126000286D0800C667C206062D063B6BF807000E
:10127000F208387B1400062B063DF170F2021422AE
:1012800058C11800588108002C102800E1F0000017
:101290003C1028000C702800D9C11800267106E205
:1012A000062410D7B9310800B713B754B7958BE9A6
:1012B00001008622383108003713375437958208E9
:1012C000B9210400062EB1D1AB070800F2021424A4
:1012D00058C118002C102800E1F000003C10280034
:1012E000D981080006B2069306A404210C3024001C
:1012F0000440D9C118004B7A070086E2824438DEE8
:101300000400047030CB997D0400997D0500997D1F
:101310000600997D0700919D99AD0100382E0400CB
:10132000303B0C401C0024282B9E0F000470997D3C
:101330000200997D0300283E0A00062D4BE50100BE
:10134000992D02007724992D0300187C0D00186C4C
:101350000C0057746676186C0E0004445768666774
:10136000187C0F00062E577C6676B7D104300471C6
:1013700026410C50FF000460B1712B150800062EA9
:101380008B64070058C11800588108002C102800F1
:10139000E1F00000341406432424043BB1F18B1720
:1013A000080030F12414E1F03C101800D9C1080005
:1013B000C1A138D2040006E2382D040006C317E5A7
:1013C00017A45774E676921F17E110625774667679
:1013D00017A204385768666717E30C401400577C5F
:1013E0006676263EB97E04002B9E0F00062D043142
:1013F0004B1D0800062DCBBE010006B2062D8B64E6
:101400000700F20204B038DE0400F219385D04006F
:10141000062D18650100107557646667187502007F
:1014200018A503005778667657AC66A7CBBE0100B7
:1014300026B223BB062D06DA8B640700C4D092E7E0
:101440003870C82FC67E9205307EB970C82FF2035F
:10145000307EB17C062E6B0907002870763058C1AB
:101460000800367B062BA970763040A12C1018009E
:10147000E1F000003C101400D9C10400B1B106E253
:1014800006B304D03870C82F04C004300420F23DE5
:10149000186E0D00185E0C0057646665185E0E002D
:1014A00057586656186E0F00576C6665385714000B
:1014B000C656921D186E1100185E100057646665BE
:1014C000185E120057586656186E1300576C666502
:1014D00038571800C656920B186E0500184E0400B7
:1014E000576428570C006664C656820BC42024C17A
:1014F000820718571F0018621F00C656D20206271F
:10150000B067820206370676C47092C3C420820494
:10151000EB1D080026D2C6DB3203C4C112B4062D6F
:1015200058C1040030B12C101400E1F0341406430B
:1015300024240433B1F18B17080030F12414E1F0B6
:101540003C102800D9C11800D981080038A2040035
:101550000683103A0472543F27A426735771C66756
:1015600006D2220757311633CBBA0100C4208206B7
:10157000062D8B640700FACF00003870402F389D8D
:10158000040006270638B7D1EBEC0100186901000A
:1015900010595764666506B657B4776466B618691D
:1015A0000300185902005764666506C206265724D0
:1015B000776466262322CC20440023BB37D19212C5
:1015C000CCB04300924BB86820008248B8E60400D3
:1015D0008245B85E0400824938601C2FC656923E90
:1015E000F24438601C2F38302C2FB16106E30460C0
:1015F0000450F230284E1200C6429229C4C0920311
:10160000B04E820D304EC647820AC4C08220C4400C
:10161000820638F808007647D64F9219C460927651
:10162000184E1000D4448271F271B84E0400820446
:1016300030F1C64F920CC4508218386E0C00B9E0DD
:101640002C2FB9650C00B93E0C00F20F065E38EE87
:101650000C00C4E092D0C460920738680400C667EA
:10166000925004E0F20206E61879070018690600B5
:101670005774E6768212286D0800062D0C301C2F58
:101680000C40402F0C5011000BDF0100C4208205DC
:10169000062D8B640700F23F062D1438CBBA0100EB
:1016A000C4208205062D8B640700F235C4E0821148
:1016B000B87E1800820A382E1C00063E064D0C50DB
:1016C0001C2F066BF170F227062D8B640700F223A6
:1016D000C4C092133870402F5C70F000CC70E000F2
:1016E000820C103A062D543F24325731CBBA0100F8
:1016F000062D04330B2A0800062D8B640700F20B1D
:10170000062D8B640700F207066E284E1400C64BA8
:10171000929EF28C58C11800588108002C102800A5
:10172000E1F000003C101C00D9C10C00C9A104006C
:10173000B8B2700006E29204B8B26C008260386BF6
:101740000C0018760D00D471820628AB080034A175
:10175000F7AFF20204A0185605001876040057549B
:101760006657187606001846070013AA577866755C
:10177000574C063A062E743166478B98070086C28E
:10178000823EC4A038DC04008211187D0D00186D63
:101790000C00577466765C70FFC06C700011997D08
:1017A0000C007774997D0D00F20E382B0400287B15
:1017B000080027640C3014003657263D0441235599
:1017C000CBC7010004B4286C080026BE063E064BB9
:1017D0000456062C0BDF0100992D10007724992D5B
:1017E0001100185E0A000476062C063E064B0460C3
:1017F000B1712B150800062C8B64070058C10C0032
:1018000048A104002C101C00E1F000003C10140062
:10181000D9C1040006E2382250003421EBEE010069
:1018200004300642062E8B98070086D2821E04C41E
:10183000286D080026CE063E064C04560BDF01003C
:10184000387D0400063E992710007724992711005F
:10185000185E0A000476062D064C0460B1712B1543
:101860000800062D8B64070058C104002C101400DA
:10187000E1F000003C101800D9C10800B9B1040023
:1018800006E238225000EBEE010004300642062E3C
:101890008B98070086D28227187E1E0004C45C70D5
:1018A000FC0038BD040026CE997E1E00286D08007D
:1018B000063E064C04560BDF0100992B10007724DE
:1018C000992B1100185E0A00186E09000476063E76
:1018D000064C062DB1712B150800062D8B640700F0
:1018E0000420F202142258C1080038B104002C1060
:1018F0001800E1F0187085303C101400DC70100006
:10190000D9C10400B1B106E28AAE010038725400B8
:101910003860B82F284260003F360700C430385284
:1019200058002217C67692073870BC2F3F77050003
:10193000C470220F3870BC2FC65792313870B42F44
:1019400018370E0018770F0057746673C674C227D5
:101950003870B42F18370E0018770F00577466735D
:10196000283E6200A97E6000C637B203A97E6200ED
:10197000B96E5400C4703860BC2F187E9100B96EE7
:1019800058009209C470920B0471990E9000997ED0
:101990009100F205C4708203990E91003870BC2F3B
:1019A000386E48003F360700C4301239A830743012
:1019B000A90E64009230282E6000383E580026544C
:1019C0002632C6359228F85E34002225C667922357
:1019D000186E4700047126761377C676C203997E87
:1019E0004700187E4700C473C20E286E4C00287E44
:1019F000360026762377C676CAD70000A97E4C002B
:101A0000FAD30000C4739AD00000062E2BF5010013
:101A1000FACB0000990E4700FAC70000155626576A
:101A2000C4502AA00000385E50003F550700C45043
:101A30001A990000185E1E000645D44482095C50C5
:101A4000FB00995E1E00285E4E00A95E4C00785E89
:101A50004000284E4200E75126543F660700B97EF9
:101A60004800187E1800A95E4400285E66002366C0
:101A7000C473A96E64002665990E4600A96E6600BF
:101A8000990E4700C23A28DE4C00287E4E00C67DE3
:101A9000C20A287E3600267D2377C67DC22EA97E07
:101AA0004C00F22B282E360006322B970F00063DF5
:101AB000CB860F00262D2322C62DC21FA92E4C0037
:101AC000F21C306D382D0400B96E7000CBBE0100E1
:101AD000A87E64008206D4C182043471A97E6400A9
:101AE000382D0400CBBE0100287E68003672062D1A
:101AF000A97E68002BC50700B8DE7000822D38CDA6
:101B00000C00186C0500187C040057646667187C8C
:101B10000600182C070057786676572C6627EBEEE0
:101B20000100187C0D00186C0C005774667606C70F
:101B300057C4777466C723CC067C5473286D08009D
:101B40001677F77F26763860BC2F36762672C470FB
:101B500002B9FA8C01001471A97E3400990E1F009D
:101B6000F223A90E6400F220307DC470B97E6C00AF
:101B70009203A90E6A00382D0400CBBE0100A87E96
:101B800064008206D4C182043471A97E6400382DB9
:101B90000400CBBE0100287E68003672062DA97EA7
:101BA00068002BC50700B8DE6C00823138CD0C0010
:101BB00038B0BC2F186C0500187C040057646667A9
:101BC000187C0600182C070057786676572C662775
:101BD000EBEE0100187C0D00186C0C005774667653
:101BE00006C757C4777466C723CC067C5473167730
:101BF000286D0800F77F26763F770B003672C47099
